:020000040000FA
:04000000B6EF00F067
:100008005482D9CF05F0DACF06F00F0112A91CD01F
:100018008EBC02D0839483928EA802D083A20FD084
:10002800899425EE04F0010EDBBE08D0000EDE5CDC
:10003800020EDE58D8A002D0899201D089828EB8EB
:1000480083B201D08984129912A184D08EB883B268
:1000580089929050FF0A096E8E50FF0A086E04C5F7
:100068000AF005C50BF00BBE04D0020E0B5CD8B02D
:100078002CD00A4A0B2A0AC004F50BC005F502C5A4
:100088000AF003C50BF0060E0A24D96E050E0B20E4
:10009800DA6E09C0DFFF060E0A24D96E070E0B20A0
:1000A800DA6E08C0DFFF0A4A0B2AFF0E016E010E46
:1000B800026E0AC003F00BC004F001500316025090
:1000C800041603C002F504C003F58EB883B2898410
:1000D80089848EA0FED78EA802D083A202D08994EC
:1000E80001D0898425EE04F0010EDBBE08D0000E95
:1000F800DE5C020EDE58D8A002D0899201D0898237
:1001080008B80CD025D0838202D0838405D083948C
:100118001FD083A21DD0839483921AD00950016EF8
:10012800026A0250000AD8A413D00150040AD8B4B5
:10013800F0D7100AD8B4EDD7340AD8B4E4D71F0AD8
:10014800D8B4EAD77F0AD8B4E0D71F0AD8B4DFD723
:100158000F0112910E01CA9906C0DAFF05C0D9FF36
:1001680054921100C2EF49F045C0D9FF46C0DAFFEA
:10017800000EDE6E000EDD6E47C00CF04EEC46F051
:100188000CC0BCF00DC0BDF00001BDAF02D00B0E1D
:100198001200D890BC35D96EBD35DA6E8C0ED926D2
:1001A800010EDA22DECFD6F0DDCFD7F0D651D71147
:1001B800D8A402D00C0E120045C0D9FF46C0DAFF01
:1001C800D6C0DEFFD7C0DDFFD6C0D9FFD7C0DAFF63
:1001D800DF50D8B415D020EE01F0D651D926D7512A
:1001E800DA22DF5049EC5AF00001C86FC8B108D0D4
:1001F8004850D8A4C8A502D00A0E1200000E12005A
:10020800D6C0D9FFD7C0DAFF000EDF6E20EE01F0AE
:10021800D651D926D751DA22BCC0DFFF20EE01F033
:10022800D651D926D751DA22DF50CEEC3FF0000163
:10023800C86FC8A102D0030E12004850D8B402D02B
:10024800C8B5DAD7000ECF6F000ED06F000ED16F91
:10025800000ED26FD6C060F0D7C061F0000E626F9A
:10026800000E636F000E646F000E656F50EC35F082
:100278000001D56FD505D8A4E6D0000ED46F000EC6
:10028800D36FD45105E1040ED35DD8B098D001D016
:1002980096D0D3C084F0D4C085F0843B853BF00E63
:1002A800851784510F0B8513F00E8417D6C086F07E
:1002B800D7C087F08451862785518723EC0E862581
:1002C800C96F010E8721CA6F20EE04F0C951D926E3
:1002D800CA51DA22DF50D8A408D0000EAE6F000E43
:1002E800AF6F000EB06F000E58D020EE09F0C95164
:1002F800D926CA51DA22DF50846F8451866F856B04
:1003080020EE0AF0C951D926CA51DA22DF50876F88
:1003180087C088F0896B8A6B8B6B89C08BF088C02B
:100328008AF0896B886B20EE0BF0C951D926CA5127
:10033800DA22DF508C6F8CC08DF08E6B8F6B906BD8
:100348008DC090F08F6B8E6B8D6B88518D11916F76
:1003580089518E11926F8A518F11936F8B51901121
:10036800946F85519111956F86519211966F000E79
:100378009311976F000E9411986F20EE08F0C951F1
:10038800D926CA51DA22DF50996F99519511AE6F6B
:100398009651AF6F9751B06F9851B16FD351040D0B
:1003A800F3509E0FD96EDA6AAEC0DEFFAFC0DEFF33
:1003B800B0C0DEFFB1C0DEFFD34BD42B62D7000E36
:1003C800D46F000ED36FD351D411D8B403D0D30750
:1003D800D8A0D407D351040DF3509E0FD96EDA6A12
:1003E800DECFCFF0DECFD0F0DECFD1F0DECFD2F04F
:1003F800CF51D011D111D211D8A405D0000EB36FAE
:10040800020EB26F13D0D6C060F0D7C061F0CFC073
:1004180062F0D0C063F0D1C064F0D2C065F050EC97
:1004280035F00001846F8451B26FB36BB2C0D5F060
:10043800D551D8B408D0D34BD42BD45104E1040EF1
:10044800D35DD8A0C7D7030ED519D8A402D0010E02
:100458001200D551D8B402D00D0E120020EE3AF099
:10046800D651D926D751DA22DF50846F8451866F4E
:10047800856B20EE39F0D651D926D751DA22DF50D4
:10048800876F87518513000E8613020E8619851112
:10049800D8A4E2D720EE45F0D651D926D751DA2292
:1004A800DF50846F8451866F856B20EE44F0D651FF
:1004B800D926D751DA22DF50876F87518513000E6E
:1004C800861385C0CBF086C0CCF0CD6BCE6BCB51FC
:1004D800CC11CD11CE11D8A459D020EE53F0D6515D
:1004E800D926D751DA22DF50846F8451866F856B05
:1004F80020EE54F0D651D926D751DA22DF50876F33
:1005080087C088F0896B8A6B8B6B89C08BF088C039
:100518008AF0896B886B20EE55F0D651D926D751D1
:10052800DA22DF508C6F8CC08DF08E6B8F6B906BE6
:100538008DC090F08F6B8E6B8D6B88518D11916F84
:1005480089518E11926F8A518F11936F8B5190112F
:10055800946F85519111956F86519211966F000E87
:100568009311976F000E9411986F20EE52F0D651A8
:10057800D926D751DA22DF50996F99519511CB6F4F
:100588009651CC6F9751CD6F9851CE6F20EE16F0E3
:10059800D651D926D751DA22CBC0DEFFCCC0DEFF38
:1005A800CDC0DEFFCEC0DEFF20EE3EF0D651D9260C
:1005B800D751DA2210EE03F0D651E126D751E222C4
:1005C800DFCFE7FF20EE03F0D651D926D751DA2244
:1005D800DE04D8B40AD020EE03F0D651D926D7517C
:1005E800DA22020EDE18D8A437D7CBC00CF0CCC064
:1005F8000DF0CDC00EF0CEC00FF020EE03F0D651B6
:10060800D926D751DA22DF50846F8451106E116ACF
:10061800126A136AC1EC55F00CC0CBF00DC0CCF0D7
:100628000EC0CDF00FC0CEF0000120EE3BF0D65149
:10063800D926D751DA2210EE02F0D651E126D75149
:10064800E222DFCFE7FF20EE02F0D651D926D751BC
:10065800DA22DF50D8B400D720EE02F0D651D926DE
:10066800D751DA22DF50846F20EE02F0D651D92616
:10067800D751DA22DF50856F850584150009D8A483
:10068800EBD620EE40F0D651D926D751DA22DF50EA
:10069800846F8451866F856B20EE3FF0D651D92642
:1006A800D751DA22DF50876F87518513000E8613E2
:1006B80020EE08F0D651D926D751DA2285C0DEFFC0
:1006C80086C0DDFF20EE08F0D651D926D751DA22B0
:1006D800DF50846F0F0E8417D8A4BED620EE42F0E8
:1006E800D651D926D751DA22DF50846F8451866FCC
:1006F800856B20EE41F0D651D926D751DA22DF504A
:10070800876F87518513000E861385C0C0F086C099
:10071800C1F0C26BC36BC051C111C211C311D8A4BF
:1007280059D020EE4FF0D651D926D751DA22DF50D2
:10073800846F8451866F856B20EE50F0D651D92690
:10074800D751DA22DF50876F87C088F0896B8A6BB0
:100758008B6B89C08BF088C08AF0896B886B20EE20
:1007680051F0D651D926D751DA22DF508C6F8CC080
:100778008DF08E6B8F6B906B8DC090F08F6B8E6B46
:100788008D6B88518D11916F89518E11926F8A519D
:100798008F11936F8B519011946F85519111956FB3
:1007A80086519211966F000E9311976F000E941157
:1007B800986F20EE4EF0D651D926D751DA22DF5065
:1007C800996F99519511C06F9651C16F9751C26F2A
:1007D8009851C36F20EE3CF0D651D926D751DA2272
:1007E800DF50846F20EE3DF0D651D926D751DA225A
:1007F800DF50856F8451BE6F85C0BFF0BE51BF11F9
:10080800D8B42AD620EE08F0D651D926D751DA2204
:10081800DECF84F0DDCF85F0040E866FD890853367
:100828008433862FFBD7BE518425876FBF5185211E
:10083800886F896BD8B0892B8A6BCB518725B86FA5
:10084800CC518821B96FCD518921BA6FCE518A21F7
:10085800BB6FB851C05DB951C159BA51C259BB51EA
:10086800C359D8A0F9D5B851C05D0C6EB951C1595A
:100878000D6EBA51C2590E6EBB51C3590F6E20EEA0
:1008880002F0D651D926D751DA22DF50846F84512D
:10089800106E116A126A136ABFEC51F00CC0C4F0F2
:1008A8000DC0C5F00EC0C6F00FC0C7F00001C4519E
:1008B800C511C611C711D8B4CFD5010ED56FC75110
:1008C800C61106E1F60EC45D0F0EC559D8A002D0B8
:1008D800020ED56FC751C61106E1F60EC45DFF0EB4
:1008E800C559D8A002D0030ED56F020EC425846F57
:1008F800000EC521856F000EC621866F000EC72128
:10090800876F20EE12F0D651D926D751DA2284C04B
:10091800DEFF85C0DEFF86C0DEFF87C0DEFF20EE7B
:100928001AF0D651D926D751DA22CFC0DEFFD0C06F
:10093800DEFFD1C0DEFFD2C0DEFFBE51CF25846FFF
:10094800BF51D021856F000ED121866F000ED221B4
:10095800876F20EE1EF0D651D926D751DA2284C0EF
:10096800DEFF85C0DEFF86C0DEFF87C0DEFFB85130
:10097800CF25846FB951D021856FBA51D121866FA7
:10098800BB51D221876F20EE26F0D651D926D751F8
:10099800DA2284C0DEFF85C0DEFF86C0DEFF87C0A6
:1009A800DEFF030ED519D8A490D020EE08F0D6515A
:1009B800D926D751DA22DE50DE10D8A44DD520EE44
:1009C8005BF0D651D926D751DA22DF50846F845193
:1009D800866F856B20EE5CF0D651D926D751DA2286
:1009E800DF50876F87C088F0896B8A6B8B6B89C0F3
:1009F8008BF088C08AF0896B886B20EE5DF0D65149
:100A0800D926D751DA22DF508C6F8CC08DF08E6BCF
:100A18008F6B906B8DC090F08F6B8E6B8D6B885148
:100A28008D11916F89518E11926F8A518F11936F29
:100A38008B519011946F85519111956F8651921138
:100A4800966F000E9311976F000E9411986F20EE19
:100A58005AF0D651D926D751DA22DF50996F9951D9
:100A680095119A6F96519B6F97519C6F98519D6FF6
:100A780020EE22F0D651D926D751DA229AC0DEFFCD
:100A88009BC0DEFF9CC0DEFF9DC0DEFF20EE12F0A3
:100A9800D651D926D751DA22DECF84F0DECF85F0C1
:100AA800DECF86F0DECF87F0020ED8908437853708
:100AB80086378737E82EF9D784C0B4F085C0B5F0FB
:100AC80086C0B6F087C0B7F091D020EE08F0D651B6
:100AD800D926D751DA22DE50DE10D8B4BDD420EEA4
:100AE8001EF0D651D926D751DA22DECF84F0DECFD8
:100AF80085F0DECF86F0DECF87F0CB518425886F76
:100B0800CC518521896FCD5186218A6FCE5187219D
:100B18008B6F20EE22F0D651D926D751DA2288C021
:100B2800DEFF89C0DEFF8AC0DEFF8BC0DEFF020E5B
:100B3800D519D8B444D020EE12F0D651D926D751C1
:100B4800DA22DECF84F0DECF85F0DECF86F0DECF8E
:100B580087F0010E8415886F000E8515896F000EC9
:100B680086158A6F000E87158B6F20EE12F0D6510E
:100B7800D926D751DA22DECF0CF0DECF0DF0DECF4A
:100B88000EF0DECF0FF0030E106E000E116E000E89
:100B9800126E000E136EC1EC55F0D8900F320E3263
:100BA8000D320C32000188510C24B46F89510D208C
:100BB800B56F8A510E20B66F8B510F2016D020EEDC
:100BC80012F0D651D926D751DA22DECF84F0DECF03
:100BD80085F0DECF86F0DECF87F0D8908435B46F0D
:100BE8008535B56F8635B66F8735B76FFF0EB42577
:100BF800846F010EB521856F000EB621866F000E39
:100C0800B721876F0A0E05D0D8908733863385338E
:100C18008433E82EF9D720EE16F0D651D926D751CD
:100C2800DA228451DE5C8551DE588651DE588751C0
:100C3800DE58D8A011D420EE0EF0D651D926D751BF
:100C4800DA22FF0EDE6EFF0EDE6EFF0EDE6EFF0E88
:100C5800DD6EDD52DD5210EE0AF0D651E126D75195
:100C6800E222DECFE6FFDECFE6FFDECFE6FFDECF15
:100C7800E6FF20EE05F0D651D926D751DA22800EAC
:100C8800DF6E030ED519D8A4F1D120EE5FF0D6514E
:100C9800D926D751DA22DF50846F8451866F856B4D
:100CA80020EE5EF0D651D926D751DA22DF50876F71
:100CB80087518513000E861385058611D8A4D6D1D1
:100CC800D6C03AF0D7C03BF0010ECF253C6E000EDF
:100CD800D0213D6E000ED1213E6E000ED2213F6E16
:100CE80087EC4EF00009D8A4C1D1000120EE05F030
:100CF800D651D926D751DA22000EDF6E22EE2DF01A
:100D0800D651D926D751DA22DF50846F8451866FA5
:100D1800856B22EE2CF0D651D926D751DA22DF5036
:100D2800876F87518513000E8613550E851903E1C9
:100D3800AA0E8619D8A49AD120EE2FF0D651D9261A
:100D4800D751DA22DF50846F8451866F856B20EE8D
:100D580030F0D651D926D751DA22DF50876F87C0B5
:100D680088F0896B8A6B8B6B89C08BF088C08AF09E
:100D7800896B886B20EE31F0D651D926D751DA220B
:100D8800DF508C6F8CC08DF08E6B8F6B906B8DC02D
:100D980090F08F6B8E6B8D6B88518D11916F89518F
:100DA8008E11926F8A518F11936F8B519011946F9E
:100DB80085519111956F86519211966F000E93117E
:100DC800976F000E9411986F20EE2EF0D651D92609
:100DD800D751DA22DF50996F995195119A6F965130
:100DE8009B6F97519C6F98519D6F520E9A1909E10C
:100DF800520E9B1906E1610E9C1903E1410E9D19E3
:100E0800D8A434D122EE13F0D651D926D751DA22FC
:100E1800DF50846F8451866F856B22EE14F0D651B3
:100E2800D926D751DA22DF50876F87C088F0896BBF
:100E38008A6B8B6B89C08BF088C08AF0896B886B52
:100E480022EE15F0D651D926D751DA22DF508C6F11
:100E58008CC08DF08E6B8F6B906B8DC090F08F6B0C
:100E68008E6B8D6B88518D11916F89518E11926F98
:100E78008A518F11936F8B519011946F85519111F5
:100E8800956F86519211966F000E9311976F000E11
:100E98009411986F22EE12F0D651D926D751DA2242
:100EA800DF50996F995195119A6F96519B6F975191
:100EB8009C6F98519D6F720E9A1909E1720E9B19D9
:100EC80006E1410E9C1903E1610E9D19D8A4CED00C
:100ED80022EE17F0D651D926D751DA22DF50846F87
:100EE8008451866F856B22EE18F0D651D926D751DA
:100EF800DA22DF50876F87C088F0896B8A6B8B6B2B
:100F080089C08BF088C08AF0896B886B22EE19F053
:100F1800D651D926D751DA22DF508C6F8CC08DF08C
:100F28008E6B8F6B906B8DC090F08F6B8E6B8D6B13
:100F380088518D11916F89518E11926F8A518F113D
:100F4800936F8B519011946F85519111956F8651C4
:100F58009211966F000E9311976F000E9411986F6F
:100F680022EE16F0D651D926D751DA22DF50996FE2
:100F7800995195119A6F96519B6F97519C6F985103
:100F88009D6F20EE0EF0D651D926D751DA229AC09D
:100F9800DEFF9BC0DEFF9CC0DEFF9DC0DEFF22EEB1
:100FA8001BF0D651D926D751DA22DF50846F8451ED
:100FB800866F856B22EE1CF0D651D926D751DA22DE
:100FC800DF50876F87C088F0896B8A6B8B6B89C00D
:100FD8008BF088C08AF0896B886B22EE1DF0D651A1
:100FE800D926D751DA22DF508C6F8CC08DF08E6BEA
:100FF8008F6B906B8DC090F08F6B8E6B8D6B885163
:101008008D11916F89518E11926F8A518F11936F43
:101018008B519011946F85519111956F8651921152
:10102800966F000E9311976F000E9411986F22EE31
:101038001AF0D651D926D751DA22DF50996F995133
:1010480095119A6F96519B6F97519C6F98519D6F10
:1010580020EE0AF0D651D926D751DA229AC0DEFFFF
:101068009BC0DEFF9CC0DEFF9DC0DEFFD6C0D9FF5F
:10107800D7C0DAFFD5C0DFFF01018A4B8B2B0001F7
:1010880020EE06F0D651D926D751DA228AC1DEFFE2
:101098008BC1DDFF02EF01F0000E0D6E000E0C6E2D
:1010A8000AEC5AF00F0B0101EB6F000EA06F070E50
:1010B8008C6E010EEA6F000EA56F0F0E0F01596FAF
:1010C800000E116F000E196F000E216F000E266FB3
:1010D800000E2E6F886889688A688A8E8890889240
:1010E8008382020E526EA5EC58F088948384889C03
:1010F800839C889E838E8B688968860E0001606F4A
:10110800FB0E616FA60E626FFF0E636FF70E646FC2
:10111800FE0E656F2D0E666FFF0E676F21EC5AF09D
:101128008AEC58F017D0B80E0001606FFE0E616FA0
:101138008FCF62F0636B21EC5AF0290E0101E46F46
:10114800960EE36F7F0EE82EFED7E32FFCD7E42F31
:10115800FAD704008FB2E7D713EC48F00101EB6F20
:101168009F0E0001606FFC0E616FEBC162F0636B54
:1011780021EC5AF00400290E0101E46F960EE36F8A
:101188007F0EE82EFED7E32FFCD7E42FFAD7D250F4
:10119800F00B0109D26ED09E0E01C691CF0ECF166C
:1011A800CF82CF80C2890F01138113891489F28EEF
:1011B8000E01BA89DAEC4EF083928394BEEC4BF0C0
:1011C800BEEC4BF0000E0C6E340E17EC56F0480EC9
:1011D800106EFF0E116E3EEC52F0A60E106EFF0E52
:1011E800116E3EEC52F0000E0C6E390E17EC56F0F4
:1011F8008380040069EC31F041EC42F0F0EC50F0EF
:10120800000E0C6E800E17EC56F00101EB510F0D1D
:10121800340EF324106E0D0EF420116E3EEC52F0D5
:1012280001019F51D8B4EDD0D40E0001606FFD0EBE
:10123800616F21EC5AF07CEC52F010C0AAF311C097
:10124800ABF312C0ACF313C0ADF30301AA51AB1159
:10125800AC11AD11D8A419D0FC0E0001606FFC0EC2
:10126800616FAAC362F0ABC363F0ACC364F0ADC3F3
:1012780065F021EC5AF00A0E0F6E000E106E000E8B
:10128800116E000E126E96EC55F0000E0301AF6F52
:10129800000EAE6FAFBF06D0AF511DE1040EAE5DBC
:1012A800D8B019D0DB0E0001606FFF0E616FAA0E77
:1012B8000301AE25D96E030EAF21DA6EDF500101AE
:1012C800E36FE3510001626F636B21EC5AF0030195
:1012D800AE4BAF2BDFD7B40E0001606FFB0E616F12
:1012E80021EC5AF0540E0001606FFC0E616F21EC86
:1012F8005AF022EE10F000EECBF01F0EDBCFEBFF22
:10130800E806FCE2D30E0001EB6FFF0EEC6FC3ECB6
:1013180032F0CBC06CF1CCC06DF1CDC06EF1CEC057
:101328006FF101016C516D116E116F11D8B469D054
:101338003A0E0001606FFC0E616F6CC162F06DC106
:1013480063F06EC164F06FC165F021EC5AF0100EC5
:101358000001A46F020EA56F6CC1E4F16DC1E5F147
:101368006EC1E6F10101E36B000EE3250001A66FF3
:10137800010E0101E4210001A76F000E0101E52122
:101388000001A86F000E0101E6210001A96FCDEC54
:101398000FF0100E8C6F020E8D6F340E8E6F0B0EC9
:1013A8008F6F000E916F080E906FA80E926F030E4C
:1013B800936FD2EC12F0000E0301B16F000EB06F04
:1013C800B1BF06D0B1511DE1080EB05DD8B019D03B
:1013D800D70E0001606FFF0E616F340E0301B02558
:1013E800D96E0B0EB121DA6EDF500101E36FE351C4
:1013F8000001626F636B21EC5AF00301B04BB12B13
:10140800DFD70101A5AF12D08A6883928382290EA3
:101418000101E46F960EE36F7F0EE82EFED7E32FEF
:10142800FCD7E42FFAD7EDEC3DF0EFD7EA51D8B46A
:101438000CD0F40E0001606FFD0E616F21EC5AF0C4
:10144800020E0101A46F220E0BD0E40E0001606FA2
:10145800FD0E616F21EC5AF0010E0101A46F040E1C
:10146800A36F000E0301A56F000EA46F000EB56FE9
:10147800000EB46F010EB36FB4BF06D0B4516EE165
:10148800040EB35DD8B06AD0B3C30CF0B4C30DF08A
:10149800000E0F6E0F0E0E6EB9EC59F0240E0C24D0
:1014A800126E0E0E0D20136E12EC57F0135004E15D
:1014B800030E125CD8A04ED0B3C30CF0B4C30DF029
:1014C800000E0F6E0F0E0E6EB9EC59F0240E0C24A0
:1014D8000301A16F0E0E0D20A26F420E0001606F76
:1014E800FE0E616FA1C362F0A2C363F021EC5AF053
:1014F800B3C3E3F1B4C3E4F1050ED8900101E337B7
:10150800E437E82EFAD7100EE3250001D86F020E53
:101518000101E4210001D96FB3C30CF0B4C30DF08D
:10152800000E0F6E0F0E0E6EB9EC59F0240E0C243F
:101538000001DA6F0E0E0D20DB6F030EDC6F44EC3A
:1015480018F00101E56FE5510301A66FA76BA651DD
:10155800DAEC54F00301B34BB42B8ED7020E010121
:10156800A119D8A404D00F01108B070E2D6F839EEC
:10157800000E0C6EC00E17EC56F052EC59F0000E2F
:101588000C6EC00E17EC56F0940E106EFF0E116E16
:101598003EEC52F021D18EA8899464EC5AF00C509C
:1015A8000D10D8B4F8D0B5C3A3F3B20E0C6E030E69
:1015B8000D6E5FEC50F00301B56F350EB519D8A468
:1015C80007D0B40E0001606FFB0E616F21EC5AF07A
:1015D800360E0001606FFF0E616FB5C362F0636B7A
:1015E8008DA004D00101E36BE32B02D00101E36B72
:1015F800E3510001646F656B21EC5AF00301B2A955
:1016080028D0600EB519D8A424D05F0EA319D8A489
:1016180020D052500209526E2BEE34F0A4C1DFFFE5
:101628002BEE35F0A3C1DFFF8384000E0001876F26
:10163800020E866FB0EC38F083945250FD0B526E58
:10164800000E0101AB6F93EC59F0000E0301B56F6A
:10165800C3D00101EA51D8B44AD00301B251100BEA
:1016680000019E6F000E9F6F0301B5510BEC34F023
:101678009EC0B6F39FC0B7F3080E0301B619B711A1
:10168800D8B400F0070E0301B619B711D8B4A3EC0B
:1016980053F00301B605B711D8B4B9EC52F0020EF5
:1016A8000301B619B711D8B4F1EC3CF0030E0301ED
:1016B800B619B711D8A406D08AEC2BF0E2C0A4F36F
:1016C800E3C0A5F3050E0301B619B711D8A406D0D7
:1016D8007EEC36F0EDC0A4F3EEC0A5F3090E0301CD
:1016E800B619B711D8A478D051EC5AF075D00301C7
:1016F800B251100B0C6E000E0D6EB5517BEC1FF045
:101708000CC0B6F30DC0B7F3070E0301B619B71135
:10171800D8B431EC53F0020E0301B619B711D8B49E
:101728003BEC55F00301B605B711D8B4B5EC43F05E
:10173800030E0301B619B711D8B47BEC51F0040EAF
:101748000301B619B711D8B450EC58F0050E0301CF
:10175800B619B711D8B4A9EC48F0060E0301B619AA
:10176800B711D8B45FEC5AF0080E0301B619B711D7
:10177800D8B4DFEC3EF0090E0301B619B711D8B49E
:10178800C7EC4AF00A0E0301B619B711D8A424D041
:1017980045EC4AF021D013EC48F00101A06FA151AB
:1017A800D8B41AD0EB51A019D8B416D0838E000E35
:1017B8000C6EC00E17EC56F052EC59F0000E0C6E81
:1017C800C00E17EC56F0030E106EFF0E116E3EECB5
:1017D80052F0A0C1EBF132D08FB230D0050E030128
:1017E800A419A511D8B42AD0D6D6B80E0001606FB6
:1017F800FE0E616F8FCF62F0636B21EC5AF0290EF9
:101808000101E46F960EE36F7F0EE82EFED7E32FFB
:10181800FCD7E42FFAD70400000E0C6EC00E17ECAC
:1018280056F052EC59F0000E0C6EC00E17EC56F044
:10183800500E106EFF0E116E3EEC52F08FB2D5D7DF
:10184800290E0101E46F960EE36F7F0EE82EFED796
:10185800E32FFCD7E42FFAD783948392000E00017C
:10186800D86F000ED96FB60EDA6FFB0EDB6F000E65
:10187800DC6F33EC4EF0BDD4A6C0B8F0A7C0B9F009
:10188800AA51D96EDA6A000EDE6E000EDD6EA4C0B3
:101898000DF0A5C00EF015EC50F00001B76FB75170
:1018A800D8B402D0B751120020EE05F0A451D926C1
:1018B800A551DA22DF50D8B408D020EE05F0A451A3
:1018C800D926A551DA22DF50120020EE04F0A451E7
:1018D800D926A551DA22DFB202D0070E120020EE77
:1018E80006F0A451D926A551DA2210EE06F0A4512B
:1018F800E126A551E222E6CFAFF0E6CFB0F0E6CF81
:10190800B1F0E6CFB2F0A851AF25B36FA951B0211D
:10191800B46F000EB121B56F000EB221B66FDE5064
:10192800B35DDE50B459DE50B559DE50B659D8B063
:10193800F8D2000EA96F000EA86FF3D220EE06F0C1
:10194800A451D926A551DA22FF0EDE14AB6F010E81
:10195800DE14AC6F000EDE14AD6F000EDE14AE6F39
:10196800AB51AC11AD11AE11D8A443D220EE06F0A4
:10197800A451D926A551DA22DECFABF0DECFACF0E8
:10198800DECFADF0DECFAEF00A0E05D0D890AE3384
:10199800AD33AC33AB33E82EF9D7A4C0D9FFA5C01B
:1019A800DAFF10EE02F0DE50E126DD50E222E750C9
:1019B800AF6FAF05AB15BA6FBA51D8A4A4D020EE5B
:1019C80006F0A451D926A551DA22DE50DE10DE1029
:1019D800DE10D8A427D020EE0EF0A451D926A551A8
:1019E800DA22DECFC1F0DECFC2F0DECFC3F0DECF29
:1019F800C4F0C151C211C311C411D8A433D0A4C0BA
:101A0800D9FFA5C0DAFFDECF91F0DDCF92F0000E4E
:101A1800936F000E946F000E956F000E966F23EC77
:101A28002DF018D0A4C0D9FFA5C0DAFFDECF91F001
:101A3800DDCF92F020EE12F0A451D926A551DA227A
:101A4800DECF93F0DECF94F0DECF95F0DECF96F0C8
:101A580023EC2DF091C0C1F092C0C2F093C0C3F046
:101A680094C0C4F0C151C211C311C411D8B45DD21D
:101A7800C105C211C311C411D8A40AD020EE05F0C3
:101A8800A451D926A551DA22020EDF6E020E1200E9
:101A9800C12911E1C2290FE1C3290DE1C429D8A444
:101AA8000AD020EE05F0A451D926A551DA22010E5C
:101AB800DF6E010E120020EE12F0A451D926A551B6
:101AC800DA22C1C0DEFFC2C0DEFFC3C0DEFFC4C071
:101AD800DEFF20EE0EF0A451D926A551DA22DE5001
:101AE800DE10DE10DE10D8A40ED020EE0EF0A451C9
:101AF800D926A551DA22C1C0DEFFC2C0DEFFC3C0AD
:101B0800DEFFC4C0DEFF20EE16F0A451D926A55191
:101B1800DA22A4C0E1FFA5C0E2FF00EE2AF0E650F9
:101B2800E926E550EA22DE50EE1817E1DE50EE18FD
:101B380014E1DE50EE1811E1DE50EE18D8A40DD0F5
:101B4800A4C0D9FFA5C0DAFFDECF25F0DDCF26F08F
:101B580066EC44F00009D8A48BD1A4C0D9FFA5C075
:101B6800DAFFDECF18F0DDCF19F0000120EE12F019
:101B7800A451D926A551DA22DECF1AF0DECF1BF008
:101B8800DECF1CF0DECF1DF0D6EC4DF018C0BDF056
:101B980019C0BEF01AC0BFF01BC0C0F00001BD5193
:101BA800BE11BF11C011D8B469D7BA51BD27000EF4
:101BB800BE23BF23C023A8C0ABF0A9C0ACF0090E58
:101BC800AD6FD890AC33AB33AD2FFBD7ABC0BBF008
:101BD800ACC0BCF0BB51BC11D8B4C7D0BA51BB25FE
:101BE800AB6F000EBC21AC6FA4C0D9FFA5C0DAFF53
:101BF80010EE02F0DE50E126DD50E222E750AD6F34
:101C0800AE6BAB51AD5DAC51AE59D8B012D0A4C0DB
:101C1800D9FFA5C0DAFF10EE02F0DE50E126DD5054
:101C2800E222E750AB6FBA51AB5DBB6FBC6BD8A07B
:101C3800BC07B8C01BF0B9C01CF0BDC01DF0BEC0C9
:101C48001EF0BFC01FF0C0C020F0BBC021F0BCC058
:101C580022F0A4C0D9FFA5C0DAFF10EE01F0DE50D3
:101C6800E126DD50E222E7503BEC49F00009D8A418
:101C7800FFD00001BB51AB6FBC51AC6FAD6BAE6B0D
:101C8800A4C0D9FFA5C0DAFF10EE2AF0DE50E12685
:101C9800DD50E222E6CFAFF0E6CFB0F0E6CFB1F00C
:101CA800E6CFB2F0BD51AF5DB36FBE51B059B46F5E
:101CB800BF51B159B56FC051B259B66FAB51B35D91
:101CC800AC51B459AD51B559AE51B659D8B03ED052
:101CD800A4C0D9FFA5C0DAFFDECFABF0DDCFACF0F2
:101CE8002E0EAB250C6E000EAC210D6EA4C0D9FFD4
:101CF800A5C0DAFF10EE2AF0DE50E126DD50E22220
:101D0800E6CFADF0E5CFAEF0BD51AD5FBE51AE5BF5
:101D1800090ED890AD37AE37E82EFBD7AD51B825B0
:101D28000E6EAE51B9210F6E020E116E000E106EBE
:101D380076EC57F0A4C0D9FFA5C0DAFF10EE04F086
:101D4800DE50E126DD50E222000EE76EBBC0ABF0AC
:101D5800BCC0ACF0090ED890AB37AC37E82EFBD737
:101D6800ABC0C5F0ACC0C6F0C0D020EE0AF0A4519C
:101D7800D926A551DA2210EE06F0A451E126A55184
:101D8800E222DE50E65CDE50E658DE50E658DE50D1
:101D9800E658D8A01FD0A4C0D9FFA5C0DAFFDECF6F
:101DA80025F0DDCF26F066EC44F00009D8A460D019
:101DB800A4C0D9FFA5C0DAFF10EE2AF0DE50E12654
:101DC800DD50E222BDC0E6FFBEC0E6FFBFC0E6FFB1
:101DD800C0C0E6FF000120EE16F0A451D926A55197
:101DE800DA22BDC0DEFFBEC0DEFFBFC0DEFFC0C05E
:101DF800DEFFFF0EAB6F010EAC6F20EE06F0A451B4
:101E0800D926A551DA22DECFADF0DDCFAEF0AB5149
:101E1800AD17AC51AE17AD510008C56FAE51D8A083
:101E2800E82A0208C66FC551A85DC651A959D8B09D
:101E380004D0A8C0C5F0A9C0C6F0A4C0D9FFA5C0E9
:101E4800DAFFDECF3AF0DDCF3BF020EE16F0A451FA
:101E5800D926A551DA22DECF3CF0DECF3DF0DECF29
:101E68003EF0DECF3FF087EC4EF00009D8B402D048
:101E7800000117D6FF0E0001AB6F010EAC6F20EE0C
:101E880006F0A451D926A551DA22DECFADF0DDCF78
:101E9800AEF0AB51AD17AC51AE17A4C0D9FFA5C079
:101EA800DAFFDECFAFF0DDCFB0F0AD51AF27AE51E6
:101EB800B0232E0EAF250C6E000EB0210D6EB8C0EB
:101EC8000EF0B9C00FF0C5C010F0C6C011F076EC26
:101ED80057F0A4C0D9FFA5C0DAFF10EE04F0DE5019
:101EE800E126DD50E222010EE76EC551B827C65142
:101EF800B92320EE06F0A451D926A551DA22C551FE
:101F0800DE26C651DE22000EDE22DE22AA51D96E5E
:101F1800DA6AC551DE26C651DD22C551A85FC65111
:101F2800A95BA851A911D8A409D520EE06F0A4519F
:101F3800D926A551DA2210EE0AF0A451E126A551BE
:101F4800E222DE50E65CDE50E658DE50E658DE500F
:101F5800E658D8B014D020EE06F0A451D926A551E1
:101F6800DA2210EE0AF0A451E126A551E222DECFD2
:101F7800E6FFDECFE6FFDECFE6FFDECFE6FF20EEB0
:101F880004F0A451D926A551DA22000EDB8A000EEE
:101F98001200A4C00DF0A5C00EF015EC50F0000121
:101FA800BE6FBE51D8B402D0BE51120020EE05F06B
:101FB800A451D926A551DA22DF50D8B408D020EE92
:101FC80005F0A451D926A551DA22DF50120020EEDF
:101FD8000AF0A451D926A551DA22A651DE5CA751F0
:101FE800DE58A851DE58A951DE58D8B016D020EED8
:101FF80004F0A451D926A551DA22DFB20ED020EE82
:102008000AF0A451D926A551DA22DECFA6F0DECFF8
:10201800A7F0DECFA8F0DECFA9F020EE06F0A4519D
:10202800D926A551DA22DECFBAF0DECFBBF0DECF5B
:10203800BCF0DECFBDF0000EBF6F000EC06F000E0B
:10204800C16F000EC26F20EE06F0A451D926A5512B
:10205800DA22BFC0DEFFC0C0DEFFC1C0DEFFC2C0E3
:10206800DEFFA651A711A811A911D8B42BD2A4C07C
:10207800D9FFA5C0DAFF10EE02F0DE50E126DD50F0
:10208800E222E750AA6FAAC0ABF0AC6BAD6BAE6BA7
:10209800090ED890AB37AC37AD37AE37E82EF9D745
:1020A800ABC0C3F0ACC0C4F0ADC0C5F0AEC0C6F0A4
:1020B800BA51BB11BC11BD11D8B497D0FF0EA625DB
:1020C8000C6EFF0EA7210D6EFF0EA8210E6EFF0EDF
:1020D800A9210F6EC3C010F0C4C011F0C5C012F022
:1020E800C6C013F0BFEC51F00CC0AAF00DC0ABF0A5
:1020F8000EC0ACF00FC0ADF0FF0E0001BA250C6E9B
:10210800FF0EBB210D6EFF0EBC210E6EFF0EBD2112
:102118000F6EC3C010F0C4C011F0C5C012F0C6C025
:1021280013F0BFEC51F00C500001AA5D0D50AB59F3
:102138000E50AC590F50AD59D8A057D0FF0EC3253B
:10214800AA6FFF0EC421AB6FFF0EC521AC6FFF0E47
:10215800C621AD6FAA1DAE6FAB1DAF6FAC1DB06FC2
:10216800AD1DB16FFF0EBA25B26FFF0EBB21B36F65
:10217800FF0EBC21B46FFF0EBD21B56FAE51B21575
:10218800B66FAF51B315B76FB051B415B86FB15141
:10219800B515B96F20EE06F0A451D926A551DA225B
:1021A800B6C0DEFFB7C0DEFFB8C0DEFFB9C0DEFFD5
:1021B80020EE06F0A451D926A551DA22DE50A65FFA
:1021C800DE50A75BDE50A85BDD50A95B20EE12F065
:1021D800A451D926A551DA22DECFC7F0DECFC8F048
:1021E800DECFC9F0DECFCAF06DD020EE0EF0A451DC
:1021F800D926A551DA22DECFC7F0DECFC8F0DECF70
:10220800C9F0DECFCAF0C751C811C911CA11D8A484
:102218004BD0A4C0D9FFA5C0DAFFDECF91F0DDCF47
:1022280092F0000E936F000E946F000E956F000EE3
:10223800966F23EC2DF091C0C7F092C0C8F093C000
:10224800C9F094C0CAF0C705C811C911CA11D8A4E9
:102258000AD020EE05F0A451D926A551DA22020EA3
:10226800DF6E020E1200C72911E1C8290FE1C92942
:102278000DE1CA29D8A40AD020EE05F0A451D92628
:10228800A551DA22010EDF6E010E120020EE0EF0CB
:10229800A451D926A551DA22C7C0DEFFC8C0DEFF87
:1022A800C9C0DEFFCAC0DEFF20EE12F0A451D92655
:1022B800A551DA22C7C0DEFFC8C0DEFFC9C0DEFFF5
:1022C800CAC0DEFFC751C811C911CA11D8A496D017
:1022D800F9D020EE04F0A451D926A551DA22DFA2C4
:1022E80029D0A4C0D9FFA5C0DAFFDECF91F0DDCF99
:1022F80092F0C7C093F0C8C094F0C9C095F0CAC0A6
:1023080096F023EC2DF091C0C7F092C0C8F093C0AE
:10231800C9F094C0CAF0C751C811C911CA11D8A4CC
:1023280023D0C3C0A6F0C4C0A7F0C5C0A8F0C6C0DB
:10233800A9F06ED0A4C0D9FFA5C0DAFFDECF60F047
:10234800DDCF61F0C7C062F0C8C063F0C9C064F0F7
:10235800CAC065F0B4EC21F060C0C7F061C0C8F035
:1023680062C0C9F063C0CAF00001C72907E1C829E3
:1023780005E1C92903E1CA29D8B47ED7CA51C911D0
:10238800C81104E1020EC75DD8A063D7A4C0D9FF65
:10239800A5C0DAFF10EE12F0DE50E126DD50E22291
:1023A800E650C75DE650C859E650C959E650CA59C3
:1023B800D8B04FD720EE12F0A451D926A551DA2271
:1023C800C7C0DEFFC8C0DEFFC9C0DEFFCAC0DEFF6F
:1023D80020EE06F0A451D926A551DA22C351DE26F3
:1023E800C451DE22C551DE22C651DE22C351A65F8A
:1023F800C451A75BC551A85BC651A95BA651C35D73
:10240800A751C459A851C559A951C659D8A061D7CF
:1024180020EE06F0A451D926A551DA22A651DE26CF
:10242800A751DE22A851DE22A951DE22FF0EA615F1
:10243800AA6F010EA715AB6F000EA815AC6F000EA2
:10244800A915AD6FAA51AB11AC11AD11D8B43AD0E2
:10245800A4C0D9FFA5C0DAFFDECF18F0DDCF19F090
:10246800C7C01AF0C8C01BF0C9C01CF0CAC01DF014
:10247800D6EC4DF018C0BFF019C0C0F01AC0C1F0BA
:102488001BC0C2F00001BF51C011C111C211D8B4A4
:10249800E0D6A6C0AAF0A7C0ABF0A8C0ACF0A9C00F
:1024A800ADF00A0E05D0D890AD33AC33AB33AA33B8
:1024B800E82EF9D7AA51BF27AB51C023AC51C1238D
:1024C800AD51C22320EE06F0A451D926A551DA2237
:1024D800FF0EDE14AA6F010EDE14AB6F000EDE14C1
:1024E800AC6F000EDE14AD6FAA51AB11AC11AD117B
:1024F800D8B421D020EE16F0A451D926A551DA225D
:10250800BF51DE180AE1C051DE1807E1C151DE18DB
:1025180004E1C251DE18D8B40ED020EE16F0A45152
:10252800D926A551DA22BFC0DEFFC0C0DEFFC1C078
:10253800DEFFC2C0DEFF20EE06F0A451D926A55169
:10254800DA2210EE0AF0A451E126A551E222DE506B
:10255800E65CDE50E658DE50E658DE50E658D8B065
:1025680023D520EE06F0A451D926A551DA2210EE83
:102578000AF0A451E126A551E222DECFE6FFDECF24
:10258800E6FFDECFE6FFDECFE6FF20EE04F0A45143
:10259800D926A551DA22000EDB8A06D58EC0A9F00D
:1025A8008FC0AAF092C0D9FF93C0DAFF000EDE6E8A
:1025B800000EDD6E8CC00DF08DC00EF015EC50F0E5
:1025C8000001A46FA451D8B402D0A451120020EE87
:1025D80005F08C51D9268D51DA22DF50D8B408D0B5
:1025E80020EE05F08C51D9268D51DA22DF501200E9
:1025F80020EE04F08C51D9268D51DA22DFB002D0BA
:10260800070E120020EE06F08C51D9268D51DA22E1
:10261800DECF94F0DECF95F0DECF96F0DECF97F0E8
:1026280020EE0AF08C51D9268D51DA22DECF98F0AF
:10263800DECF99F0DECF9AF0DECF9BF09451985D13
:10264800A06F95519959A16F96519A59A26F9751B8
:102658009B59A36F9051946F9151956F966B976B9F
:102668009451A05D9551A1599651A2599751A359DA
:10267800D8B059D2A0C090F0A1C091F054D220EEA9
:1026880006F08C51D9268D51DA22FF0EDE14946F94
:10269800010EDE14956F000EDE14966F000EDE1428
:1026A800976F9451951196119711D8A4AFD120EE38
:1026B80006F08C51D9268D51DA22DECF94F0DECF88
:1026C80095F0DECF96F0DECF97F00A0E05D0D890C1
:1026D8009733963395339433E82EF9D78CC0D9FFC6
:1026E8008DC0DAFF10EE02F0DE50E126DD50E22266
:1026F800E750986F98059415AB6FAB51D8A46FD07D
:1027080020EE06F08C51D9268D51DA22DE50DE10EB
:10271800DE10DE10D8A40FD020EE0EF08C51D92692
:102728008D51DA22DECFA5F0DECFA6F0DECFA7F0FE
:10273800DECFA8F020D08CC0D9FF8DC0DAFFDECF65
:1027480060F0DDCF61F020EE12F08C51D9268D516A
:10275800DA22DECF62F0DECF63F0DECF64F0DECFC8
:1027680065F0B4EC21F060C0A5F061C0A6F062C0CD
:10277800A7F063C0A8F00001A851A711A6110EE1A7
:10278800020EA55DD8B00AD020EE05F08C51D926EE
:102798008D51DA22020EDF6E020E1200A52911E118
:1027A800A6290FE1A7290DE1A829D8A40AD020EE6F
:1027B80005F08C51D9268D51DA22010EDF6E010EFB
:1027C800120020EE12F08C51D9268D51DA22A5C0C4
:1027D800DEFFA6C0DEFFA7C0DEFFA8C0DEFF8CC0FC
:1027E800D9FF8DC0DAFFDECF18F0DDCF19F020EE6B
:1027F80012F08C51D9268D51DA22DECF1AF0DECFB5
:102808001BF0DECF1CF0DECF1DF0D6EC4DF018C06B
:10281800ACF019C0ADF01AC0AEF01BC0AFF00001AB
:10282800AC51AD11AE11AF11D8B4AED7AB51AC2786
:10283800000EAD23AE23AF2390C094F091C095F065
:10284800090E966FD89095339433962FFBD794C082
:10285800B0F095C0B1F0B051B111D8B4C9D0AB51F6
:10286800B025946F000EB121956F8CC0D9FF8DC033
:10287800DAFF10EE02F0DE50E126DD50E222E750EA
:10288800966F976B9451965D95519759D8B012D021
:102898008CC0D9FF8DC0DAFF10EE02F0DE50E126C1
:1028A800DD50E222E750946FAB51945DB06FB16B8D
:1028B800D8A0B107A9C01BF0AAC01CF0ACC01DF07D
:1028C800ADC01EF0AEC01FF0AFC020F0B0C021F008
:1028D800B1C022F08CC0D9FF8DC0DAFF10EE01F034
:1028E800DE50E126DD50E222E7500FEC4DF0000902
:1028F800D8A4CBD08CC0D9FF8DC0DAFF10EE04F07D
:10290800DE50E126DD50E222E750D8B461D0000164
:10291800B051946FB151956F966B976B8CC0D9FF7E
:102928008DC0DAFF10EE2AF0DE50E126DD50E222FB
:10293800E6CF98F0E6CF99F0E6CF9AF0E6CF9BF095
:10294800AC51985D9C6FAD5199599D6FAE519A5994
:102958009E6FAF519B599F6F94519C5D95519D59A6
:1029680096519E5997519F59D8B032D08CC0D9FFF3
:102978008DC0DAFF10EE2AF0DE50E126DD50E222AB
:10298800E6CF94F0E5CF95F0AC51945FAD51955BEF
:10299800090ED89094379537E82EFBD79451A9257E
:1029A8000C6E9551AA210D6E8CC0D9FF8DC0DAFF2F
:1029B800DECF96F0DDCF97F02E0E96250E6E000E28
:1029C80097210F6E020E116E000E106E76EC57F006
:1029D800B0C094F0B1C095F0090ED89000019437BA
:1029E8009537E82EFAD794C0B2F095C0B3F07ED0F0
:1029F80020EE16F08C51D9268D51DA22ACC0DEFFBC
:102A0800ADC0DEFFAEC0DEFFAFC0DEFFFF0E946FCD
:102A1800010E956F20EE06F08C51D9268D51DA22E1
:102A2800DECF96F0DDCF97F0945196179551971712
:102A380096510008B26F9751D8A0E82A0208B36FE0
:102A4800B251905DB3519159D8B004D090C0B2F052
:102A580091C0B3F08CC0D9FF8DC0DAFFDECF3AF059
:102A6800DDCF3BF020EE16F08C51D9268D51DA22BD
:102A7800DECF3CF0DECF3DF0DECF3EF0DECF3FF0E4
:102A880087EC4EF00009D8B402D0000190D6A9C056
:102A98000CF0AAC00DF0FF0E0001946F010E956FA7
:102AA80020EE06F08C51D9268D51DA22DECF96F031
:102AB800DDCF97F094519617955197178CC0D9FF91
:102AC8008DC0DAFFDECF98F0DDCF99F096519827C8
:102AD800975199232E0E98250E6E000E99210F6E90
:102AE800B2C010F0B3C011F076EC57F0B251A9277C
:102AF800B351AA2320EE06F08C51D9268D51DA2243
:102B0800B251DE26B351DE22000EDE22DE2292C052
:102B1800D9FF93C0DAFFB251DE26B351DD22B2519C
:102B2800905FB351915B90519111D8A4A8D5000E34
:102B38001200296E000E286E2FD22950D8A40DD06D
:102B48000001FD51D8B409D0000E286E000E010115
:102B5800836F0A0E47D0839091D2020E2918D8A409
:102B68000BD00001FD51D8B407D0000E286E000E1E
:102B78000101836F140E36D01F0E296435D0300E34
:102B8800296032D00001FD51D8B42ED02950E00F71
:102B9800FE6F000E286EFE51200D1A0EF324D96E1A
:102BA800020EF420DA6EDE50DE10DE10DE10D8B42D
:102BB80003D0030EFE652FD0010E4F6EFE51140D8B
:102BC800130EF324D96E010EF420DA6EFE51140DA3
:102BD800130EF324E16E010EF420E26EE7500409AF
:102BE800DF6E19D0826FB7D73F0E296419D0500E07
:102BF800296016D00001FD51D8B412D0FE51140D31
:102C0800000EF324D96E010EF420DA6E2950C00F9D
:102C1800DF6E000E286E000E0101836F000EE2D7F2
:102C2800340E2918D8A40BD00001FD51D8B407D010
:102C3800000E0101836F000E826F000EABD1350EBE
:102C48002918D8A40BD00001FD51D8B407D0000E24
:102C5800286E0D0E0101836FAC0EC4D7370E2918EC
:102C6800D8A409D00001FD51D8B405D00E0E010139
:102C7800836F750E87D10D0E2918D8A40BD00001CB
:102C8800FD51D8B407D0000E286E020E0101836FE3
:102C9800BC0EA8D7100E2918D8A409D00001FD51E0
:102CA800D8B405D0030E0101836FE90E6BD1180E5D
:102CB8002918D8A409D00001FD51D8B405D0070EB1
:102CC8000101836F090E5ED13E0E2918D8A4D6D112
:102CD8000001FD51D8B4D2D10F0E0101836F3D0E12
:102CE80051D10001FE51140D010EF324D96E010ECD
:102CF800F420DA6E29C0DFFF030E0101836FEA0EAC
:102D080041D10001FE51140D020EF324D96E010EBB
:102D1800F420DA6E29C0DFFF030E0101836FEB0E8A
:102D280031D10001FE51140D030EF324D96E010EAA
:102D3800F420DA6E29C0DFFF030E0101836FEC0E69
:102D480021D10001FE51140D040EF324D96E010E99
:102D5800F420DA6E29C0DFFF030E0101836FED0E48
:102D680011D10001FE51140D050EF324D96E010E88
:102D7800F420DA6E29C0DFFF030E0101836FEE0E27
:102D880001D10001FE51140D060EF324D96E010E77
:102D9800F420DA6E29C0DFFFFE51140D060EF3246D
:102DA800D96E010EF420DA6EDF500C6E0CC00DF0F7
:102DB8000E6A0F6A106A0FC010F00EC00FF00DC037
:102DC8000EF00D6AFE51140D050EF324D96E010E96
:102DD800F420DA6EDF50116E11C012F0136A146A13
:102DE800156A13C015F012C014F0136A126AFE5166
:102DF800140D040EF324D96E010EF420DA6EDF50A0
:102E0800166E16C017F0186A196A1A6A17C01AF0EF
:102E1800196A186A176AFE51140D030EF324D96E45
:102E2800010EF420DA6EDF501B6E1B5017241C6E47
:102E3800000E18201D6E000E19201E6E000E1A209E
:102E48001F6E12501C24206E13501D20216E14502A
:102E58001E20226E15501F20236E0D502024246E34
:102E68000E502120256E0F502220266E1050232050
:102E7800276EFE51140D070EF324D96E010EF420AF
:102E8800DA6E24C0DEFF25C0DEFF26C0DEFF27C0C5
:102E9800DEFF000E0101836F000E74D00001FE51A9
:102EA800140D120EF324D96E010EF420DA6E29C027
:102EB800DFFF070E0101836F0A0E64D00001FE5187
:102EC800140D110EF324D96E010EF420DA6E29C008
:102ED800DFFF070E0101836F0B0E54D00001FE5176
:102EE800140D100EF324D96E010EF420DA6E29C0E9
:102EF800DFFF070E0101836F0C0E44D00001FE5165
:102F0800140D0F0EF324D96E010EF420DA6E29C0C9
:102F1800DFFFBFD729C000F20F0E0101836F3E0EFD
:102F280031D029C001F20F0E0101836F3F0E2AD064
:102F380029C002F20F0E0101836F400E23D029C071
:102F480003F20F0E0101836F410E1CD029C004F259
:102F58000F0E0101836F420E15D029C005F20F0E26
:102F68000101836F430E0ED029C006F20F0E010136
:102F7800836F440E07D029C007F28BD70E0E0101CC
:102F8800836F760E826F7AD0000E0101836F000E78
:102F9800826F090E286EDFD582C10CF083C10DF057
:102FA8000D50000AD8B416D0030AD8B418D0040AB1
:102FB800D8B429D00A0AD8B434D0030AD8B437D040
:102FC800010AD8B43CD0130AD8B453D03B0AD8B4B9
:102FD80053D054D00C50000AD8B4AFD54FD00C50B1
:102FE800E90AD8B47ED6030AD8B48BD6010AD8B475
:102FF80098D6070AD8B4A5D6010AD8B4B2D6030A17
:10300800D8B4BFD63BD00C50090AD8B447D7030A66
:10301800D8B454D7010AD8B461D7070AD8B46ED740
:103028002DD00C50480AD8B434D7E40A27D00C5015
:10303800750AD8B4A3D7030AD8B4A6D71FD00C50A2
:103048003D0AD8B467D7030AD8B46BD7010AD8B4F5
:103058006FD77F0AD8B473D7010AD8B477D7030AD1
:10306800D8B47BD7010AD8B47FD7070AD8B483D796
:1030780005D00C502A0A02D00C500F0A2850120012
:10308800D851D911D8A402D0090E1200D8C0D9FF3E
:10309800D9C0DAFF000EDE6E000EDD6E8CC1C9F1FC
:1030A8008DC1CAF11F0EDC17C90E456E010E466EA2
:1030B800DA0E476EDC51FE0B486EB8EC00F00101E9
:1030C800C66FC651D8A45BD2B20EDD6F010EDE6F9B
:1030D800C90E0001BD6F010EBE6FDAC0BFF0DBC0C4
:1030E800C0F07EEC41F00101C66FDBC1C7F1DCC165
:1030F800C8F1C651D8A406D0C751C811D8A402D067
:10310800060EC66FDCC0DDF01C0E0001DD17D8B45A
:1031180026D10101C651D8B414D0040EC619D8A4BA
:1031280009D0C90E0001C16F010EC26FA7EC4CF0A7
:103138000101C66F0001DC87DBC1C7F1DCC1C8F142
:1031480014D020EE0BF0C751D926C851DA22DF502F
:103158000001DD6F110EDD17D8B402D0070E03D0C1
:10316800DCA503D0080E0101C66F0101C651D8A421
:1031780012D10001DCA70FD1000E0101C26F000EB1
:10318800C36F210EC46F460EC56F20EE0EF0C751F7
:10319800D926C851DA22000EDF6E20EE0FF0C75193
:1031A800D926C851DA22C3C1DFFF20EE10F0C7517B
:1031B800D926C851DA22C4C1DFFF20EE11F0C75169
:1031C800D926C851DA22C5C1DFFF20EE16F0C75153
:1031D800D926C851DA22000EDF6E20EE17F0C7514B
:1031E800D926C851DA22C3C1DFFF20EE18F0C75133
:1031F800D926C851DA22C4C1DFFF20EE19F0C75121
:10320800D926C851DA22C5C1DFFF20EE0BF0C7511D
:10321800D926C851DA22000EDF6E20EE1CF0C75105
:10322800D926C851DA22000EDF6E20EE1DF0C751F4
:10323800D926C851DA22000EDF6E20EE1EF0C751E3
:10324800D926C851DA22000EDF6E20EE1FF0C751D2
:10325800D926C851DA22000EDF6EC9C10CF0CAC1E6
:103268000DF0C7C10EF0C8C10FF074EC4DF00CC0E2
:10327800BEF10DC0BFF10EC0C0F10FC0C1F1C7C192
:103288000CF0C8C10DF0000E0E6E000E0F6E000E91
:10329800106E000E116E34EC57F0010120EE04F0B0
:1032A800C951D926CA51DA22010EDF6EBE51BF11AB
:1032B800C011C111D8B46FD020EE2AF0C951D92657
:1032C800CA51DA22DECFC2F1DECFC3F1DECFC4F1BC
:1032D800DECFC5F1C9C191F0CAC192F0BEC193F069
:1032E800BFC194F0C0C195F0C1C196F012EC45F091
:1032F8000101C66FC651D8A44ED0FF0EBE250001ED
:10330800DD6FFF0E0101BF210001DE6FFF0E01011D
:10331800C0210001DF6FFF0E0101C1210001E06F34
:10332800010120EE0AF0C951D926CA51DA22DDC0BE
:10333800DEFFDEC0DEFFDFC0DEFFE0C0DEFFC9C1AA
:103348003AF0CAC13BF0C2C13CF0C3C13DF0C4C1B0
:103358003EF0C5C13FF087EC4EF001011BD00101E2
:10336800C651D8A418D020EE0BF0C751D926C851A1
:10337800DA22DFA802D0040E0DD00001DCA30BD0A6
:10338800010120EE0BF0C751D926C851DA22DFA07F
:1033980002D0070EC66F0101C651D8A423D0000180
:1033A800DCB7DC8B010120EE2AF0C951D926CA51BD
:1033B800DA22000110EE1AF0D851E126D951E222A2
:1033C800DECFE6FFDECFE6FFDECFE6FFDECFE6FFAD
:1033D80020EE1EF0D851D926D951DA22C7C1DEFF16
:1033E800C8C1DDFF0101C651D8A4C9D0000120EE33
:1033F80004F0D851D926D951DA22DCC0DFFF20EEFB
:1034080005F0D851D926D951DA22000EDF6EC9C18C
:103418000CF0CAC10DF0C7C10EF0C8C10FF074ECB2
:103428004DF0000120EE0EF0D851D926D951DA22FC
:103438000CC0DEFF0DC0DEFF0EC0DEFF0FC0DEFFDA
:10344800010120EE1DF0C751D926C851DA22DF50FC
:103458000001DD6FDD51DF6FDE6B010120EE1EF034
:10346800C751D926C851DA22DF500001E06FE0C009
:10347800E1F0E26BE36BE46BE2C0E4F0E1C0E3F09F
:10348800E26BE16B010120EE1FF0C751D926C8514C
:10349800DA22DF500001E56FE5C0E6F0E76BE86B84
:1034A800E96BE6C0E9F0E86BE76BE66BE151E61122
:1034B800EA6FE251E711EB6FE351E811EC6FE45169
:1034C800E911ED6FDE51EA11EE6FDF51EB11EF6F8D
:1034D800000EEC11F06F000EED11F16F010120EEFE
:1034E8001CF0C751D926C851DA22DF500001F26F0B
:1034F800F251EE11F36FEF51F46FF051F56FF15196
:10350800F66F20EE0AF0D851D926D951DA22F3C045
:10351800DEFFF4C0DEFFF5C0DEFFF6C0DEFF20EE02
:1035280006F0D851D926D951DA22DE6ADE6ADE6A77
:10353800DD6A20EE16F0D851D926D951DA22DE6A92
:10354800DE6ADE6ADD6AD8C0D9FFD9C0DAFFC9C130
:10355800DEFFCAC1DDFFD8C0D9FFD9C0DAFF10EE3F
:1035680006F0DE50E126DD50E22220EE02F0D851CE
:10357800D926D951DA22E6CFDEFFE5CFDDFF0101FA
:10358800C651120065516411631104E1020E625DB7
:10359800D8A010D020EE12F06051D9266151DA225D
:1035A800DE50625DDE506359DE506459DE50655965
:1035B800D8A03FD2020E8E6F52D262C08CF063C088
:1035C8008DF0D8908D316B6F8C316A6F6A518C2772
:1035D8006B518D2360C03AF061C03BF020EE1EF0C5
:1035E8006051D9266151DA22DECF6AF0DECF6BF066
:1035F800DECF6CF0DECF6DF08CC06EF08DC06FF05A
:10360800090E706FD8906F336E33702FFBD76E51E1
:103618006A253C6E6F516B213D6E000E6C213E6E2B
:10362800000E6D213F6E87EC4EF000018E6F8E51BB
:10363800D8A415D2FF0E6A6F010E6B6F8CC06CF0A8
:103648008DC06DF06A516C176B516D1760C06EF0CC
:1036580061C06FF06C516E276D516F232E0E6E2571
:103668008F6F000E6F21906F8C4B8D2B62B104D041
:1036780066C088F0896B1AD066516A6F6B6B6A3BBB
:103688006B3BF00E6B176A510F0B6B13F00E6A173A
:103698008FC0D9FF90C0DAFFDF500F0B6C6F6D6BD6
:1036A8006A516C11886F6B516D11896F8FC0D9FF8A
:1036B80090C0DAFF88C0DFFF20EE04F06051D92601
:1036C8006151DA22010EDF6E60C03AF061C03BF052
:1036D80020EE1EF06051D9266151DA22DECF6AF061
:1036E800DECF6BF0DECF6CF0DECF6DF08CC06EF00D
:1036F8008DC06FF0090E706FD8906F336E33702FD6
:10370800FBD76E516A253C6E6F516B213D6E000EE2
:103718006C213E6E000E6D213F6E87EC4EF000016D
:103728008E6F8E51D8A49BD1FF0E6A6F010E6B6FFE
:103738008CC06CF08DC06DF06A516C176B516D17B1
:1037480060C06EF061C06FF06C516E276D516F23D1
:103758002E0E6E258F6F000E6F21906F62B10ED006
:1037680067C06AF00F0E6A178FC0D9FF90C0DAFFE2
:10377800DF50F00B6A116B6F6B5112D066C06AF0A4
:1037880067C06BF068C06CF069C06DF0050E05D0BD
:10379800D8906D336C336B336A33E82EF9D76A519E
:1037A8008A6F8B6B8FC0D9FF90C0DAFF8AC0DFFFAA
:1037B80037D160C03AF061C03BF020EE1EF0605196
:1037C800D9266151DA22DECF6AF0DECF6BF0DECF88
:1037D8006CF0DECF6DF063516E6F64516F6F6551A1
:1037E800706F716B6A516E253C6E6B516F213D6E27
:1037F8006C5170213E6E6D5171213F6E87EC4EF019
:1038080000018E6F8E51D8A42AD1FF0E6A6F010E67
:103818006B6F62C06CF063C06DF0D8906C376D3719
:103828006A516C176B516D1760C06EF061C06FF014
:103838006C516E276D516F232E0E6E258F6F000E03
:103848006F21906F8FC0D9FF90C0DAFF66C0DFFF8D
:1038580020EE01F08F51D9269051DA2267C0DFFFA0
:10386800DFD060C03AF061C03BF020EE1EF060513E
:10387800D9266151DA22DECF6AF0DECF6BF0DECFD7
:103888006CF0DECF6DF062C06EF063C06FF064C0A4
:1038980070F065C071F0080E05D0D89071337033A0
:1038A8006F336E33E82EF9D76A516E253C6E6B5133
:1038B8006F213D6E6C5170213E6E6D5171213F6ECE
:1038C80087EC4EF000018E6F8E51D8A4C8D0FF0E41
:1038D8006A6F010E6B6F62C06CF063C06DF0D890B8
:1038E8006C376D37D8906C376D376A516C176B51E0
:1038F8006D1760C06EF061C06FF06C516E276D512E
:103908006F232E0E6E258F6F000E6F21906F20EEA5
:1039180001F08F51D9269051DA22DF506A6F6A512F
:103928006C6F6B6B20EE02F08F51D9269051DA2222
:10393800DF506D6F6DC06EF06F6B706B716B6FC029
:1039480071F06EC070F06F6B6E6B20EE03F08F51EC
:10395800D9269051DA22DF50726F72C073F0746BFF
:10396800756B766B73C076F0756B746B736B6E5199
:103978007311776F6F517411786F70517511796F7A
:10398800715176117A6F6B5177117B6F6C51781189
:103998007C6F000E79117D6F000E7A117E6F8FC0DB
:1039A800D9FF90C0DAFFDF507F6F7F517B11806FA6
:1039B8007C51816F7D51826F7E51836F000E80151F
:1039C800846F000E8115856F000E8215866FF00ECC
:1039D8008315876F84516613855167138651681361
:1039E800875169138FC0D9FF90C0DAFF66C0DFFF27
:1039F80020EE01F08F51D9269051DA2267C0DFFFFF
:103A080020EE02F08F51D9269051DA2268C0DFFFEC
:103A180020EE03F08F51D9269051DA2269C0DFFFDA
:103A280020EE04F06051D9266151DA22010EDF6ED2
:103A380016D060C0D9FF61C0DAFFDF506A6F6B6BC8
:103A48006B51000AD8A4B6D56A51010AD8B4B5D5C5
:103A5800030AD8B4AED6010AD8B403D7ABD58E5171
:103A680012002B6E1CC042F01DC043F02B50D8B47E
:103A780002D0040E1200010E406E53A013D2030EA2
:103A88001200EDEC59F00009D8B42DD2000E08D27E
:103A9800000E156E000E166E000E176E000E186ED4
:103AA800090E55EC57F00009D8A41DD22C0E0C6E47
:103AB8000D6A000E0F6E100E0E6ED8EC53F0000952
:103AC800D8B411D22C44E846030BE806D8A44ED04B
:103AD80033C01EF03F0E1E161EC01FF0206A216A5A
:103AE800226A20C022F01FC021F0206A1F6A3450C9
:103AF800246E236A3550256E266A235025262450C5
:103B0800262225501F24276E26502020286E000EBE
:103B18002120296E000E22202A6E010E27243C6ED9
:103B2800000E28203D6E000E29203E6E000E2A2031
:103B38003F6E3CC01EF03DC01FF03EC020F03FC0AD
:103B480021F00A0ED8901E361F3620362136E82E70
:103B5800F9D71CC0D9FF1DC0DAFF1EC0DEFF1FC089
:103B6800DEFF20C0DEFF21C0DEFF90D71E6A36AE22
:103B780001D01E2A010E1E1631C01FF00F0E1F168F
:103B88003550030B020DF3501F241E24020F416E03
:103B98003250030B1E6E1F6A0A0ED8901E361F364F
:103BA800E82EFBD73350206E216AD8902036213674
:103BB800D890203621363444E846030B226E236A17
:103BC80020502226215023221E5022261F50232215
:103BD800010E2226000E232222C03CF023C03DF015
:103BE8003E6A3F6A41C01EF0F70E1E263CC01FF019
:103BF8003DC020F03EC021F03FC022F01E2A05D073
:103C0800D8901F362036213622361E2EF9D73AD0C4
:103C180050A445D0000E156E000E166E000E176EDD
:103C2800000E186E8D0E55EC57F00009D8A45BD124
:103C380058EC5AF02C0E0C6E0D6A000E0F6E100E1A
:103C48000E6ED8EC53F00009D8B44DD1300E416E49
:103C580003D058EC5AF041064150D8A4FAD736C0E0
:103C68001EF01E3A0F0E1E16100E1F6E206A216AD5
:103C7800226A1E2A05D0D8901F36203621362236D1
:103C88001E2EF9D71CC0D9FF1DC0DAFF1FC0DEFFEA
:103C980020C0DEFF21C0DEFF22C0DEFFF7D6000E07
:103CA800156E000E166E000E176E000E186E090EB9
:103CB80055EC57F00009D8A416D12C0E0C6E0D6ADD
:103CC800000E0F6E100E0E6ED8EC53F00009D8B42B
:103CD8000AD150A22AD039C01EF0060E1F6ED89005
:103CE8001E321F2EFCD7FF0E1E2636503F0B206EAD
:103CF800216AD89020362136226A37AE01D0222A8E
:103D0800010E221622502026000E2122010E202606
:103D1800000E21221E2A03D0D890203621361E2ECE
:103D2800FBD72050236E215034D036C01EF0D890D7
:103D38001E32D8901E321F0E1E16010E1E240C6E47
:103D48000D6A000E0D223750030B1F6E206AD890A3
:103D58001F362036D8901F362036D8901F3620368A
:103D680037C021F0050E226ED8902132222EFCD7C2
:103D7800070E211621501F26000E2022010E1F2497
:103D88000E6E000E20200F6EB9EC59F00C50236E09
:103D98000D50246E256A266A1CC0D9FF1DC0DAFFA3
:103DA80023C0DEFF24C0DEFF25C0DEFF26C0DEFF05
:103DB8006DD642C0D9FF43C0DAFF50C0DFFF66D6D8
:103DC800000E156E000E166E000E176E000E186EA1
:103DD800090E55EC57F00009D8A485D042C00CF064
:103DE80043C00DF0000E0F6E100E0E6ED8EC53F09F
:103DF8000009D8A44BD677D0000E156E000E166EAB
:103E0800000E176E000E186E0A0E55EC57F00009DA
:103E1800D8A469D042C00CF043C00DF0000E0F6E5C
:103E2800100E0E6ED8EC53F0E3D7000E156E000E90
:103E3800166E000E176E000E186E3A0E55EC57F0FF
:103E48000009D8A450D0040E416E0AD058EC5AF09C
:103E580042C0D9FF43C0DAFFDF6E424A432A410617
:103E68004150D8B413D6F2D7000E156E000E166E58
:103E7800000E176E000E186E8D0E55EC57F00009E7
:103E8800D8A431D058EC5AF042C00CF043C00DF021
:103E9800000E0F6E400E0E6ED8EC53F0A9D7040E2C
:103EA800406E21D01B501E6E1F6A1F50000AD8A4F6
:103EB800F6D71E50000AD8B4E4D5010AD8B4E8D51C
:103EC800020AD8B4A5D6090AD8B473D7010AD8B457
:103ED80077D7070AD8B490D7010AD8B4A6D7030A67
:103EE800D8B4C2D7DCD769EC5AF040501200116E32
:103EF8000D50D8A4F0EC50F0000E106E0C50D8B451
:103F0800C3D111507F0B116E040E1118D8B404D010
:103F1800140E1118D8A40AD0000E0101816F000EEA
:103F2800806F000E0D6E070E0C6E12003F0E1118FA
:103F3800D8A40CD0000E4D6E000E0101816F000E4A
:103F4800806F000E0D6E000E0C6E12005F0E1118C1
:103F5800D8A40CD0000E4E6E000E0101816F000E29
:103F6800806F000E0D6E000E0C6E12003F0E116475
:103F780007D05F0E116004D0400E1118D8A4EAD7FC
:103F8800400E1118D8A40ED0010E4E6E000E4D6EC4
:103F9800000E0101816F000E806F000E0D6E000E85
:103FA8000C6E1200200E1118D8A46ED1010E4D6EA1
:103FB800000E0101816F000E806F000E0D6E000E65
:103FC8000C6E1200600E1118D8A40DD04E50D8B443
:103FD8000AD001019651D8B402D0080E01D0030EC0
:103FE800106E000E27D0600E1118D8A40BD04D50BB
:103FF800D8B408D001019651D8B402D0090EF0D730
:10400800050EEED7680E1118D8A40AD04D50D8B4B2
:1040180007D01A0E0101816F900E22D183809CD1A6
:10402800680E1118D8A40AD04E50D8B407D0020E82
:10403800106E65D0816F000E806F8ED16A0E1118D8
:10404800D8A408D04D50D8B405D01A0E0101816FFC
:10405800F40E06D16C0E1118D8A408D04D50D8B45F
:1040680005D01A0E0101816F2C0EFAD0700E1118AE
:10407800D8A40AD04E50D8B407D0040E106E000E43
:104088000101816F000EECD0700E1118D8A464D114
:104098004D50D8B461D11B0E0101816F620EE0D082
:1040A8008380020E1118D8A405D01A0E0101816F61
:1040B800920E806F050E1118D8A405D01A0E0101B2
:1040C800816FAE0E806F070E1118D8A405D01A0E96
:1040D8000101816FB80E806F080E1118D8A405D0A1
:1040E8001A0E0101816FCC0E806F030E1118D8B41F
:1040F80003D01128D8A406D0000E106E8390000EAD
:10410800010198D7160E1118D8A426D11A0E01014C
:10411800816FA40E91D7050E1118D8A41DD11A0EBF
:104128000101816FF50E88D711C0FEF01A0E01014A
:10413800816F9B0E81D71A0E0101816F9C0E7CD76F
:104148000001FE51070D500EF324D96E010EF42024
:10415800DA6E11C0DFFF1A0E0101816F9D0E6CD758
:104168000001FE51070D510EF324D96E010EF42003
:10417800DA6E11C0DFFF1A0E0101816F9E0E5CD747
:104188000001FE51070D520EF324D96E010EF420E2
:10419800DA6E11C0DFFF000E0101816F000E806F23
:1041A800010E64D01A0E0101816FB90E59D01A0E92
:1041B8000101816FBA0E40D71A0E0101816FBB0E43
:1041C8003BD7000E0101816F000E806F41D0000EB9
:1041D8000101816F000E806F060E48D011C0FEF0FD
:1041E800000E0101816F000E806F000E30D0000EAE
:1041F8000101966F1A0E816FF70EE7D71A0E0101AB
:10420800816FF70E19D78390270E0101816F0F0E6A
:1042180013D7180E1118D8A49FD01A0E0101816F58
:104228002D0E0AD71A0E0101816F2E0E05D71A0E10
:104238000101816F2F0E00D71A0E0101816F300E18
:10424800FBD6000E0101816F000E806F0A0E106E02
:10425800839082D0040E106E270E0101816F0F0E1D
:10426800806FDCD68380000E010109D0106E74D0F7
:104278008390010E0101966F080E106E000E816F7B
:10428800000E806F000EF2D780C10EF081C10FF0D2
:104298000F50000AD8B40AD01A0AD8B40CD0010AB0
:1042A800D8B450D03C0AD8B455D056D00E50000AD5
:1042B800D8B488D651D00E502C0AD8B4AAD7010A3F
:1042C800D8B4B0D7030AD8B4B2D7010AD8B4B4D78F
:1042D8001F0AD8B4B6D7A00AD8B4E2D6020AD8B40E
:1042E80023D7090AD8B427D7070AD8B429D7010A87
:1042F800D8B436D7030AD8B443D73A0AD8B467D75C
:104308000A0AD8B4B5D7160AD8B44CD7010AD8B413
:104318004ED7030AD8B450D7010AD8B452D7790A6D
:10432800D8B485D60E0AD8B459D7380AD8B4F3D633
:10433800010AD8B45CD7030AD8B460D7010AD8B444
:1043480062D70AD00E50580AD8B484D73A0AD8B4DB
:1043580089D702D00E500F0A10C00CF00D6A120057
:10436800000165516411631104E1020E625DD8A079
:1043780010D020EE12F06051D9266151DA22DE50B9
:10438800625DDE506359DE506459DE506559D8A02D
:1043980008D0010E846F000E856F000E866F000E28
:1043A800ECD18469856986698769E9D162C088F03A
:1043B80063C089F0D8908931676F8831666F66511C
:1043C80088276751892360C03AF061C03BF020EE2E
:1043D8001EF06051D9266151DA22DECF66F0DECFB9
:1043E80067F0DECF68F0DECF69F088C06AF089C078
:1043F8006BF0090E6C6FD8906B336A336C2FFBD758
:104408006A5166253C6E6B5167213D6E000E68212E
:104418003E6E000E69213F6E87EC4EF00009D8A46D
:10442800C4D1FF0E0001666F010E676F88C068F087
:1044380089C069F0665168176751691760C06AF0EA
:1044480061C06BF068516A2769516B232E0E6A258B
:10445800D96E000E6B21DA6EDF506C6F6C51826F73
:10446800836B884B892B60C03AF061C03BF020EE2B
:104478001EF06051D9266151DA22DECF66F0DECF18
:1044880067F0DECF68F0DECF69F088C06AF089C0D7
:104498006BF0090E6C6FD8906B336A336C2FFBD7B7
:1044A8006A5166253C6E6B5167213D6E000E68218E
:1044B8003E6E000E69213F6E87EC4EF00009D8A4CD
:1044C80074D1FF0E0001666F010E676F88C068F037
:1044D80089C069F0665168176751691760C06AF04A
:1044E80061C06BF068516A2769516B232E0E6A25EB
:1044F800D96E000E6B21DA6EDF506C6F6C516E6FE7
:104508006D6B6D5182136E51831362B107D0FF0E2C
:104518008215806F0F0E8315816F0FD082C066F0F1
:1045280083C067F0040E686FD89067336633682FCE
:10453800FBD766C080F067C081F080C084F081C07E
:1045480085F061D060C03AF061C03BF020EE1EF00B
:104558006051D9266151DA22DECF66F0DECF67F0EE
:10456800DECF68F0DECF69F063516A6F64516B6F1C
:1045780065516C6F6D6B66516A253C6E67516B2196
:104588003D6E68516C213E6E69516D213F6E87EC1E
:104598004EF00009D8A409D1FF0E0001666F010E84
:1045A800676F62C068F063C069F0D8906837693790
:1045B800665168176751691760C06AF061C06BF08F
:1045C80068516A2769516B232E0E6A258A6F000E7F
:1045D8006B218B6F20EE01F08A51D9268B51DA229C
:1045E800DF50666F6651686F676B8AC0D9FF8BC0F2
:1045F800DAFFDF50696F69516713000E681367C0EF
:1046080084F068C085F0866B876BCFD060C03AF0C5
:1046180061C03BF020EE1EF06051D9266151DA22CC
:10462800DECF66F0DECF67F0DECF68F0DECF69F070
:1046380062C06AF063C06BF064C06CF065C06DF076
:10464800080E05D0D8906D336C336B336A33E82E7F
:10465800F9D766516A253C6E67516B213D6E6851EA
:104668006C213E6E69516D213F6E87EC4EF000095A
:10467800D8A49BD0FF0E0001666F010E676F62C061
:1046880068F063C069F0D89068376937D8906837A0
:104698006937665168176751691760C06AF061C069
:1046A8006BF068516A2769516B232E0E6A258A6F51
:1046B800000E6B218B6F20EE01F08A51D9268B51A9
:1046C800DA22DF50666F6651686F676B20EE02F082
:1046D8008A51D9268B51DA22DF50696F69C06AF096
:1046E8006B6B6C6B6D6B6BC06DF06AC06CF06B6B59
:1046F8006A6B20EE03F08A51D9268B51DA22DF50FB
:104708006E6F6EC06FF0706B716B726B6FC072F012
:10471800716B706B6F6B6A516F11736F6B517011A6
:10472800746F6C517111756F6D517211766F67519D
:104738007311776F68517411786F000E7511796F66
:10474800000E76117A6F8AC0D9FF8BC0DAFFDF506E
:104758007B6F7B5177117C6F78517D6F79517E6FBC
:104768007A517F6FFF0E7C15846FFF0E7D15856F64
:10477800FF0E7E15866F0F0E7F15876F16D060C0EF
:10478800D9FF61C0DAFFDF50666F676B6751000AB7
:10479800D8A4FFD56651010AD8B408D6030AD8B4FC
:1047A800D1D6010AD8B432D7F4D584C060F085C018
:1047B80061F086C062F087C063F0120019C0F6FF8E
:1047C8001AC0F7FF0800F5CF47F0194A1A2A4750D0
:1047D800D8B41200250E4718D8B404D047502CEC92
:1047E8005AF0ECD7000E436E000E426E19C0F6FF69
:1047F8001AC0F7FF0800F5CF47F0194A1A2A300EF9
:104808004718D8A40ED0000E436E010E426E19C090
:10481800F6FF1AC0F7FF0800F5CF47F0194A1A2A21
:1048280008D02D0E4718D8A404D0000E436E020EEF
:10483800EDD7000E3B6E000E3A6E1DD03AC00CF05C
:104848003BC00DF0000E0F6E0A0E0E6EB9EC59F05B
:1048580047500C26000E0D22D00E0C243A6EFF0E87
:104868000D203B6E19C0F6FF1AC0F7FF0800F5CF00
:1048780047F0194A1A2A2F0E476403D0390E4764A5
:10488800DDD76C0E4718D8B404D04C0E4718D8A4FE
:104898000AD0428419C0F6FF1AC0F7FF0800F5CF06
:1048A80047F0194A1A2A4750D8B4120047C046F0B0
:1048B800600E46647AD0200E465E77D01B50D96EC3
:1048C800DA6A020EDF26DF5CD96EDA6ADECF36F0EE
:1048D800DECF37F0000E3D6E000E3C6E02D03C4A33
:1048E8003D2A3C5036241C6E3D5037201D6E1CC09E
:1048F800F6FF1DC0F7FF000EF86E0E0EF76403D02A
:104908000800F55005D0F6CFE9FFF7CFEAFFEF50E2
:104918000009D8B404D0E3D7200E2CEC5AF042B2E8
:104928000CD03C501C6E3D501D6E3C4A3D2A3A50FE
:104938001C5C3B501D58D8A0EFD736C00DF037C0CF
:104948000EF0ECEC55F003D0200E2CEC5AF03C5055
:104958001C6E3D501D6E3C4A3D2A3A501C5C3B5033
:104968001D58D8B02BD7F0D71B50D96EDA6ADF5054
:10497800DF2ADF2AD96EDA6ADF502CEC5AF01ED70C
:10498800000E396E020E0BD0000E396E080E07D0DD
:10499800000E396E0A0E03D0000E396E100E386EF6
:1049A80022D047502CEC5AF009D746501C6E1D6A8D
:1049B8001D50000AD8A4F5D71C50420AD8B4E0D735
:1049C800010AD8B4D1D7070AD8B4E2D70B0AD8B4A9
:1049D800DBD71C0AD8B472D7060AD8B4D9D70D0ABF
:1049E800D8B4DAD7DED742B431D0440E4618D8B49A
:1049F80013D01B50D96EDA6ADF50DF2ADF2AD96E4E
:104A0800DA6ADECF1CF0DDCF1DF01CC02EF01DC011
:104A18002FF0306A316A11D01B50D96EDA6ADF5034
:104A2800DF2ADF2AD96EDA6ADECF2EF0DDCF2FF04B
:104A3800000E2FBEFF0E306E316E2EC03EF02FC01E
:104A48003FF030C040F031C041F010D01B50D96E5B
:104A5800DA6A040EDF26DF5CD96EDA6ADECF3EF052
:104A6800DECF3FF0DECF40F0DECF41F0440E4618F7
:104A7800D8B441AE0AD03E6C3F1ED8B03F2A401E83
:104A8800D8B0402A000E41564286000E456E000EF0
:104A9800446E3EC00CF03FC00DF040C00EF041C067
:104AA8000FF038C010F039C011F0126A136A74ECB4
:104AB80054F00C50466E3EC00CF03FC00DF040C0A4
:104AC8000EF041C00FF038C010F039C011F0126A72
:104AD800136ABFEC51F00CC03EF00DC03FF00EC0A1
:104AE80040F00FC041F0090E46640ED0780E47180A
:104AF800D8B404D0000E336E070E03D0000E336E08
:104B0800270E326E3250462644501E0FD96EDA6A8E
:104B18004650300FDF6E444A452A3E503F10401041
:104B28004110D8B406D0455004E1100E445CD8A01A
:104B3800B0D742A608D044501E0FD96EDA6A2D0E9F
:104B4800DF6E444A452A44C03CF045C03DF042B0BF
:104B580004D0000E356E200E03D0000E356E300ED8
:104B6800346E34C046F003D046502CEC5AF042B2B2
:104B78000CD03C501C6E3D501D6E3C4A3D2A3A50AC
:104B88001C5C3B501D58D8A0EFD74406D8A045065A
:104B980044501E0FD96EDA6ADF502CEC5AF044509C
:104BA8004510D8B404D0F1D7200E2CEC5AF03C5064
:104BB8001C6E3D501D6E3C4A3D2A3A501C5C3B50D1
:104BC8001D58D8B0FBD5F0D7100E8C6F020E8D6F24
:104BD800340E8E6F0B0E8F6F020E916F000E906F5A
:104BE800E60E926F936BD2EC12F0FF6F140E606FAB
:104BF800FE0E616FE6C062F0E7C063F021EC5AF088
:104C0800000E0001E96F000EE86F000EE36F000E62
:104C1800E26F000EEB6F000EEA6FEA51C40FD96E17
:104C2800DA6A000EDF6EEA51D30FD96EDA6A000E27
:104C3800DF6EEA4BEB2BEBBFF0D7EB5104E10F0E25
:104C4800EA5DD8A0EAD7000EED6F000EEC6F35D103
:104C5800340EEC25D96E0B0EED21DA6E0D0EDE1832
:104C6800D8A4E9D08E0E0C6EFF0E0D6EC40E0E6E1B
:104C78007CEC4FF00C500D10D8A407D0D30E136E57
:104C88007DEC47F013500101EA6F880E0C6EFF0EA1
:104C98000D6EC40E0E6E7CEC4FF00C500D10D8A4A7
:104CA80007D0D30E136E7DEC47F013500101A56FAA
:104CB8006D0E0C6EFF0E0D6EC40E0E6E7CEC4FF07A
:104CC8000C500D10D8A407D0D30E136E7DEC47F00E
:104CD80013500101A16FD30E0C6EFF0E0D6EC40EA2
:104CE8000E6E7CEC4FF00C500D10D8A407D0D30EEC
:104CF800136E7DEC47F0135001019F6F000E000109
:104D0800EF6F000EEE6FB50E766F776B740E786FDF
:104D1800FF0E796FEEC07AF0EFC07BF0F0EC56F042
:104D2800B50E0C6E0D6AC40E0E6E7CEC4FF00C5076
:104D38000D10D8A418D0EEC00CF0EFC00DF0000E86
:104D48000F6E0F0E0E6EB9EC59F0340E0C24126E65
:104D58000D0E0D20136ED30E146E000E166E0F0E70
:104D6800156E69EC55F00001EE4BEF2BEFBFCBD77A
:104D7800EF5104E1100EEE5DD8A0C5D7000EEF6F1D
:104D8800010EEE6FB50E766F776B7B0E786FFF0EA8
:104D9800796FEEC07AF0EFC07BF0F0EC56F0B50E0C
:104DA8000C6E0D6AC40E0E6E7CEC4FF00C500D109C
:104DB800D8A418D0EEC00CF0EFC00DF0000E0F6EA6
:104DC8000F0E0E6EB9EC59F0240E0C24126E0E0E56
:104DD8000D20136ED30E146E000E166E0F0E156E88
:104DE80069EC55F00001EE4BEF2BEFBFCBD7EF513D
:104DF80004E1040EEE5DD8A0C5D7000EEB6F000EDF
:104E0800EA6FEA51C40FD96EDA6A000EDF6EEA5112
:104E1800D30FD96EDA6A000EDF6EEA4BEB2BEBBFCD
:104E2800F0D7EB5104E10F0EEA5DD8A0EAD7000EE7
:104E3800E36F000E17D0340EEC25D96E0B0EED2162
:104E4800DA6E0A0EDE18D8B436D0340EEC25D96ED8
:104E58000B0EED21DA6E200EDE18D8A409D0000E54
:104E6800E36F010EE26F000EE96F000EE86F23D0CA
:104E7800E251E311D8B409D0340EEC25D96E0B0EEB
:104E8800ED21DA6EE851D30F08D0340EEC25D96E37
:104E98000B0EED21DA6EE851C40FE16EE26ADFCF46
:104EA800E7FFE9BF06D0E95106E10F0EE85DD8B08B
:104EB80002D0E84BE92BEC4BED2BE651EC5DE751CA
:104EC800ED59D8A0C5D6040E606FFE0E616FA1C162
:104ED80062F0636B21EC5AF0600E0001606FFE0E09
:104EE800616FEAC162F0636B21EC5AF0510E000168
:104EF800606FFE0E616FA5C162F0636B21EC5AF022
:104F0800000E0001EF6F000EEE6FEEC00CF0EFC068
:104F18000DF0000E0F6E0F0E0E6EB9EC59F0340E38
:104F28000C240001E46F0D0E0D20E56F920E606FEA
:104F3800FD0E616FEEC062F0EFC063F0E4C064F094
:104F4800E5C065F021EC5AF00001EE4BEF2BEFBF06
:104F5800DCD7EF5104E1100EEE5DD8A0D6D7000ED5
:104F6800ED6F010EEC6FECC00CF0EDC00DF0000E13
:104F78000F6E0F0E0E6EB9EC59F0240E0C240001C2
:104F8800E46F0E0E0D20E56FA30E606FFD0E616FCE
:104F9800ECC062F0EDC063F0E4C064F0E5C065F019
:104FA80021EC5AF00001EC4BED2BEDBFDCD7ED51B5
:104FB80004E1040EEC5DD8A0D6D7B40E606FFB0EEA
:104FC800616F21EC5AF0120020EE04F0A451D926AA
:104FD800A551DA22DECFA8F0DDCFA9F0010EA82571
:104FE800B16F000EA921B26FB151B211D8B40CD073
:104FF80020EE0EF0A451D926A551DA22DE50DE109B
:10500800DE10DE10D8A402D0040E1200B1C0A8F041
:105018000F0EA817D8A4A3D120EE0EF0A451D926BC
:10502800A551DA22DE2A000EDE22DE22DE2220EE62
:105038000AF0A451D926A551DA22DE50DE10DE107E
:10504800DE10D8A411D0A4C0D9FFA5C0DAFF10EE95
:1050580008F0DE50E126DD50E222E650B15DE65070
:10506800B259D8B0D1D77BD1B1C0A8F0B2C0A9F09D
:10507800040EAA6FD890A933A833AA2FFBD7FF0E26
:10508800AB6FFF0EAC6FA4C0D9FFA5C0DAFF10EE5E
:1050980002F0DE50E126DD50E222E750AD6FAE6B44
:1050A800AB51AD27AC51AE23A851AD17A951AE17DE
:1050B800AD51AE11D8A453D1A4C0D9FFA5C0DAFF11
:1050C800DECF60F0DDCF61F020EE0AF0A451D926E2
:1050D800A551DA22DECF62F0DECF63F0DECF64F0D6
:1050E800DECF65F0B4EC21F060C0B3F061C0B4F07D
:1050F80062C0B5F063C0B6F00001B651B511B41185
:1051080006E1020EB35DD8B002D0020E1200B32938
:1051180009E1B42907E1B52905E1B629D8A402D0E7
:10512800010E1200A4C0D9FFA5C0DAFF10EE12F0DC
:10513800DE50E126DD50E222E650B35DE650B45978
:10514800E650B559E650B659D8A0DAD0A651A711FD
:10515800D8B45AD7A4C0D9FFA5C0DAFFDECF91F0E2
:10516800DDCF92F020EE0AF0A451D926A551DA221B
:10517800DECF93F0DECF94F0DECF95F0DECF96F061
:1051880023EC2DF091C0B3F092C0B4F093C0B5F009
:1051980094C0B6F0B351B411B511B611D8A402D069
:1051A800070E1200B305B411B511B611D8B4ADD7B6
:1051B800B32907E1B42905E1B52903E1B629D8B433
:1051C800AFD7A4C0D9FFA5C0DAFFDECF25F0DDCF69
:1051D80026F066EC44F00009D8A4A2D7A4C0D9FFF1
:1051E800A5C0DAFFDECFA8F0DDCFA9F02E0E0001B2
:1051F800A8250C6E000EA9210D6E000E0F6E000E74
:105208000E6E020E116E000E106E69EC59F0A4C0FD
:10521800D9FFA5C0DAFFDECF18F0DDCF19F0B3C093
:105228001AF0B4C01BF0B5C01CF0B6C01DF0D6EC27
:105238004DF0A4C0D9FFA5C0DAFF10EE2AF0DE5069
:10524800E126DD50E22218C0E6FF19C0E6FF1AC0C9
:10525800E6FF1BC0E6FF000E0001B06F000EAF6F47
:105268002BD0A4C0D9FFA5C0DAFF10EE04F0DE50A1
:10527800E126DD50E222010EE76EA4C0D9FFA5C0E9
:10528800DAFFDECF25F0DDCF26F066EC44F000092A
:10529800D8A446D7A4C0D9FFA5C0DAFF10EE2AF0DB
:1052A800DE50E126DD50E222E62A000EE622E62262
:1052B800E6220001AF4BB02BA4C0D9FFA5C0DAFF8E
:1052C80010EE02F0DE50E126DD50E222E750A86F32
:1052D800A96BA851AF5DA951B059D8A0C2D7A4C035
:1052E800D9FFA5C0DAFF10EE2AF0DE50E126DD5026
:1052F800E222AF51E65EB051E65A000EE65AE65A8F
:1053080020EE0AF0A451D926A551DA22B3C0DEFF57
:10531800B4C0DEFFB5C0DEFFB6C0DEFFA4C0D9FF53
:10532800A5C0DAFFDECF18F0DDCF19F0B3C01AF050
:10533800B4C01BF0B5C01CF0B6C01DF0D6EC4DF0E3
:10534800000120EE0EF0A451D926A551DA2218C08A
:10535800DEFF19C0DEFF1AC0DEFF1BC0DEFF20EE35
:1053680004F0A451D926A551DA22B1C0DEFFB2C09B
:10537800DDFF0F0EB115A86F000EB215A96F050E4F
:10538800D890A837A937E82EFBD7A4C0D9FFA5C065
:10539800DAFFDECFAAF0DDCFABF0A851AA27A951DA
:1053A800AB232E0EAA27000EAB2320EE12F0A45139
:1053B800D926A551DA22AAC0DEFFABC0DDFF000E58
:1053C800120044C025F045C026F066EC44F0466E55
:1053D8004650D8A499D144C0D9FF45C0DAFF030E7E
:1053E800DE18D8A47DD120EE05F04450D9264550CA
:1053F800DA22DE04D8A474D12E0E44240C6E000EDA
:1054080045200D6E000E0F6E000E0E6E020E116E10
:10541800000E106E69EC59F022EE2CF04450D9269B
:105428004550DA22550EDF6E22EE2DF04450D92673
:105438004550DA22AA0EDF6E20EE2EF04450D9260F
:105448004550DA22520EDF6E20EE2FF04450D92656
:105458004550DA22520EDF6E20EE30F04450D92645
:105468004550DA22610EDF6E20EE31F04450D92625
:105478004550DA22410EDF6E22EE12F04450D92652
:105488004550DA22720EDF6E22EE13F04450D92610
:105498004550DA22720EDF6E22EE14F04450D926FF
:1054A8004550DA22410EDF6E22EE15F04450D9261F
:1054B8004550DA22610EDF6E20EE0EF04450D926F8
:1054C8004550DA2212EE16F04450E1264550E22209
:1054D800DFCFE7FF22EE17F04450D9264550DA22F5
:1054E80010EE0EF04450E1264550E222E6CF60F07F
:1054F800E5CF61F061C060F00001616B6051DF6E63
:1055080022EE18F04450D9264550DA2210EE0EF05B
:105518004450E1264550E222E6CF60F0E6CF61F044
:10552800E6CF62F0E6CF63F0110E05D0D890633372
:10553800623361336033E82EF9D76051DF6E22EEB3
:1055480019F04450D9264550DA2210EE0EF0445096
:10555800E1264550E222E6CF60F0E6CF61F0E6CFE3
:1055680062F0E6CF63F0190E05D0D890633362334A
:1055780061336033E82EF9D76051DF6E20EE0AF010
:105588004450D9264550DA2212EE1AF04450E1264A
:105598004550E222DFCFE7FF22EE1BF04450D92628
:1055A8004550DA2210EE0AF04450E1264550E22236
:1055B800E6CF60F0E5CF61F061C060F0616B6051EB
:1055C800DF6E22EE1CF04450D9264550DA2210EE48
:1055D8000AF04450E1264550E222E6CF60F0E6CFDB
:1055E80061F0E6CF62F0E6CF63F0110E05D0D890F7
:1055F8006333623361336033E82EF9D76051DF6E6D
:1056080022EE1DF04450D9264550DA2210EE0AF059
:105618004450E1264550E222E6CF60F0E6CF61F043
:10562800E6CF62F0E6CF63F0190E05D0D890633369
:10563800623361336033E82EF9D76051DF6E20EEB4
:105648001AF04450D9264550DA22DECF60F0DECF7A
:1056580061F0DECF62F0DECF63F0010E6025646F8B
:10566800000E6121656F000E6221666F000E6321D6
:10567800676F20EE2AF04450D9264550DA2264C0DC
:10568800DEFF65C0DEFF66C0DEFF67C0DEFF2E0EF0
:1056980044241B6E000E45201C6E20EE2AF0445058
:1056A800D9264550DA22DECF1DF0DECF1EF0DECF40
:1056B8001FF0DECF20F0000E226E010E216E20EECC
:1056C80001F04450D9264550DA22DF503BEC49F02E
:1056D80020EE05F04450D9264550DA22000EDF6E40
:1056E800000E1B6E000E1C6E000E1D6E20EE01F0EB
:1056F8004450D9264550DA22DF5035EC1DF0000918
:10570800D8B402D0010E466E465012008380BAEC1F
:1057180040F0CBC0B9F1CCC0BAF10101B951BA110E
:10572800D8B41BD00001FE51140D130EF324D96E0A
:10573800010EF420DA6EFE51140D130EF324E16EFF
:10574800010EF420E26EE7500409DF6EB6EC57F064
:10575800B9C1E2F0BAC1E3F012000001FE51140D24
:10576800070EF324D96E010EF420DA6E6CC1E9F04D
:105778006DC1EAF06EC1EBF0E86B000EE825EC6F46
:10578800010EE921ED6F000EEA21EE6F000EEB210C
:10579800EF6FDE50EC1945E1DE50ED1942E1DE50C5
:1057A800EE193FE1DE50EF19D8A43BD07CEC52F063
:1057B80010C0BDF111C0BEF112C0BFF113C0C0F1DD
:1057C800000EE8CF34FB2BEE35F0C0C1DFFF000E32
:1057D800E8CF36FB2BEE37F0BFC1DFFF000EE8CF76
:1057E80038FB2BEE39F0BEC1DFFF000EE8CF3AFBE5
:1057F8002BEE3BF0BDC1DFFF5250FD0B526E010E88
:105808000001876F000E866FB0EC38F05250FD0B28
:10581800526E000E4F6E83904FC0E2F00001E36BB2
:105828001200FE51140D0F0EF324D96E010EF42050
:10583800DA6EDECFE4F0DECFE5F0DECFE6F0DECFE5
:10584800E7F0E5C0E4F0E6C0E5F0E7C0E6F0E76BB6
:10585800E4C0B2F1E5C0B3F1FE51140D0F0EF3240C
:10586800D96E010EF420DA6EDECFE4F0DDCFE5F07C
:10587800E4510101BB6FBC6B5250FD0B526E000E20
:10588800B86F000EB76F000EB56F000EB46F70D012
:10589800FF0EE46FFF0EE56FB2C1E6F0B3C1E7F0AB
:1058A800E451E627E551E7230101B4510001E61967
:1058B8000EE10101B5510001E719D8A408D0010192
:1058C800BB51BC11D8A403D052500209526E00013A
:1058D800FE51200D100EF3248C6F020EF4208D6FF4
:1058E800340E8E6F0B0E8F6F010E916F000E906F3E
:1058F800C10E926F010E936FD2EC12F00101B66FD8
:10590800B651D8A40FD7C1C186F0C2C187F0B0EC98
:1059180038F00101C151B725B76FC251B821B86F2E
:105928000001FE51140D070EF324D96E010EF42068
:10593800DA6E000EDE24E46F010EDE20E56F000E45
:10594800DE20E66F000EDE20E76FFE51140D070E15
:10595800F324D96E010EF420DA6EE4C0DEFFE5C050
:10596800DEFFE6C0DEFFE7C0DEFF0101B44BB52B6A
:10597800B251B45DB551800A0001E46F0101B35121
:10598800800A0001E459D8A083D70101BCBF3ED7E3
:10599800BC5103E1BB05D8A039D70001FE51200D49
:1059A800100EF3248C6F020EF4208D6F340E8E6F60
:1059B8000B0E8F6FBBC190F0BCC191F0C10E926FFE
:1059C800010E936FD2EC12F00101B66FB651D8A454
:1059D800A9D652500209526EBBC186F0BCC187F0ED
:1059E800B0EC38F00101C151B725B76FC251B821E9
:1059F800B86F0001FE51140D070EF324D96E010E85
:105A0800F420DA6E000EDE24E46F010EDE20E56F6E
:105A1800000EDE20E66F000EDE20E76FFE51140D4B
:105A2800070EF324D96E010EF420DA6EE4C0DEFF0F
:105A3800E5C0DEFFE6C0DEFFE7C0DEFFE7D6935134
:105A4800941195119611D8A42DD020EE0AF09151F9
:105A5800D9269251DA22DECF98F0DECF99F0DECF48
:105A68009AF0DECF9BF0985199119A119B11D8B4F6
:105A780010D020EE12F09151D9269251DA22DE5040
:105A8800985DDE509959DE509A59DE509B59D8A03E
:105A98005BD0010E986F000E996F000E9A6F000E82
:105AA8009B6F52D091C060F092C061F093C062F0D9
:105AB80094C063F095C064F096C065F0B4EC21F032
:105AC80060C0A0F061C0A1F062C0A2F063C0A3F002
:105AD8000001A351A211A1110DE1020EA05DD8B0E1
:105AE80009D0010E916F000E926F000E936F000E99
:105AF800946F1200A02910E1A1290EE1A2290CE15E
:105B0800A329D8A409D0A0C091F0A1C092F0A2C046
:105B180093F0A3C094F0120020EE12F09151D92610
:105B28009251DA22DE50A05DDE50A159DE50A25912
:105B3800DE50A359D8A0E7D793C098F094C099F045
:105B480095C09AF096C09BF098C09CF099C09DF0C3
:105B58009AC09EF09BC09FF0010E9C27000E9D23CB
:105B68009E239F2320EE12F09151D9269251DA22DA
:105B7800DE509C5DDE509D59DE509E59DE509F5987
:105B8800D8A019D0020E9C6F000E9D6F000E9E6F5C
:105B9800000E9F6F9B519A1199110DE1020E985DAD
:105BA800D8B009D0000E916F000E926F000E936F5F
:105BB800000E946F120091C060F092C061F09CC01A
:105BC80062F09DC063F09EC064F09FC065F0B4ECC5
:105BD80021F060C0A0F061C0A1F062C0A2F063C073
:105BE800A3F00001A051A111A211A311D8B41DD096
:105BF800A02907E1A12905E1A22903E1A329D8B435
:105C080082D7A005A111A211A311D8B47CD79851AD
:105C18009C19A2E199519D199FE19A519E199CE105
:105C28009B519F19D8B4BED797D791C060F092C046
:105C380061F09CC062F09DC063F09EC064F09FC09C
:105C480065F0FF0E666FFF0E676FFF0E686F0F0E31
:105C5800696FC6EC1AF0976F9751D8A41DD093516D
:105C6800941195119611D8B417D091C060F092C0D4
:105C780061F093C062F094C063F095C064F096C080
:105C880065F09CC066F09DC067F09EC068F09FC03C
:105C980069F0C6EC1AF0976F9751D8A431D020EE6E
:105CA8000AF09151D9269251DA229CC0DEFF9DC09C
:105CB800DEFF9EC0DEFF9FC0DEFF20EE0EF091519A
:105CC800D9269251DA22DE2807E1DE2805E1DE280E
:105CD80003E1DE28D8B424D020EE0EF09151D92665
:105CE8009251DA22DE06000EDE5ADE5ADE5A20EE25
:105CF80005F09151D9269251DA22000EDB8010D09E
:105D08009705D8B409D0010E9C6F000E9D6F000E48
:105D18009E6F000E9F6F04D09C699D699E699F6964
:105D28009CC091F09DC092F09EC093F09FC094F0EB
:105D380012001650D96EDA6ADECF23F0DDCF24F0D8
:105D480002D0234A242A23C0F6FF24C0F7FF000EFE
:105D5800F86E0E0EF76403D00800F55005D0F6CFA4
:105D6800E9FFF7CFEAFFEF502F0AD8B4EAD723C0EC
:105D7800F6FF24C0F7FF000EF86E0E0EF76403D08E
:105D88000800F55005D0F6CFE9FFF7CFEAFFEF504E
:105D98005C0AD8B4D6D720EE14F01450D926155082
:105DA800DA22DECF25F0DDCF26F025C00CF026C0A4
:105DB8000DF0000E0F6E200E0E6E000E116E0B0E03
:105DC800106E69EC59F0000E1F6E1FC027F0286A8C
:105DD80027C01DF028C01EF0000E216E080E206E90
:105DE8001D502324176E1E502420186E17C0F6FF6E
:105DF80018C0F7FF000EF86E0E0EF76403D0080007
:105E0800F55005D0F6CFE9FFF7CFEAFFEF50296E3E
:105E18001D4A1E2A200E2964AFD02F0E2918D8B487
:105E2800ABD05C0E2918D8B4A7D02E0E2918D8B438
:105E380006D02050275C21502858D8A018D0080E2A
:105E480020182110D8A404D02E0E2918D8B402D0B6
:105E5800060E1200000E286E080E276E000E216E28
:105E68000B0E206ED8901F36D8901F36B9D77F0EEC
:105E7800296402D0030E1F12800E296403D09F0EDE
:105E8800296406D0DF0E29644ED0FD0E29604BD060
:105E98001D502324176E1E502420186E17C0F6FFBD
:105EA80018C0F7FF000EF86E0E0EF76403D0080056
:105EB800F55005D0F6CFE9FFF7CFEAFFEF50226E95
:105EC8001D4A1E2A3F0E226403D07E0E226406D08D
:105ED8007F0E2264BDD7FD0E2260BAD7FF0E176E63
:105EE800FF0E186E20C019F021C01AF0175019269D
:105EF80018501A221950275C1A502858D8B0A8D719
:105F080027502524D96E28502620DA6E29C0DFFFB5
:105F1800274A282A27502524D96E28502620DA6EA9
:105F280022C0DFFF26D0330E0C6EFE0E0D6E29C088
:105F38000EF00F6A87EC56F00C500D10D8A488D7D5
:105F4800400E296405D05B0E296002D01F8209D05B
:105F5800600E296406D07B0E296003D01F80200EB6
:105F6800295E27502524D96E28502620DA6E29C0AC
:105F7800DFFF274A282A34D71D502324176E1E50C6
:105F88002420186E1650D96EDA6A17C0DEFF18C0C2
:105F9800DDFF200E296404D0000E1C6E000E03D015
:105FA800000E1C6E040E1B6E1BC029F02750281013
:105FB800D8B44ED725C0D9FF26C0DAFFE50EDE18C3
:105FC800D8A406D025C0D9FF26C0DAFF050EDF6E9B
:105FD800080E20182110D8A404D0D8901F36D890C5
:105FE8001F361F50030BE806D8B429881F500C0B26
:105FF800040AD8B4298620EE0BF02550D92626505D
:10600800DA2229C0DFFF000E120020EE04F045500E
:10601800D9264650DA2247C0DEFF48C0DDFF20EE11
:1060280006F04550D9264650DA22DECF99F0DECF69
:106038009AF0DECF9BF0DECF9CF099059A119B1168
:106048009C11D8B414D045C0D9FF46C0DAFF10EE71
:1060580012F0DE50E126DD50E222E650995DE6506E
:106068009A59E6509B59E6509C59D8A002D0020E86
:10607800120099519A119B119C11D8A422D045C0A5
:10608800D9FF46C0DAFFDECF8CF0DDCF8DF08CC0B3
:10609800D9FF8DC0DAFF030EDE18D8A412D045C090
:1060A800D9FF46C0DAFF10EE22F0DE50E126DD50BF
:1060B800E222E6CF99F0E6CF9AF0E6CF9BF0E6CF62
:1060C8009CF099519A119B119C11D8A423D045C0DA
:1060D800D9FF46C0DAFF10EE08F0DE50E126DD50A9
:1060E800E222E650475CE6504858D8B0C0D745C0D1
:1060F800D9FF46C0DAFF10EE22F0DE50E126DD506F
:10610800E222E6CF95F0E6CF96F0E6CF97F0E6CF1D
:1061180098F079D045C0D9FF46C0DAFF10EE02F0FA
:10612800DE50E126DD50E222E7508C6F8C51100DD5
:10613800F3CF93F0F4CF94F046D045C0D9FF46C0D2
:10614800DAFFDECF60F0DDCF61F099C062F09AC06F
:1061580063F09BC064F09CC065F0B4EC21F060C0B3
:1061680099F061C09AF062C09BF063C09CF0000196
:10617800992909E19A2907E19B2905E19C29D8A4D5
:1061880002D0010E12009C519B119A1104E1020EDB
:10619800995DD8A06CD745C0D9FF46C0DAFF10EE8C
:1061A80012F0DE50E126DD50E222E650995DE6501D
:1061B8009A59E6509B59E6509C59D8B058D79351F4
:1061C800475E9451485A9351475C94514858D8B007
:1061D800B4D745C0D9FF46C0DAFFDECF18F0DDCF0F
:1061E80019F099C01AF09AC01BF09BC01CF09CC013
:1061F8001DF0D6EC4DF018C095F019C096F01AC0F5
:1062080097F01BC098F020EE0AF04550D92646506A
:10621800DA2299C0DEFF9AC0DEFF9BC0DEFF9CC079
:10622800DEFF00019551961197119811D8B41FD728
:1062380047C08CF048C08DF0040E8E6FD8908D3317
:106248008C338E2FFBD78C5195258F6F8D519621CE
:10625800906F000E9721916F000E9821926F20EE9B
:106268000EF04550D9264650DA228FC0DEFF90C086
:10627800DEFF91C0DEFF92C0DEFF0F0E47148C6F69
:10628800000E48148D6F050ED8908C378D37E82E88
:10629800FBD745C0D9FF46C0DAFFDECF8EF0DDCF91
:1062A8008FF08C518E278D518F232E0E8E27000E46
:1062B8008F2320EE12F04550D9264650DA228EC0A0
:1062C800DEFF8FC0DDFF000E1200000E0101E26F3D
:1062D8000A0EE16F000EE06F050EDF6F43D1000E6E
:1062E8000101E26F140EE16F34D1130E0D6EFD0E35
:1062F8000E6EECEC55F08FB205D0000E0101E26F86
:106308001E0EE16F290E0001FA6F960EF96F7F0ECF
:10631800E82EFED7F92FFCD7FA2FFAD71AD1EB0EB1
:106328000D6EFE0E0E6EECEC55F0060E0001D86FE9
:10633800090ED96FB60EDA6FFB0EDB6F000EDC6F3D
:1063480033EC4EF0FF6FFF51DAEC54F00001FF51CF
:10635800D8A4D8D7000E0101E26F230ED2D76F0E52
:106368000D6EFE0E0E6EECEC55F0100E0001D86F9F
:10637800020ED96F0E0EDA6FFF0EDB6F010EDC6FA7
:1063880044EC18F00001FF6FFF51DAEC54F0000103
:10639800FF51D8A40AD0E8EC25F0100E0001736F65
:1063A800020E746FF4EC57F0FF6FFF51DAEC54F003
:1063B800000E0101E26F280EE16FA151D8A40ED0A2
:1063C800000EEB6F340E0001766F0D0E776FC50E61
:1063D800786FFE0E796FF0EC56F00DD01C0E0001B0
:1063E800606FFC0E616FA1C162F0636BEBC164F07A
:1063F800656B21EC5AF07E0E0001606FFE0E616F36
:106408000101EB510F0D340EF3240001626F0D0EE4
:10641800F420636F21EC5AF075D7E50E606FFC0E1F
:10642800616F0101EB510F0D340EF3240001626F0F
:106438000D0EF420636F21EC5AF0100E0001D86F96
:10644800020ED96F0101EB510F0D340EF324000138
:10645800DA6F0D0EF420DB6F030EDC6F44EC18F0DE
:106468000001FF6FFF51D8A405D0000E0101E26FB3
:106478003C0EE16F040E0001FF19D8A443D7000EAB
:106488000101E26F320E3DD74D0E606FFD0E616F58
:106498000101EB510F0D340EF3240001626F0D0E54
:1064A800F420636F21EC5AF0100E0001D86F020E31
:1064B800D96F0101EB510F0D340EF3240001DA6F8F
:1064C8000D0EF420DB6F070EDC6F44EC18F00001B2
:1064D800FF6FFF51D8A416D7000E0101E26F3C0EE2
:1064E80010D7270E606FFD0E616F0101EB510F0D84
:1064F800340EF3240001626F0D0EF420636F21EC5B
:106508005AF0000E0001F86F010EF76F1200E1C19A
:10651800F9F0E2C1FAF00001FA51000AD8A419D042
:10652800F9510A0AD8B4DBD61E0AD8B4DED60A0A4C
:10653800D8B4F5D63D0AD8B412D70B0AD8B46DD75B
:10654800050AD8B406D01F0AD8B49ED70E0AD8B404
:10655800C8D7140E0101E119E211D8B403D0DF073E
:10656800D8A0E007E0BF05D0E051D1E1DF05D8B001
:10657800CED7000E0001F86F000EF76F1200340E30
:106588000101BE6F0B0EBF6FEBC012F0ECC013F031
:1065980012EC57F012500101B26FCB0E0001A46F3C
:1065A800A56B000EA66F000EA76F000EA86F000E59
:1065B800A96FCDEC0FF00101BB6FBB51D8B411D05E
:1065C8006E0E0001606FFC0E616F21EC5AF0000E38
:1065D8000001CB6F000ECC6F000ECD6F000ECE6F9A
:1065E8001200CB0E00018C6F8D6BBEC18EF0BFC147
:1065F8008FF0010E916F000E906FB90E926F010E21
:10660800936FD2EC12F00101BB6FBB51D8B408D024
:10661800CE0E0001606FFC0E616F21EC5AF0D7D7E7
:10662800BEC1D9FFBFC1DAFF800EDE18D8B408D0CA
:10663800700E0001606FFD0E616F21EC5AF0C7D734
:1066480020EE0AF0BE51D926BF51DA22DF500001F0
:10665800ED6FED51EF6FEE6B010120EE0BF0BE51C7
:10666800D926BF51DA22DF500001F06FF051EE2534
:106678000101B76F000E0001EF210101B86FB70EDD
:106688000001606FFC0E616FB7C162F0B8C163F0C2
:1066980021EC5AF0CB0E0001A46FA56B0101B75194
:1066A8000001EE6FED6BEDC0A6F0EEC0A7F0A86B91
:1066B800A96BCDEC0FF00101BB6FBB51D8A487D7F4
:1066C800CB0E00018C6F8D6BBEC18EF0BFC18FF0F9
:1066D800010E916F000E906FB90E926F010E936FBD
:1066E800D2EC12F00101BB6FBB51D8A470D7000ED9
:1066F800BD6F000EBC6FEBC00CF0ECC00DF0BCC160
:10670800EDF0BDC1EEF0050ED8900001ED37EE3783
:10671800E82EFAD7ED510101BE250E6E0001EE51AB
:106728000101BF210F6EB2C110F0116A2BEC4FF0BE
:106738000C500D10D8A45FD0BCC1EDF0BDC1EEF077
:10674800050ED8900001ED37EE37E82EFAD7BEC116
:10675800EFF0BFC1F0F0ED51EF27EE51F0230E0E30
:10676800EF25D96E000EF021DA6EDF50F16FF1518E
:10677800F36FF26BBCC1F4F0BDC1F5F0050ED89013
:10678800F437F537E82EFBD7BEC1F6F0BFC1F7F0F6
:10679800F451F627F551F7230F0EF625D96E000EA2
:1067A800F721DA6EDF50F86FF96BF251F827F351E1
:1067B800F923F8C0B3F1F9C0B4F10101000EB4BF78
:1067C800FF0EB56FB66F240E0001606FFE0E616F8D
:1067D800B3C162F0B4C163F0B5C164F0B6C165F08D
:1067E80021EC5AF0B3C1CBF0B4C1CCF0B5C1CDF0B7
:1067F800B6C1CEF01200BC4BBD2BBDBF7CD7BD517E
:1068080005E10F0EBC5DD8B0E2D675D7E0D6000121
:10681800A36F00019F51D8A441EC42F0000E000183
:10682800A26F9E51D8B417D1040EA319D8B404D0BE
:10683800140EA319D8A40DD0000E0101986F000EF4
:10684800836F000E826F000E00019F6F070E9E6F10
:1068580012003F0EA319D8A40BD0000EFD6F000E36
:106868000101986F000E00019F6F000E9E6F1200CD
:106878005F0EA319D8A40BD0000E0101996F000E6A
:10688800986F000E00019F6F000E9E6F12003F0E62
:10689800A36507D05F0EA36104D0400EA319D8A446
:1068A800EBD7400EA319D8A40BD0010E0101996FA4
:1068B800000E986F000E00019F6F000E9E6F120071
:1068C800200EA319D8A412D0010EFD6F000E0101ED
:1068D800986F820E0001606FFF0E616F21EC5AF015
:1068E800000E00019F6F000E9E6F1200650EA31927
:1068F800D8A410D0FD51D8B40DD0000E0101836F7B
:10690800000E826F010E986F000E00019F6F000E3F
:106918009E6F12006E0EA319D8A403D0020E0101B7
:10692800986F700E0001A319D8A40AD001019951DB
:10693800D8B406D0000E836F000E826F030E986FD6
:10694800700E0001A319D8A411D0FD51D8B40ED0EF
:106958008380000E0101836F000E826F040E986F12
:10696800000E00019F6F000E9E6F1200720EA31999
:10697800D8A471D0FD51D8B46ED083801C0E01010B
:10698800836F2A0E826F050E986F000E00019F6FAD
:10699800000E9E6F1200A3519DEC15F0000148D027
:1069A8008380A351F5EC52F00001A26F000E0101A3
:1069B800986F6DD08380340E0C6E0B0E0D6E000E2A
:1069C8000F6E000E0E6E010E116E000E106EB5ECFD
:1069D80045F052500209526E2BEE34F04FC0DFFFE3
:1069E800810E0001606FFD0E616F000E636F010E76
:1069F800626F21EC5AF0340E0001866F0B0E876F20
:106A0800000E896F010E886F660E8A6FFF0E8B6FFE
:106A1800C6EC39F0000E0001876F010E866FB0ECEE
:106A280038F05250FD0B526E080EBED78390000E00
:106A3800A26F2DD0080EA319D8A429D08390000ED8
:106A4800A26F000E4F6E000E0101986F000E836F4B
:106A5800000E826F1CD0010198510001A06FA16B3C
:106A6800A151000AD8A413D0A051000AD8B40FD05D
:106A7800010AD8B490D7030AD8B492D7010AD8B477
:106A880099D7070AD8B4D2D7010AD8B4D3D7A2C0A5
:106A98009EF000019F6B120020EE04F06051D92691
:106AA8006151DA22000EDF6E20EE2AF06051D926FD
:106AB8006151DA22FF0EDE6EFF0EDE6EFF0EDE6E15
:106AC800FF0EDD6E60C03AF061C03BF062C03CF082
:106AD80063C03DF064C03EF065C03FF087EC4EF007
:106AE8000009D8B402D0030E1200000122EE2DF0E6
:106AF8006051D9266151DA22DF50666F6651686F9E
:106B0800676B22EE2CF06051D9266151DA22DF50F2
:106B1800696F69516713000E6813550E671904E110
:106B2800AA0E6819D8B402D0020E120020EE65F041
:106B38006051D9266151DA22DF50666F6651686F5D
:106B4800676B20EE66F06051D9266151DA22DF507A
:106B5800696F69C06AF06B6B6C6B6D6B6BC06DF0C5
:106B68006AC06CF06B6B6A6B20EE67F06051D926D7
:106B78006151DA22DF506E6F6EC06FF0706B716B0F
:106B8800726B6FC072F0716B706B6F6B6A516F11C3
:106B9800736F6B517011746F6C517111756F6D510A
:106BA8007211766F67517311776F68517411786F2E
:106BB800000E7511796F000E76117A6F20EE64F071
:106BC8006051D9266151DA22DF507B6F7B517711F2
:106BD8007C6F78517D6F79517E6F7A517F6FFF0E90
:106BE8007C15806FFF0E7D15816FFF0E7E15826FFD
:106BF800000E7F15836F460E80190AE1410E811938
:106C080007E1540E82198311D8A402D0000E120095
:106C180020EE81F06051D9266151DA22DF50666F8B
:106C28006651686F676B20EE82F06051D92661511A
:106C3800DA22DF50696F69C06AF06B6B6C6B6D6B41
:106C48006BC06DF06AC06CF06B6B6A6B20EE83F002
:106C58006051D9266151DA22DF506E6F6EC06FF035
:106C6800706B716B726B6FC072F0716B706B6F6B66
:106C78006A516F11736F6B517011746F6C51711190
:106C8800756F6D517211766F67517311776F685117
:106C98007411786F000E7511796F000E76117A6F86
:106CA80020EE80F06051D9266151DA22DF507B6FE7
:106CB8007B5177117C6F78517D6F79517E6F7A5156
:106CC8007F6FFF0E7C15806FFF0E7D15816FFF0EA5
:106CD8007E15826F000E7F15836F460E801908E1BE
:106CE800410E811905E1540E82198311D8B48ED74B
:106CF800010E12008380000E4F6EBAEC40F0CBC03C
:106D0800B6F1CCC0B7F10101B651B711D8B405D06E
:106D1800B6C1EDF0B7C1EEF01200000EB86F000E6C
:106D2800B96F000EBA6F000EBB6F000EB56F010E83
:106D3800B46F000EBE6FE9D0000EBD6F000EBC6FC1
:106D48001DD064EC5AF00C500D10D8B413D0BE0E00
:106D58000C6E010E0D6E5FEC50F00101B36F000E6A
:106D6800AB25D96EDA6A040EDA22B3C1DFFFAB2B8A
:106D7800BC4BBD2B0101BEAB8EAC05D0BDBFE1D76E
:106D8800BD05D8A0DED7BCC1EFF0BDC1F0F0000E44
:106D98000001F0BFFF0EF16FF26F0101B851000161
:106DA800EF250101B86FB9510001F0210101B96F58
:106DB800BA510001F1210101BA6FBB510001F22162
:106DC8000101BB6F0001FE51140D0F0EF324D96EA3
:106DD800010EF420DA6EDE500101B85DDE50B959BB
:106DE800DE50BA59DE50BB59D8A004D0000EB56F9A
:106DF800000EB46FBEAB04D0000EB56F000EB46FBA
:106E08008EBC04D0000EB56F000EB46FBDBF03D0AA
:106E1800BD05D8B01DD0000EAB250C6E0D6A040E52
:106E28000D22FF0EAB25D96EDA6A030EDA22DF5087
:106E38000001EF6FEF510E6E0F6A0101AB510008B0
:106E4800106E000ED8A0E82A0108116EB5EC45F0C6
:106E58000001FE51140D070EF324D96E010EF42023
:106E6800DA6E6CC1F4F06DC1F5F06EC1F6F0F36B3B
:106E7800000EF325F76F010EF421F86F000EF521CF
:106E8800F96F000EF621FA6FDE50F7191CE1DE509B
:106E9800F81919E1DE50F91916E1DE50FA19D8A4EB
:106EA80012D001C4C2F103C4C1F105C4C0F107C4C2
:106EB800BFF1BFC10FF0C0C110F0C1C111F0C2C114
:106EC80012F096EC55F06BEC53F0E2510101B26F01
:106ED800B251D8B41AD0010E4F6E0001FE51140DF4
:106EE800130EF324D96E010EF420DA6EFE51140D40
:106EF800130EF324E16E010EF420E26EE75004094C
:106F0800DF6E4FC0EDF0EE6B1200B451B511D8A48E
:106F180013D78FA402D0010E4F6E8390000E00018C
:106F2800EE6F000EED6F12007DAF49927DBF05D068
:106F38007D5109E17C05D8B006D0000E0001656FCF
:106F4800010E646F04D07CC164F07DC165F07AC124
:106F580066F07BC167F049A805D00001FE0E6627E0
:106F6800FF0E672326C068F027C069F028C06AF0C2
:106F780029C06BF02AC06CF02BC06DF02CC06EF0ED
:106F88002DC06FF0000E0001716F1F0E706F000EA4
:106F98000201AF6F93D07007D8A071070F0E681564
:106FA800726F736B73BF08D0735104E10A0E725D80
:106FB800D8A002D0570E01D0300E7225726F000E85
:106FC8007321736FBF0E2F6EFF0E306E2E50316E11
:106FD800326A2F50312630503222325006E11A0ED2
:106FE800315CD8B002D0010E01D0000E606F616B29
:106FF80060516111D8B427D09F0E2F6EFF0E306EEE
:10700800200E7211316E000E7311326E2F50312620
:1070180030503222325006E11A0E315CD8B002D01C
:10702800010E01D0000E626F636B62516311D8B418
:107038000AD072C012F073C013F062EC56F012C09E
:1070480072F013C073F0900E7025D96E020E712184
:10705800DA6E72C0DFFF6407D8A065076607D8A09C
:10706800670768C02FF069C030F06AC031F06BC0A4
:1070780032F06CC033F06DC034F06EC035F06FC0C4
:1070880036F0050E09D0D8903632353234323332E4
:107098003232313230322F32E82EF5D72FC068F035
:1070A80030C069F031C06AF032C06BF033C06CF0A8
:1070B80034C06DF035C06EF036C06FF0000171BF9E
:1070C80020D0715104E1020E705DD8A01AD0685129
:1070D80069116A116B116C116D116E116F11D8A4C1
:1070E8005AD765BF05D0655102E16405D8B053D7BA
:1070F80067BF07D0675103E16605D8A002D049B23F
:107108004AD749A816D07007D8A07107900E7025E5
:10711800D96E020E7121DA6E2EC0DFFF7007D8A07B
:107128007107900E7025D96E020E7121DA6E300E3D
:10713800DF6E25C01BF0900E70251C6E020E7121AB
:107148001D6E66C01EF067C01FF036EC51F01BC004
:1071580025F01CC026F01200000E0101A96F000ED8
:107168004C6E000E4B6E8986898089828984898855
:107178008B688490849284948498838E83B40FD08F
:10718800E9A707D0B70E0001606FFB0E616F21EC15
:107198005AF0000E0001876F000E866F12000F0173
:1071A8001391350EE82EFED700F0D7D08EB808D050
:1071B8008B680F0113814BC086F04CC087F012001A
:1071C8008EB80BD08D0E0001606FFE0E616F21EC42
:1071D8005AF0630E0101A96FC7D0100E746F270E05
:1071E800756F000E766F000E776F96D08EB28EA4F4
:1071F80011D001017407000E755B765B775B74290B
:1072080006E1752904E1762902E17729D8A4A5D0F9
:10721800620E02D0010E77D0A96F9FD08EA89DD0A4
:10722800020E71D0FF0E886FFF0E896F86C08AF03C
:1072380087C08BF088518A2789518B234B508A1934
:1072480006E14C508B19D8B452A201D0899A340E59
:107258004B24D96E0B0E4C20DA6EDF50FF0A866E77
:107268004B4A4C2A000E8B6E030E23D0100E746FFF
:10727800270E756F000E766F000E776F6ED08EB288
:107288000FD001017407000E755B765B775B74297C
:107298000AE1752908E1762906E17729D8A403D0FF
:1072A800040E0101A96F8EA258D0040EB5D789909B
:1072B800050E0101A96FDAD789848EB40FD00101B8
:1072C8007407000E755B765B775B74290AE1752994
:1072D80008E1762906E17729D8A403D0060E010132
:1072E800A96F8EA43AD0060E97D7898A89808B68B1
:1072F80086514B5C4C50800A886F8751800A8859A8
:10730800D8A088D7630E010187D7A00E606FFF0E43
:10731800616F21EC5AF0F6D7A9510001886F896B8B
:107328008951000AD8A419D08851000AD8B45ED768
:10733800010AD8B473D7030AD8B474D7010AD8B4E9
:107348009ED7070AD8B4B3D7010AD8B4B5D7030A69
:10735800D8B4CBD7640AD8B4D8D7630E0101A91919
:10736800D8B402D08EBC22D7898089828984898842
:10737800898A8B68839E0F0113814BC086F04CC0AD
:1073880087F01200D20E606FFE0E616F8AC062F045
:107398008BC063F086C064F087C065F088C066F073
:1073A80089C067F021EC5AF0000E0001936F000EBF
:1073B800926FD7D0B40E606FFB0E616F21EC5AF05C
:1073C800000E0001956F000E946F29D092C08CF0CA
:1073D80093C08DF08C3B8D3BF00E8D178C510F0BAD
:1073E8008D13F00E8C1786C08EF087C08FF08C51ED
:1073F8008E278D518F2394518E25D96E95518F21CB
:10740800DA6EDF50916F9A0E606FFF0E616F91C058
:1074180062F0636B21EC5AF00001944B952B95BFF9
:1074280006D095511FE1100E945DD8B01BD092C0C4
:107438008CF093C08DF08C3B8D3BF00E8D178C51EA
:107448000F0B8D13F00E8C1794518C2795518D23AB
:107458008C51885D8951800A8E6F8D51800A8E59B2
:10746800D8B0B4D7DF0E606FFF0E616F21EC5AF011
:10747800000E0001956F000E946F4ED092C08CF0F4
:1074880093C08DF08C3B8D3BF00E8D178C510F0BFC
:107498008D13F00E8C1786C08EF087C08FF08C513C
:1074A8008E278D518F2394518E25D96E95518F211A
:1074B800DA6E200EDF6427D0FB0E606FFF0E616F5F
:1074C80092C08CF093C08DF08C3B8D3BF00E8D17E5
:1074D8008C510F0B8D13F00E8C1786C08EF087C061
:1074E8008FF08C518E278D518F2394518E25D96E14
:1074F80095518F21DA6EDF50906F9051626F636BF8
:1075080021EC5AF006D00C0E606FFF0E616F21EC73
:107518005AF00001944B952B95BF06D095511FE169
:10752800100E945DD8B01BD092C08CF093C08DF033
:107538008C3B8D3BF00E8D178C510F0B8D13F00E7D
:107548008C1794518C2795518D238C51885D8951C6
:10755800800A8E6F8D51800A8E59D8B08FD7924B82
:10756800932B93BF06D093511BE1500E925DD8B078
:1075780017D092C08CF093C08DF08C3B8D3BF00EF1
:107588008D178C510F0B8D13F00E8C1788518C5D55
:107598008D51800A8E6F8951800A8E59D8A00AD7DA
:1075A800B40E606FFB0E616F21EC5AF0120047C0F9
:1075B8000DF048C00EF015EC50F000016C6F6C51E6
:1075C800D8A405D120EE04F04750D9264850DA2235
:1075D800DFAAFDD047C0D9FF48C0DAFFDECF3AF0B6
:1075E800DDCF3BF020EE1AF04750D9264850DA227A
:1075F800DECF3CF0DECF3DF0DECF3EF0DECF3FF019
:1076080087EC4EF000016C6F6C51D8A4E0D020EEEE
:107618001EF04750D9264850DA22DECF71F0DDCF70
:1076280072F020EE0BF07151D9267251DA22000E59
:10763800DB8A20EE0AF04750D9264850DA2210EEAD
:107648001CF07151E1267251E222DFCFE7FF20EEF4
:107658001DF07151D9267251DA2210EE0AF0475006
:10766800E1264850E222E6CF68F0E5CF69F069C02C
:1076780068F0696B6851DF6E20EE1EF07151D926F3
:107688007251DA2210EE0AF04750E1264850E22201
:10769800E6CF68F0E6CF69F0E6CF6AF0E6CF6BF0A8
:1076A800110E05D0D8906B336A3369336833E82EEE
:1076B800F9D76851DF6E20EE1FF07151D92672514B
:1076C800DA2210EE0AF04750E1264850E222E6CFCF
:1076D80068F0E6CF69F0E6CF6AF0E6CF6BF0190EF6
:1076E80005D0D8906B336A3369336833E82EF9D7FD
:1076F8006851DF6E71C00CF072C00DF020EE0EF014
:107708004750D9264850DA22DECF0EF0DECF0FF0F0
:10771800DECF10F0DECF11F034EC57F0000E000190
:107728006D6F000E6E6F210E6F6F460E706F20EE3C
:1077380016F07151D9267251DA22000EDF6E20EE52
:1077480017F07151D9267251DA226EC0DFFF20EE90
:1077580018F07151D9267251DA226FC0DFFF20EE7E
:1077680019F07151D9267251DA2270C0DFFF20EE6C
:1077780012F07151D9267251DA22000EDF6E20EE16
:1077880013F07151D9267251DA22000EDF6E20EE05
:1077980004F04750D9264850DA22DF0EDF1647C0DA
:1077A800D9FF48C0DAFF10EE04F0DE50E126DD50C4
:1077B800E222010EE76E47C0D9FF48C0DAFFDECFEC
:1077C80044F0DDCF45F0E5EC29F000016C6F6C5119
:1077D80012000001FE51070D520EF324D96E010E5E
:1077E800F420DA6EDF2AFE51070D520EF324D96E0B
:1077F800010EF420DA6E0F0EDF6431D0FE51070D52
:10780800520EF324D96E010EF420DA6E000EDF6EEC
:10781800FE51070D510EF324D96E010EF420DA6ED5
:10782800DF2AFE51070D510EF324D96E010EF42004
:10783800DA6E010EDF6413D0FE51070D510EF324EA
:10784800D96E010EF420DA6E000EDF6EFE51070DC0
:10785800500EF324D96E010EF420DA6EDF2AFE51A1
:10786800070D520EF324D96E010EF420DA6EDF50A4
:10787800CB6FCBC0CCF0CD6BCE6BCF6BCEC0CFF087
:10788800CDC0CEF0CCC0CDF0CC6BFE51070D510E63
:10789800F324D96E010EF420DA6EDF50D06FD0C019
:1078A800D1F0D26BD36BD46BD3C0D4F0D2C0D3F0A9
:1078B800D1C0D2F0D16B040ED890D137D237D3379C
:1078C800D437E82EF9D7FE51070D500EF324D96EA0
:1078D800010EF420DA6EDF50D56FD5C0D6F0D76B25
:1078E800D86BD96B040ED890D637D737D837D93755
:1078F800E82EF9D7D8C0D9F0D7C0D8F0D6C0D7F07D
:10790800D66BD890D635DA6FD735DB6FD835DC6FC4
:10791800D935DD6FD151DA25DE6FD251DB21DF6F2A
:10792800D351DC21E06FD451DD21E16FCC51DE254C
:10793800E26FCD51DF21E36FCE51E021E46FCF51EB
:10794800E121E56FFE51070D530EF324D96E010EA8
:10795800F420DA6EE2C0DEFFE3C0DEFFE4C0DEFF43
:10796800E5C0DEFFFE51200D100EF324A46F020EB9
:10797800F420A56FFE51070D530EF324D96E010EA6
:10798800F420DA6EDECFA6F0DECFA7F0DECFA8F0C7
:10799800DECFA9F0CDEC0FF0E66FE651D8B419D0E0
:1079A800870E606FFC0E616FFE51070D530EF324B6
:1079B800D96E010EF420DA6EDECF62F0DECF63F00E
:1079C800DECF64F0DECF65F0E6C066F0676B21ECD1
:1079D8005AF0000E0101976F120052500209526EC0
:1079E800340E0C6E0B0E0D6E000E0F6E000E0E6E2A
:1079F800010E116E000E106EB5EC45F02BEE34F052
:107A0800FEC0DFFFFF0EE8CF35FB0001FE51140D6D
:107A1800130EF324D96E010EF420DA6E0101DFA4EF
:107A280003D0010EE8CF38FB0001FE51140D130EF0
:107A3800F324D96E010EF420DA6E0101DFA003D021
:107A4800020EE8CF3AFB0001FE51140D130EF32489
:107A5800D96E010EF420DA6E0101DFA203D0020E06
:107A6800E8CF3AFB8FA403D0080EE8CF3AFB000E0C
:107A780000018F6F000E8E6FFC0E606FFB0E616F42
:107A8800CECF62F0636BCDCF64F0656B8EC066F0CD
:107A98008FC067F0360E8E25D96E0B0E8F21DA6EE9
:107AA800DF508C6F8C51686F696B21EC5AF0000EB7
:107AB80000018E25D96E020E8F21DA6EDF50FF0A83
:107AC8008D6F360E8E25D96E0B0E8F21DA6E360E1F
:107AD8008E25E16E0B0E8F21E26EE7508D15DF6E5D
:107AE8005F0E606FFF0E616F360E8E25D96E0B0E1E
:107AF8008F21DA6EDF508C6F8C51626F636B21ECD3
:107B08005AF000018E4B8F2B8FBFB6D78F5104E1EF
:107B1800070E8E5DD8A0B0D7FE51140D130EF324B6
:107B2800D96E010EF420DA6EDF504F6EFE51140D3F
:107B3800010EF324D96E010EF420DA6EDF508C6F3B
:107B48008CC03FFBFE51140D020EF324D96E010EBA
:107B5800F420DA6EDF508C6F8CC040FBFE51140DA0
:107B6800030EF324D96E010EF420DA6EDF508C6F09
:107B78008CC041FBFE51140D040EF324D96E010E86
:107B8800F420DA6EDF508C6F8CC042FBFE51140D6E
:107B9800050EF324D96E010EF420DA6EDF508C6FD7
:107BA8008CC043FBFE51140D060EF324D96E010E52
:107BB800F420DA6EDF508C6F8CC044FB000E876FA8
:107BC800140E866FB0EC38F05250FD0B526E839055
:107BD80012008EA605D04E0E0001876FFE0E04D04F
:107BE800B50E0001876FFF0E886F8EAA04D04E0E67
:107BF800896FFE0E03D0B00E896FFF0E8A6F8EA8B4
:107C080004D04E0E8B6FFE0E03D0BA0E8B6FFF0E94
:107C18008C6F8EAE04D04E0E8D6FFE0E03D0BF0E4D
:107C28008D6FFF0E8E6F8EAC04D04E0E8F6FFE0ED2
:107C380003D0AB0E8F6FFF0E906F8EA404D04E0E44
:107C4800916FFE0E03D0C90E916FFF0E926F8EA238
:107C580004D04E0E936FFE0E03D0CE0E936FFF0E20
:107C6800946F8EA004D04E0E956FFE0E03D0C40EF6
:107C7800956FFF0E966F90AE04D04E0E976FFE0E66
:107C880003D0F80E976FFF0E986F90AC04D04E0E8D
:107C9800996FFE0E03D0F50E996FFF0E9A6F90AA9A
:107CA80004D04E0E9B6FFE0E03D0F20E9B6FFF0E9C
:107CB8009C6F90A804D04E0E9D6FFE0E03D0EF0E61
:107CC8009D6FFF0E9E6F90A604D04E0E9F6FFE0E06
:107CD80003D0EC0E9F6FFF0EA06F90A404D04E0E41
:107CE800A16FFE0E03D0E90EA16FFF0EA26F90A246
:107CF80004D04E0EA36FFE0E03D0E60EA36FFF0E48
:107D0800A46F90A004D04E0EA56FFE0E03D0E30E14
:107D1800A56FFF0EA66F3A0E606FFB0E616F905055
:107D2800FF0A866F8651626F636B8ECF64F0656B56
:107D3800A5C066F0A6C067F0A3C068F0A4C069F04B
:107D4800A1C06AF0A2C06BF09FC06CF0A0C06DF03B
:107D58009DC06EF09EC06FF09BC070F09CC071F02B
:107D680099C072F09AC073F097C074F098C075F01B
:107D780095C076F096C077F093C078F094C079F00B
:107D880091C07AF092C07BF08FC07CF090C07DF0FB
:107D98008DC07EF08EC07FF08BC080F08CC081F0EB
:107DA80089C082F08AC083F087C084F088C085F0DB
:107DB80021EC5AF01200000E0001C86F010EC76FC7
:107DC8008380000EC16F000EC26F000EC36F000EDD
:107DD800C46FD6D0FE51200D100EF3248C6F020E06
:107DE800F4208D6F340E8E6F0B0E8F6F010E916F16
:107DF800000E906FCB0E926F936BD2EC12F0FE5187
:107E0800070D530EF324D96E010EF420DA6E6CC1FF
:107E1800B9F06DC1BAF06EC1BBF0B86B000EB825F1
:107E2800BC6F010EB921BD6F000EBA21BE6F000EE6
:107E3800BB21BF6FDE50BC1930E1DE50BD192DE10A
:107E4800DE50BE192AE1DE50BF19D8A426D07CEC3A
:107E580052F010C0CDF011C0CEF012C0CFF013C058
:107E6800D0F0000EE8CF34FB2BEE35F0D0C0DFFFAA
:107E7800000EE8CF36FB2BEE37F0CFC0DFFF000E49
:107E8800E8CF38FB2BEE39F0CEC0DFFF000EE8CF8D
:107E98003AFB2BEE3BF0CDC0DFFF5250FD0B526E8C
:107EA800CBC086F0CCC087F0B0EC38F086C0C9F003
:107EB80087C0CAF00001C951C125C16FCA51C2218A
:107EC800C26F000EC321C36F000EC421C46F8EACF5
:107ED8005CD0CB51C91904E1CC51CA19D8B40BD024
:107EE800DF0E606FFE0E616FC9C062F0CAC063F03A
:107EF80021EC5AF04AD093EC59F064EC5AF00C504B
:107F08000D10D8B404D0010E0101976F3ED0000EB9
:107F18000001C66F050EC56F1FD0D00E0001B46FEB
:107F2800C90EE82EFED7B42FFCD700D064EC5AF067
:107F38000C500D10D8B410D0000E0001C86F000E00
:107F4800C76FB40E606FFD0E616FC5C062F0C6C02A
:107F580063F021EC5AF009D00001C507D8A0C60784
:107F6800C529DBE1C629D8A4D8D764EC5AF00C504F
:107F78000D10D8B405D0000E0001C86F000EC76FF1
:107F88000001C751C811D8A425D7000E0101976F69
:107F9800839012001C6E1C50D8B402D0010E12003F
:107FA80053A202D053501200000E3BEC59F00A0EB7
:107FB800276E03D058EC5AF027062750D8A4FAD7D2
:107FC800000E246E000E156E000E166E000E176E53
:107FD800000E186E000E55EC57F0E806D8A4BDD078
:107FE800AA0E156E010E166E000E176E000E186E94
:107FF800080E55EC57F0E806D8A462D0000E276E9C
:1080080027501D0FD96EDA6A58EC5AF0DF6E272A0E
:10801800030E2764F5D71F04D8A49FD0AA0E2018F2
:10802800D8A49BD0030E266EE80E256E19D0000E3C
:10803800156E000E166E000E176E400E186EA90E05
:1080480055EC57F00009D8B40FD0150E1B6EC60EAC
:10805800E82EFED71B2EFCD700D02506D8A0260672
:1080680025502610D8A4E3D725502610D8B475D0AB
:10807800000E156E000E166E000E176E000E186EAE
:108088003A0E55EC57F00009D8A467D0000E276EB9
:1080980027501D0FD96EDA6A58EC5AF0DF6E272A7E
:1080A800030E2764F5D71DBC04D0000E226E040E03
:1080B80003D0000E226E0C0E216E21C024F04DD08C
:1080C800000E156E000E166E000E176E000E186E5E
:1080D800A90E55EC57F01B6E020E1B6004D0020E61
:1080E800246EA90E03D0010E246E010E236E030E1A
:1080F800266EE80E256E19D0000E156E000E166E4F
:10810800000E176E000E186E235055EC57F000093C
:10811800D8B40FD0150E1B6EC60EE82EFED71B2E38
:10812800FCD700D02506D8A0260625502610D8A4AE
:10813800E3D725502610D8B40ED0000E156E020EC7
:10814800166E000E176E000E186E100E55EC57F0D6
:108158000009D8B402D0000E246E24C050F069EC97
:108168005AF02450D8B41ED753901CD70001FE51A2
:10817800140D070EF324D96E010EF420DA6EDECF4B
:10818800DDF0DECFDEF0DECFDFF0DECFE0F0FE5157
:10819800140D070EF324D96E010EF420DA6EFE5189
:1081A800140D0B0EF324E16E010EF420E26EDE5086
:1081B800E65CDE50E658DE50E658DE50E658D8B0A9
:1081C80015D0010E4F6EFE51140D130EF324D96E07
:1081D800010EF420DA6EFE51140D130EF324E16E35
:1081E800010EF420E26EE7500409DF6EFE51140D13
:1081F8000F0EF324D96E010EF420DA6EDECFCDF027
:10820800DECFCEF0DECFCFF0DECFD0F0FE51140DB2
:10821800070EF324D96E010EF420DA6EDECFD1F00A
:10822800DECFD2F0DECFD3F0DECFD4F0CD51D125E2
:10823800D56FCE51D221D66FCF51D321D76FD05120
:10824800D421D86FFE51140D0B0EF324D96E010EF4
:10825800F420DA6ED551DE5CD651DE58D751DE589F
:10826800D851DE58D8B015D0010E4F6EFE51140DFE
:10827800130EF324D96E010EF420DA6EFE51140D9C
:10828800130EF324E16E010EF420E26EE7500409A8
:10829800DF6E000E4F6EFE51200D100EF324A46FFA
:1082A800020EF420A56FDDC0A6F0DEC0A7F0DFC087
:1082B800A8F0E0C0A9F0CDEC0FF0E16FE151D8B41F
:1082C80015D0010E4F6EFE51140D130EF324D96E06
:1082D800010EF420DA6EFE51140D130EF324E16E34
:1082E800010EF420E26EE7500409DF6E4FC0CBF0B8
:1082F800CC6B1200BFC0F6FFC0C0F7FF000EF86ECF
:108308000E0EF76403D00800F55005D0F6CFE9FF4C
:10831800F7CFEAFFEF502F0AD8B414D0BFC0F6FF4A
:10832800C0C0F7FF000EF86E0E0EF76403D0080009
:10833800F55005D0F6CFE9FFF7CFEAFFEF505C0A1A
:10834800D8A403D00001BF4BC02B000120EE06F0DB
:10835800BD51D926BE51DA22DE6ADE6ADE6ADD6ADE
:10836800BFC0F6FFC0C0F7FF000EF86E0E0EF76430
:1083780003D00800F55005D0F6CFE9FFF7CFEAFFA4
:10838800EF500001C16F200EC16116D0BDC045F08D
:10839800BEC046F0000E486E000E476E09EC30F085
:1083A800C56F20EE12F0BD51D926BE51DA22000E5B
:1083B800DE6E000EDD6E5FD0BDC014F0BEC015F0DD
:1083C800BF0E166E9DEC2EF00001C56FC551D8A4E6
:1083D80052D0BDC0B7F0BEC0B8F034EC4CF0C56F99
:1083E80020EE14F0BD51D926BE51DA2210EE0BF062
:1083F800DE50E126DD50E222E750C46FC551D8B403
:1084080008D0040EC519D8B4C4B535D0050EC56F4B
:1084180032D0C4B530D020EE12F0BD51D926BE51AD
:10842800DA22DECFC2F0DDCFC3F020EE0BF0C2516E
:10843800D926C351DA22DFA8E9D7BDC0D9FFBEC00B
:10844800DAFFDECF0CF0DDCF0DF0C2C00EF0C3C0F6
:108458000FF074EC4DF0000120EE06F0BD51D92666
:10846800BE51DA220CC0DEFF0DC0DEFF0EC0DEFFFB
:108478000FC0DEFFA1D7C5511200000EFE6F000E1F
:10848800FE6F030EFE6501D0A3D0FE51140D130E2E
:10849800F324D96E010EF420DA6E000EDF6EFE5161
:1084A800140D000EF324D96E010EF420DA6E000EBE
:1084B800DF6EFE51140D070EF324D96E010EF42061
:1084C800DA6EDE6ADE6ADE6ADD6AEFC286F0876B24
:1084D800886B896B88C089F087C088F086C087F070
:1084E800866BEEC28AF08B6B8C6B8D6B8BC08DF0BC
:1084F8008AC08CF08B6B8A6BEDC28EF08F6B906BA1
:10850800916B8EC091F0906B8F6B8E6B0201EC516A
:1085180000018E25926F000E8F21936F000E90211F
:10852800946F000E9121956F8A519225966F8B5109
:108538009321976F8C519421986F8D519521996F44
:10854800865196259A6F875197219B6F885198215C
:108558009C6F895199219D6FFE51140D0B0EF324C8
:10856800D96E010EF420DA6E9AC0DEFF9BC0DEFFE2
:108578009CC0DEFF9DC0DEFFDC0E606FFB0E616FEE
:10858800FEC062F0636BFE51140D0B0EF324D96E1E
:10859800010EF420DA6EDECF64F0DECF65F0DECFB8
:1085A80066F0DECF67F0FE51140D0B0EF324D96E82
:1085B800010EF420DA6EDECF68F0DECF69F0DECF90
:1085C8006AF0DECF6BF021EC5AF00001FE2B59D790
:1085D800000E0101996F000E0001FD6F000E0101F0
:1085E800AD6F000E986F000E836F000E826F020E43
:1085F8004F6E839012003850D96EDA6ADECFF6FFDC
:10860800DDCFF7FF0800F550250AD8A494D03850DC
:10861800D96EDA6ADE2A000EDD22000E01017B6FB8
:10862800000E7A6F7AC149F07BC14AF07C697D6996
:108638003850D96EDA6ADECFF6FFDDCFF7FF0800D3
:10864800F550780AD8B40CD03850D96EDA6ADECF33
:10865800F6FFDDCFF7FF0800F550580AD8A441D03F
:108668003850D96EDA6ADECFF6FFDDCFF7FF0800A3
:10867800F5CF44F03850D96EDA6ADE2A000EDD22D2
:108688003950D96EDA6ADF50DF2ADF2AD96EDA6A02
:10869800DECF3AF0DDCF3BF03AC03CF03BC03DF0D6
:1086A8003E6A3F6A406A416A426A436A37C025F0B7
:1086B8003CC026F03DC027F03EC028F03FC029F05E
:1086C80040C02AF041C02BF042C02CF043C02DF02E
:1086D80044C02EF098EC37F025C037F026C038F0AB
:1086E80012003850D96EDA6ADECFF6FFDDCFF7FF19
:1086F8000800F550250AD8A413D03850D96EDA6A84
:10870800DE2A000EDD22000E0E6E250E0D6E37C01D
:108718000FF0A8EC50F0000E386E010E376E120004
:108728003850D96EDA6ADE2A000EDD22000E386E65
:10873800000E376E12003850D96EDA6ADECFF6FFB7
:10874800DDCFF7FF0800F5500D6E0E6A37C00FF049
:10875800A8EC50F03850D96EDA6ADE2A000EDD2215
:10876800DAD70001FE51070D520EF324D96E010E1F
:10877800F420DA6EDF50CB6FCBC0CCF0CD6BCE6B74
:10878800CF6BCEC0CFF0CDC0CEF0CCC0CDF0CC6B8F
:10879800FE51070D510EF324D96E010EF420DA6E46
:1087A800DF50D06FD0C0D1F0D26BD36BD46BD3C0B5
:1087B800D4F0D2C0D3F0D1C0D2F0D16B040ED8908F
:1087C800D137D237D337D437E82EF9D7FE51070D32
:1087D800500EF324D96E010EF420DA6EDF50D56FF7
:1087E800D5C0D6F0D76BD86BD96B040ED890D637D6
:1087F800D737D837D937E82EF9D7D8C0D9F0D7C066
:10880800D8F0D6C0D7F0D66BD890D635DA6FD73532
:10881800DB6FD835DC6FD935DD6FD151DA25DE6FE6
:10882800D251DB21DF6FD351DC21E06FD451DD2140
:10883800E16FCC51DE25E36FCD51DF21E46FCE51DE
:10884800E021E56FCF51E121E66FFE51200D100EBA
:10885800F324A46F020EF420A56FE3C0A6F0E4C0D1
:10886800A7F0E5C0A8F0E6C0A9F0CDEC0FF0E26FE4
:10887800E251D8B411D0870E606FFC0E616FE3C06F
:1088880062F0E4C063F0E5C064F0E6C065F0E2C001
:1088980066F0676B21EC5AF00001FE51070D530E8C
:1088A800F324D96E010EF420DA6EE3C0DEFFE4C0D3
:1088B800DEFFE5C0DEFFE6C0DEFF000E0101976FB8
:1088C80083901200000E336E20EE04F02550D92656
:1088D8002650DA22DF50D8B49FD020EE2AF0255057
:1088E800D9262650DA22DECF36F0DECF37F0DECFBB
:1088F80038F0DECF39F02E0E25241B6E000E262010
:108908001C6E36C01DF037C01EF038C01FF039C0CD
:1089180020F0000E226E010E216E20EE01F025508F
:10892800D9262650DA22DF503BEC49F00009D8B4AA
:1089380003D0010E336E70D020EE04F02550D926F6
:108948002650DA22000EDF6E20EE16F02550D926CA
:108958002650DA2210EE1EF02550E1262650E2229B
:10896800E6CF2BF0E6CF2CF0E6CF2DF0E6CF2EF0B9
:108978002B50365C2F6E2C503758306E2D5038588F
:10898800316E2E503958326EDE502F5CDE50305822
:10899800DE503158DE503258D8B03ED020EE03F0C9
:1089A8002550D9262650DA22DF50276E2750346EFC
:1089B800356A355004E1020E345CD8A02DD020EE83
:1089C80016F02550D9262650DA22DE503626DE50FB
:1089D8003722DE503822DD5039222E0E25241B6E18
:1089E800000E26201C6E36C01DF037C01EF038C0A1
:1089F8001FF039C020F0000E226E010E216E20EE0D
:108A080001F02550D9262650DA22DF503BEC49F0F8
:108A18003406D8A03506CDD7335012000001965140
:108A28009511941104E1020E935DD8A010D020EEA8
:108A380012F09151D9269251DA22DE50935DDE5020
:108A48009459DE509559DE509659D8A002D0020E9E
:108A580030D0000E976F73D091C060F092C061F073
:108A680093C062F094C063F095C064F096C065F05E
:108A7800B4EC21F060C098F061C099F062C09AF03F
:108A880063C09BF00001985199119A119B11D8B4B9
:108A980066D0980599119A119B11D8B4D8D79829FE
:108AA8000AE1992908E19A2906E19B29D8A403D06B
:108AB800010E976F54D091C060F092C061F093C0DE
:108AC80062F094C063F095C064F096C065F0000E43
:108AD800666F000E676F000E686F000E696FC6EC58
:108AE8001AF0976F9751D8A43AD020EE0EF0915112
:108AF800D9269251DA22DE2807E1DE2805E1DE28B0
:108B080003E1DE28D8B413D020EE0EF09151D92617
:108B18009251DA22DE2A000EDE22DE22DE2220EE4A
:108B280005F09151D9269251DA22000EDB8098C0C7
:108B380093F099C094F09AC095F09BC096F020EEFF
:108B480012F09151D9269251DA22DE50935DDE500F
:108B58009459DE509559DE509659D8A07DD7975133
:108B680012000CC016F00DC017F010501110D8B438
:108B7800120016C0D9FF17C0DAFF0EC0DFFF105071
:108B88001624126E11501720136EFF0E1224D96E80
:108B9800FF0E1320DA6E0EC0DFFF115004E1030E42
:108BA800105CD8A0120020EE01F01650D9261750FC
:108BB800DA220EC0DFFF20EE02F01650D926175039
:108BC800DA220EC0DFFF10501624126E1150172043
:108BD800136EFE0E1224D96EFF0E1320DA6E0EC02D
:108BE800DFFF10501624126E11501720136EFD0E61
:108BF8001224D96EFF0E1320DA6E0EC0DFFF11505B
:108C080004E1070E105CD8A0120020EE03F0165005
:108C1800D9261750DA220EC0DFFF10501624126E24
:108C280011501720136EFC0E1224D96EFF0E13205C
:108C3800DA6E0EC0DFFF115004E1090E105CD8A0F7
:108C4800120016C012F017C013F0121E131E124A9B
:108C5800132A030E1214146E156A14501626155092
:108C680017221450105E1550115AFC0E1016FF0EE4
:108C780011160BD016C0D9FF17C0DAFF0EC0DFFFE0
:108C88001006D8A01106164A172A10501110D8B489
:108C98001200F0D7146815680C50D96EDA6ADE50E5
:108CA800DE10D8B486D00C50D96EDA6ADECF18F050
:108CB800DDCF19F002D0184A192A18C0F6FF19C0DA
:108CC800F7FF000EF86E0E0EF76403D00800F5509B
:108CD80005D0F6CFE9FFF7CFEAFFEF500E6E200E72
:108CE8000E6414D018C0F6FF19C0F7FF000EF86E16
:108CF8000E0EF76403D00800F55005D0F6CFE9FF53
:108D0800F7CFEAFFEF503A0AD8A4D5D718C0F6FF34
:108D180019C0F7FF000EF86E0E0EF76403D00800B6
:108D2800F55005D0F6CFE9FFF7CFEAFFEF503A0A42
:108D3800D8A444D00C50D96EDA6ADECF12F0DDCF59
:108D480013F012C0F6FF13C0F7FF000EF86E0E0EF8
:108D5800F76403D00800F55005D0F6CFE9FFF7CF48
:108D6800EAFFEF500E6ED00E0E24166E176AFF0E35
:108D78001722124A132A17501CE10A0E165CD8B0A3
:108D880018D01850121815E119501318D8A411D07A
:108D980016501710D8A40DD016C014F017C015F02F
:108DA800184A192A0C50D96EDA6A18C0DEFF19C0A1
:108DB800DDFF14C00CF015C00DF01200000E156E8A
:108DC800000E146EF6D72F6C696664617461302EDC
:108DD80062696E20002F6C696664617461312E626D
:108DE800696E20002F6C696664617461322E626955
:108DF8006E20002F6C696664617461332E62696E3F
:108E080020002F6C696664617461342E62696E207B
:108E1800002F6C696664617461352E62696E20008A
:108E28002F6C696664617461362E62696E20002F4A
:108E38006C696664617461372E62696E20002F6CFC
:108E4800696664617461382E62696E20002F6C69EE
:108E58006664617461392E62696E20002F6C6966E0
:108E680064617461612E62696E20002F6C696664AA
:108E7800617461622E62696E20002F6C696664619C
:108E88007461632E62696E20002F6C696664617478
:108E980061642E62696E20002F6C6966646174617A
:108EA800652E62696E20002F6C6966646174616664
:108EB8002E62696E20000000000000000000000023
:108EC800000000000000000000000000000000009A
:108ED800000000000000000000000000000000008A
:108EE800000000000000000000000000000000007A
:108EF8000000000E216E000E206E000E1A6E000E8D
:108F0800196E01D0132A010E1F6E1350D96EDA6A3A
:108F1800200EDE18D8B416D0F70E156EFF0E166E9A
:108F28001350D96EDA6ADF50176E186A1550172673
:108F380016501822185004E1050E175CD8A002D06C
:108F4800000E1F6E1FC01BF01C6A1B501C10D8B4EB
:108F580007D0D8D7000E1A6E010E196E132A2CD01E
:108F68001350D96EDA6ADF50156E166A1650000A69
:108F7800D8A422D015502B0AD8B4F0D7060AD8B4F2
:108F8800E9D71AD020C00CF021C00DF0000E0F6EEA
:108F98000A0E0E6EB9EC59F01350D96EDA6ADF502A
:108FA800156E15500C5E000E0D5A300E0C24206EF6
:108FB800000E0D20216ED2D7D00E156EFF0E166E44
:108FC8001350D96EDA6ADF50176E186A15501726D3
:108FD80016501822185006E10A0E175CD8B002D0B5
:108FE800010E01D0000E1D6E1E6A1D501E10D8A461
:108FF800C9D719501A10D8A40DD020C015F021C017
:1090080016F0151E161E154A162A15C013F016C09E
:1090180014F0120020C013F021C014F01200EBC1AC
:1090280088F07DD07FEC59F00001886F0101EB5189
:1090380000018819D8B486D0290E0001876F960ED2
:10904800866F7F0EE82EFED7862FFCD7872FFAD79C
:1090580079D0A7EC54F00001896F8951D8B472D047
:1090680089B1512A89B3510651500F0B516E000E28
:109078000C6EC00E17EC56F052EC59F0000E0C6E48
:10908800C00E17EC56F051500F0D340EF324106E2D
:109098000D0EF420116E3EEC52F0190E0001876F90
:1090A8005A0E866FB10EE82EFED7862FFCD7872F73
:1090B800FAD700D0000189A545D0000E0D6E000E2C
:1090C8000C6E51C00EF06DEC58F03A0E0001606F56
:1090D800FD0E616F51C062F0636B21EC5AF051C014
:1090E80088F0000E0C6E800E17EC56F052EC59F01A
:1090F800000E0C6E800E17EC56F051500F0D340E0A
:10910800F324106E0D0EF420116E3EEC52F0000E9A
:109118000C6EC00E17EC56F052EC59F013D001014A
:10912800A1510001866F876B8751000AD8A40AD025
:109138008651010AD8B476D7030AD8B473D7010A7E
:10914800D8B487D70001885112008380000E00012F
:10915800F66F000EF56F000EF36F0DEC54F016C0AD
:10916800F7F017C0F8F00001F8BF0BD0040EF85D57
:10917800D8A007D0000EF725F56FFC0EF821F66F82
:1091880004D0F7C0F5F0F8C0F6F0FE51070D530E05
:10919800F324D96E010EF420DA6E6CC1ECF06DC1C7
:1091A800EDF06EC1EEF0EB6B000EEB25EF6F010EEC
:1091B800EC21F06F000EED21F16F000EEE21F26F41
:1091C800DE50EF191CE1DE50F01919E1DE50F119FB
:1091D80016E1DE50F219D8A412D001C4FCF003C481
:1091E800FBF005C4FAF007C4F9F0F9C00FF0FAC0B3
:1091F80010F0FBC011F0FCC012F096EC55F08FB4E3
:1092080016D00001FE51200D100EF324A46F020E9B
:10921800F420A56F000EA66F040EA76F010EA96FAC
:10922800000EA86FF50EAA6F40EC0CF0F46F000169
:10923800F451D8B409D0C40E606FFD0E616FF4C04C
:1092480062F0636B21EC5AF0EDEC3BF0000E976F87
:1092580083905F0E0001606FFD0E616FCECF62F0EC
:10926800636BCDCF64F0656B21EC5AF01200246E6D
:109278002450D8A404D021502210D8A402D0040E1F
:10928800120053A002D0030E120053A402D0020E03
:10929800120050B608D0090ED8901D361E361F365B
:1092A8002036E82EF9D721042210D8A41DD01DC0DD
:1092B80015F01EC016F01FC017F020C018F0180EC9
:1092C80055EC57F00009D8A44FD01BC00EF01CC0B5
:1092D8000FF0FE0E106E0BEC55F00009D8B444D018
:1092E800000E226E000E3FD050C023F0060E23164B
:1092F800D8B409D021C015F022C016F0176A186A30
:10930800970E55EC57F01DC015F01EC016F01FC083
:1093180017F020C018F0190E55EC57F00009D8A422
:1093280023D01BC00EF01CC00FF0FC0E106E0BEC0F
:1093380055F00009D8B409D0020E1C262106D8A081
:10934800220621502210D8A4ECD7000E0E6E000E73
:109358000F6EFD0E106E0BEC55F00009D8A404D06A
:10936800000E226E010E216E69EC5AF02150221077
:10937800D8B402D0010E1200000E1200818E819C1A
:10938800CE0EF66E8D0EF76E000EF86E0DEE34F002
:1093980011EE2CF00900F5CFEEFFE550E150FAE1AF
:1093A800E250F8E1BA0EF66EB30EF76E000EF86EE4
:1093B80003EE80F010EE20F00900F5CFEEFFE55047
:1093C800E150FAE1560EF66EAD0EF76E000EF86E2D
:1093D80002EEB0F010EE46F00900F5CFEEFFE550D2
:1093E800E150FAE1F00EF66EB40EF76E000EF86E6C
:1093F8000900F5CFE7F10900F5CFE8F10900F5CF4D
:10940800E9F1F60EF66EB40EF76E000EF86E09006E
:10941800F5CF53F005EE00F018EE34F0EE6AE550A3
:10942800E150FCE1E250FAE104EE00F011EE00F048
:10943800EE6AE550E150FCE1E250FAE103EE00F09B
:10944800800EEE6AE806FDE102EE00F0B00EEE6A6C
:10945800E806FDE101EE00F0B20EEE6AE806FDE175
:109468000001FF6BFE6BFD6B00EE49F0090EEE6A22
:10947800E806FDE154905492000EF86E000150EF9A
:1094880008F08380000E0C6E040E0D6E000E0F6E39
:10949800F60E0E6E010E116E000E106EB5EC45F054
:1094A8009C0E0001606FFE0E616F21EC5AF0000EF9
:1094B8000001EC6F000EEB6F2E0E2CEC5AF08FB4FF
:1094C80016D00001FE51200D100EF324A46F020ED9
:1094D800F420A56F000EA66F040EA76F010EA96FEA
:1094E800000EA86FE80EAA6F40EC0CF0EA6F0001BE
:1094F800EA51D8B40AD0580E606FFF0E616FEAC007
:1095080062F0636B21EC5AF0120064EC5AF00C50D4
:109518000D10D8B427D0ED0E0C6E0D6A5FEC50F02C
:109528000001E76FED51100B0C6E000E0D6EE75148
:109538007BEC1FF00CC0EEF00DC0EFF0040E000144
:10954800EE19EF11D8B450EC58F0020E0001EE19E4
:10955800EF11D8B43BEC55F00001EE05EF11D8B48B
:10956800B5EC43F00001EB4BEC2BEC5104E1C80ED9
:10957800EB5DD8A0A1D7190E606FFF0E616F21ECCB
:109588005AF083901200000E0001F56F838075D0A9
:109598000DEC54F016C0F3F017C0F4F00001F4BF5E
:1095A80007D0040EF45DD8A003D0010EF56F03D0E8
:1095B800F8C0F6F0F76B8FB415D0FE51200D100EE1
:1095C800F324A46F020EF420A56F000EA66F040EFC
:1095D800A76F010EA96F000EA86FF60EAA6F40ECD8
:1095E8000CF0F86FF851D8B409D0C40E606FFD0EB6
:1095F800616FF8C062F0636B21EC5AF00001FE5114
:10960800070D530EF324D96E010EF420DA6E6CC1E7
:10961800ECF06DC1EDF06EC1EEF0EB6B000EEB25DA
:10962800EF6F010EEC21F06F000EED21F16F000ECF
:10963800EE21F26FDE50EF191CE1DE50F01919E14E
:10964800DE50F11916E1DE50F219D8A412D001C487
:10965800FCF003C4FBF005C4FAF007C4F9F0F9C044
:109668000FF0FAC010F0FBC011F0FCC012F096EC3D
:1096780055F0EDEC3BF0000E976F0001F551D8B4B2
:1096880087D783901200B7C045F0B8C046F0000EE7
:10969800486E000E476E09EC30F0C06FC051D8A478
:1096A80061D0000EBF6F000EBE6FB7C0D9FFB8C043
:1096B800DAFFDECF3AF0DDCF3BF020EE0EF0B75107
:1096C800D926B851DA22DECF3CF0DECF3DF0DECF2E
:1096D8003EF0DECF3FF087EC4EF00001C06FC05186
:1096E800D8A440D020EE12F0B751D926B851DA22CA
:1096F800DECFBBF0DDCFBCF0BBC0D9FFBCC0DAFF0A
:10970800E50EDE18D8B411D020EE12F0B751D926E4
:10971800B851DA22DECFBBF0DDCFBCF0BBC0D9FF39
:10972800BCC0DAFFDF50D8A40AD0BE4BBF2BB9515A
:10973800BE1909E1BA51BF19D8B414D004D0000E2B
:10974800BF6F000EBE6FB7C0A4F0B8C0A5F0000E82
:10975800A76F010EA66FE8EC27F00001C06FC0519B
:10976800D8B4A3D7040EC019D8A402D0070EC06F6E
:10977800C05112000F015969000E116F000E196FC8
:10978800000E216F8C948C928C90889A110E116E19
:109798003C0E106ECB0EE82EFED7102EFCD7112EE5
:1097A800FAD700F0110E116E3C0E106ECB0EE82E9B
:1097B800FED7102EFCD7112EFAD700F0020E116E2C
:1097C800A00E106E920EE82EFED7102EFCD7112E8A
:1097D800FAD700D0000E0C6E300E17EC56F02A0E99
:1097E800106E8E0EE82EFED7102EFCD7000E0C6ED3
:1097F800300E17EC56F0000E0C6E300E17EC56F0CB
:10980800000E0C6E390E17EC56F0000E0C6E140E8E
:1098180017EC56F0000E0C6E560E17EC56F0000EB4
:109828000C6E6D0E17EC56F0000E0C6E700E17ECE9
:1098380056F0000E0C6E0C0E17EC56F0000E0C6E67
:10984800060E17EC56F0000E0C6E010E17EC56F0D3
:10985800D00E106ECA0EE82EFED7102EFCD71200BE
:10986800B7C045F0B8C046F0000E486E000E476E0F
:1098780009EC30F0BC6FBC51D8B402D0BC51120016
:10988800B7C0D9FFB8C0DAFFDECF3AF0DDCF3BF082
:1098980020EE0EF0B751D926B851DA22DECF3CF0CF
:1098A800DECF3DF0DECF3EF0DECF3FF087EC4EF06E
:1098B8000001BC6FBC51D8A4E1D720EE12F0B7511B
:1098C800D926B851DA22DECFBAF0DDCFBBF0BAC064
:1098D800D9FFBBC0DAFFDF50B96FB951D8A403D0A4
:1098E800040EBC6FCBD720EE0BF0BA51D926BB5172
:1098F800DA22DFB618D0BAC00CF0BBC00DF020EEEB
:1099080014F0B751D926B851DA22DECF0EF0DDCFE8
:109918000FF0000E116E0B0E106E41EC54F00C504F
:109928000D10D8B4ABD7B7C0A4F0B8C0A5F0000EDE
:10993800A76F000EA66FE8EC27F00001BC6FBC51C2
:10994800D8A49CD79DD7C1C0B7F0C2C0B8F0000E4C
:10995800BA6F010EB96F47EC4BF0C36FC351D8A46F
:1099680058D0C1C0D9FFC2C0DAFFDECF3AF0DDCF90
:109978003BF020EE0EF0C151D926C251DA22DECFDB
:109988003CF0DECF3DF0DECF3EF0DECF3FF087EC9F
:109998004EF00001C36FC351D8A43BD020EE12F0A3
:1099A800C151D926C251DA22DECF0CF0DDCF0DF03D
:1099B800000E0F6E000E0E6E000E116E200E106E51
:1099C80069EC59F0000120EE12F0C151D926C251BC
:1099D800DA22DECF0CF0DDCF0DF020EE14F0C1510D
:1099E800D926C251DA22DECF0EF0DDCF0FF0000EFD
:1099F800116E0B0E106E76EC57F0C1C0D9FFC2C0C5
:109A0800DAFF10EE04F0DE50E126DD50E222010E0E
:109A1800E76EC3511200236E2350D8A404D02150FE
:109A28002210D8A402D0040E120053A002D0030EB4
:109A3800120050B608D0090ED8901D361E361F36B3
:109A48002036E82EF9D7225008E1020E215CD8B062
:109A580004D0000E256E110E03D0000E256E120ED6
:109A6800246E24C026F01DC015F01EC016F01FC0BD
:109A780017F020C018F0265055EC57F00009D8A46C
:109A880025D01BC00CF01CC00DF0020E0F6E000E8E
:109A98000E6ED8EC53F00009D8B409D0020E1C267B
:109AA8002106D8A0220621502210D8A4EAD7120EE7
:109AB8002618D8A40BD0000E156E000E166E000ED8
:109AC800176E000E186E0C0E55EC57F069EC5AF034
:109AD80021502210D8B402D0010E1200000E12003C
:109AE8001A0E0E24106E000E0F20116E010E102497
:109AF800D96E000E1120DA6EDF50126E1250146EFD
:109B0800136A1A0E0E24D96E000E0F20DA6EDF507B
:109B1800156E15501312000E141213C01AF014C04B
:109B28001BF01C6A1D6A0CC0D9FF0DC0DAFF030EBA
:109B3800DE18D8A42ED0140E0E24106E000E0F209E
:109B4800116E010E1024D96E000E1120DA6EDF504E
:109B5800126E1250146E136A140E0E24D96E000E73
:109B68000F20DA6EDF50156E15501310166E145054
:109B7800176E186A196A17C019F016C018F0176A14
:109B8800166A16501A1217501B1218501C12195028
:109B98001D121AC00CF01BC00DF01CC00EF01DC029
:109BA8000FF01200020E1A5E000E1B5A1C5A1D5AA4
:109BB80020EE12F01850D9261950DA22FE0EDE24B3
:109BC8001E6EFF0EDE201F6EFF0EDE20206EFF0EC3
:109BD800DE20216E1E501A5C1F501B5820501C5846
:109BE80021501D58D8A009D0000E186E000E196E0D
:109BF800000E1A6E000E1B6E120020EE26F0185092
:109C0800D9261950DA22DECF1EF0DECF1FF0DECFC4
:109C180020F0DECF21F020EE02F01850D92619509E
:109C2800DA22DF50226E22500C6E0D6A0E6A0F6A1D
:109C38001AC010F01BC011F01CC012F01DC013F0A8
:109C4800C1EC55F01E500C24186E1F500D20196ED3
:109C580020500E201A6E21500F201B6E1200DAC001
:109C6800E0F0DBC0E1F0E00E0C6E4EEC46F00CC00C
:109C7800E2F00DC0E3F00001E3AF02D00B0E1200DA
:109C8800D890E235D96EE335DA6E8C0ED926010EFE
:109C9800DA22DECFDEF0DDCFDFF0DE51DF11D8B41F
:109CA80006D0DEC0D9FFDFC0DAFF000EDF6ED85164
:109CB800D911D8B406D0D8C0D9FFD9C0DAFF000E60
:109CC800DF6ED890E235D96EE335DA6E8C0ED92680
:109CD800010EDA22D8C0DEFFD9C0DDFFD851D91174
:109CE800D8B403D0DC05D8B402D0000E1200D80EC8
:109CF800456E466ADA0E476E000E486EB8EC00F004
:109D0800DD6FDD511200000E446E20EE2AF03A504D
:109D1800D9263B50DA223C50DE180AE13D50DE18C5
:109D280007E13E50DE1804E13F50DE18D8B43CD0BD
:109D38003AC025F03BC026F066EC44F0446E44502F
:109D4800D8A432D02E0E3A241B6E000E3B201C6E77
:109D58003CC01DF03DC01EF03EC01FF03FC020F0CB
:109D6800000E226E010E216E20EE01F03A50D92627
:109D78003B50DA22DF500FEC4DF00009D8B406D082
:109D88003C683D683E683F68010E446E20EE2AF04C
:109D98003A50D9263B50DA223CC0DEFF3DC0DEFFF8
:109DA8003EC0DEFF3FC0DEFF44501200000E866E4C
:109DB800000E846E8B688968000E0101A66F000E84
:109DC800AB6F000E936F000E926F83928394000E18
:109DD800AD6F000EAC6F200EAF6F400EAE6F000E71
:109DE800916F000E906F0AD0000E9025D96E040E68
:109DF8009121DA6E000EDF6E904B912B91BFF4D754
:109E08009105D8A0F1D7000E916F000E906F0AD07F
:109E1800340E9025D96E0B0E9121DA6E000EDF6E8E
:109E2800904B912B91BFF4D79105D8A0F1D70F0192
:109E38001769D6501F0B4009D66ED6980F0ED6124A
:109E4800D5980F0ED5120E01C29BD58E12000CC0EC
:109E580014F00DC015F00EC016F00FC017F0100664
:109E6800D8A0110610280FE11128D8A40CD0000E94
:109E78000D6E000E0C6E1200144A152A164A172A87
:109E88001006D8A0110614C0F6FF15C0F7FF080089
:109E9800F5500009D8B418D016C0D9FF17C0DAFF9A
:109EA800DF50D8B411D010501110D8B40DD016C04E
:109EB800D9FF17C0DAFF14C0F6FF15C0F7FFDE5050
:109EC8000900F518D8B4D8D714C0F6FF15C0F7FFA5
:109ED8000800F5CF12F016C0D9FF17C0DAFFDF501F
:109EE800136E1350125C0C6E0D6AD8A00D0612008A
:109EF80003D00C4A0D2A0E2A0E50D96EDA6ADF50AA
:109F08000F6E0CC0F6FF0DC0F7FF000EF86E0E0EB8
:109F1800F76403D00800F55005D0F6CFE9FFF7CF76
:109F2800EAFFEF500F18D8A414D00CC0F6FF0DC0EC
:109F3800F7FF000EF86E0E0EF76403D00800F55018
:109F480005D0F6CFE9FFF7CFEAFFEF500009D8A414
:109F5800D0D70CC0F6FF0DC0F7FF000EF86E0E0E3E
:109F6800F76403D00800F55005D0F6CFE9FFF7CF26
:109F7800EAFFEF500F6E0E50D96EDA6ADF50106E9E
:109F880010500F5C0C6E0D6AD8A00D061200FE5121
:109F9800140D070EF324D96E010EF420DA6E000EAC
:109FA800DE24CB6F010EDE20CC6F000EDE20CD6FDD
:109FB800000EDE20CE6FFE51140D070EF324D96E6D
:109FC800010EF420DA6ECBC0DEFFCCC0DEFFCDC0C0
:109FD800DEFFCEC0DEFFFE51140D070EF324D96E4E
:109FE800010EF420DA6EDECFCFF0DDCFD0F0FE51D7
:109FF800200D100EF324A46F020EF420A56FCFC01D
:10A00800A6F0D0C0A7F0A86BA96BCDEC0FF0D16F6C
:10A01800D151D8B403D0010E4F6E1200000E4F6E0E
:10A0280012000DC013F00EC014F013501410D8B461
:10A038003ED013C0D9FF14C0DAFFDE50DE10D8B40A
:10A0480036D013C0D9FF14C0DAFFDECF0FF0DDCF52
:10A0580010F00FC0D9FF10C0DAFFDF50D8B427D0F6
:10A0680020EE02F01350D9261450DA2213C0E1FF73
:10A0780014C0E2FF00EE06F0E650E926E550EA22B9
:10A08800DE50EE1814E1DE50EE18D8A410D013C03C
:10A09800D9FF14C0DAFF10EE01F0DE50E126DD50E2
:10A0A800E222E75049EC5AF00F6E0FA002D0090ED9
:10A0B8001200000E120025EE04F0DE50DE10D8B4B7
:10A0C800FAD700C514F001C515F0060E1424D96E90
:10A0D800050E1520DA6EDF50126E060E1424D96EA6
:10A0E800070E1520DA6EDF50136E144A152AFF0E7C
:10A0F8000E6E010E0F6E14C010F015C011F00E5048
:10A1080010160F50111610C000F511C001F5F29E7F
:10A1180025EE04F0DE06000EDD5AF28E0CC0D9FFE3
:10A128000DC0DAFF13C0DFFF25EE04F0010EDBBE21
:10A1380006D0000EDE5C020EDE58D8B003D08EB812
:10A1480083B28982125012000F50D8B403D00F5036
:10A15800D8A404D00D5016EC5AF012000F50D96E46
:10A16800DA6A040ED926DE50DE10D8B414D00F50A7
:10A17800D96EDA6A040ED9260F50E16EE26A020E31
:10A18800E126DE50E65CE650800A146EDE50800A56
:10A198001458D8B012000F50D96EDA6A020ED926B8
:10A1A800DECF10F0DDCF11F00F50D96EDA6ADECFB6
:10A1B80012F0DDCF13F010501224D96E1150132075
:10A1C800DA6E0DC0DFFF0F50D96EDA6A020ED9269B
:10A1D800DE2A000EDD221200000E4E6E000E4D6EBD
:10A1E800000E0101816F000E806F020E976F839041
:10A1F800000E966F000E956F000E0001FE6F030EA5
:10A20800FE6501D02CD0FE51070D520EF324D96EF5
:10A21800010EF420DA6E000EDF6EFE51070D510EAE
:10A22800F324D96E010EF420DA6E000EDF6EFE51B3
:10A23800070D500EF324D96E010EF420DA6E000ECD
:10A24800DF6EFE51070D530EF324D96E010EF42074
:10A25800DA6EDE6ADE6ADE6ADD6AFE2BD0D7000EB1
:10A26800FE6F120049A008D01CC015F01DC016F0E2
:10A278001BC017F0BFEC58F01FBE05D01EC023F05E
:10A288001FC024F004D0000E246E000E236E000EB2
:10A29800226E000E216E0AD0000E0E6E200E0D6E7C
:10A2A8001BC00FF0A8EC50F0214A222A2350215C51
:10A2B8002250800A206E2450800A2058D8A0ECD75B
:10A2C80049B008D01CC015F01DC016F01BC017F00F
:10A2D800BFEC58F01CC012F01DC013F012EC57F080
:10A2E800235012241B6E245013201C6E12008380EE
:10A2F800000E0001B76F000EB86F000EB96F000EA8
:10A30800BA6FFE51200D100EF3248C6F020EF4204C
:10A318008D6F340E8E6F0B0E8F6F010E916F000EC6
:10A32800906FBB0E926F936BD2EC12F05250FD0BF4
:10A33800526E010E0101A66FBBC086F0BCC087F04B
:10A34800B0EC38F086C0B5F087C0B6F0000E010159
:10A35800A66F0001B551B725B76FB651B821B86FD0
:10A36800000EB921B96F000EBA21BA6F000E0101B3
:10A37800976F83901200000E146E000E156E000E7B
:10A38800166E000E176E1050111012101310D8B45C
:10A398002AD0010E186E06D0D89010361136123613
:10A3A8001336182A13AEF8D7D89014361536163641
:10A3B800173610500C5C11500D5812500E5813508F
:10A3C8000F58D8A009D010500C5E11500D5A1250D9
:10A3D8000E5A13500F5A1480D89013321232113279
:10A3E8001032182EE1D714C00CF015C00DF016C0AD
:10A3F8000EF017C00FF01200146E0C0E1418D8B41B
:10A4080009D069EC5AF0EDEC59F00009D8A402D053
:10A41800FF0E12001450400940EC5AF0115040EC65
:10A428005AF0105040EC5AF00F5040EC5AF00E50D1
:10A4380040EC5AF0010E136E1450D8A402D0950EB9
:10A44800136E080E1418D8A402D0870E136E13507A
:10A4580040EC5AF00C0E1418D8B458EC5AF00A0E06
:10A46800136E58EC5AF0126E12AE02D0132EF9D7B2
:10A4780012501200150E126EC60EE82EFED7122EBE
:10A48800FCD700D020D0150E126EC60EE82EFED7CF
:10A49800122EFCD700D0010E0C6E10C0F6FF11C0B2
:10A4A800F7FF000EF86E0E0EF76403D00800F550A3
:10A4B80005D0F6CFE9FFF7CFEAFFEF5017EC56F0DB
:10A4C800104A112AD7D710C0F6FF11C0F7FF000EA7
:10A4D800F86E0E0EF76403D00800F55005D0F6CFDD
:10A4E800E9FFF7CFEAFFEF500009D8B41200CBD745
:10A4F80032EC58F0CC0EFCEC59F0660EFCEC59F03E
:10A50800CCEC59F0166E1650D8A409D0000E106E77
:10A51800000E116E000E126E000E136E1200000E69
:10A52800156E000E146E1450160FD96EDA6ACCEC44
:10A5380059F0DF6E144A152A15BEF5D7155004E1F7
:10A54800040E145CD8A0EFD719501810171004E1A6
:10A55800060E165CD8A0DAD716C010F017C011F096
:10A5680018C012F019C013F012005250FD0B526EB1
:10A57800340E0C6E0B0E0D6EF10E0E6E020E0F6E7B
:10A58800000E116E050E106ECEEC56F0390E0C6EE4
:10A598000B0E0D6ED10E0E6E020E0F6E000E116EAA
:10A5A800130E106ECEEC56F052500209526E4C0E3D
:10A5B8000C6E0B0E0D6EE40E0E6E020E0F6E000E7C
:10A5C800116E0D0E106ECEEC56F0000E0001876F66
:10A5D800250E866FB0EC38F05250FD0B526E83900A
:10A5E800120011D0030E0DD0050E0E6E000E0101E3
:10A5F800836F000E826F2FD0010E03D0020E01D0A0
:10A60800000E0E6E28D082C10CF083C10DF00D50E3
:10A61800000AD8B40AD0020AD8B40FD00F0AD8B4A6
:10A6280011D02A0AD8B413D0EBD70C500A0AD8B4E0
:10A63800D9D71E0AD8B4D8D7E3D70C50BC0AD8B497
:10A64800DDD7DED70C50AC0AD8B4D6D7D9D70C5042
:10A658000F0AD8A4D5D70E501200000E0001FE6FC5
:10A66800030EFE6501D02CD0FE51070D520EF324C7
:10A67800D96E010EF420DA6E000EDF6EFE51070D62
:10A68800510EF324D96E010EF420DA6E000EDF6E3F
:10A69800FE51070D500EF324D96E010EF420DA6E28
:10A6A800000EDF6EFE51070D530EF324D96E010E16
:10A6B800F420DA6EDE6ADE6ADE6ADD6AFE2BD0D747
:10A6C800000EFE6F8390000E0101976F1200BAEC26
:10A6D80040F0CBC0E8F0CCC0E9F0E851E911D8B4BB
:10A6E80005D0E8C0E2F0E9C0E3F012008FB415D05D
:10A6F800FE51200D100EF324A46F020EF420A56F56
:10A70800000EA66F040EA76F010EA96F000EA86FAA
:10A71800E60EAA6F40EC0CF0EA6FEA51D8B404D008
:10A72800EAC0E2F0E36B1200CBEC4FF0010E01013E
:10A738009A6F000E0001E36F000EE26F1200000E28
:10A748000D6E000E0C6E0001FE51140D070EF32461
:10A75800D96E010EF420DA6EDE6ADE6ADE6ADD6A20
:10A76800FE51140D130EF324D96E010EF420DA6E87
:10A77800000EDF6EFE51140D0F0EF324D96E010E7C
:10A78800F420DA6EDE6ADE6ADE6ADD6A0C4A0D2AB9
:10A798000DBED9D70D5004E1040E0C5CD8A0D3D758
:10A7A8008390000E4F6E1200070E116ED00E106EC1
:10A7B80010D058EC5AF0126E1228D8A40ED0E40E1D
:10A7C80000D000D0E82EFCD700D000D01006D8A0CA
:10A7D800110610501110D8A4ECD7FE0E1218D8B4D8
:10A7E80002D0000E120058EC5AF00CC0D9FF0DC070
:10A7F800DAFFDF6E0C4A0D2A0E06D8A00F060E509F
:10A808000F10D8A4F0D758EC5AF058EC5AF0010EB3
:10A818001200000E1B6E000E1A6E000E196E23D069
:10A8280064EC5AF00C500D10D8B412D0190E0C6EFE
:10A838000D6A5FEC50F0186E000E0101AB25D96E61
:10A84800DA6A040EDA2218C0DFFFAB2B1A4A1B2A79
:10A8580019AA07D0000E1A24166E040E1B20176EB4
:10A8680012008EAC05D01BBEDBD71B04D8A0D8D7EE
:10A878001AC016F01BC017F012000CC014F00DC05F
:10A8880015F00EC016F00FC017F0000E196E000E6E
:10A89800186E1006D8A01106102803E11128D8B4A4
:10A8A8001AD014C0D9FF15C0DAFF144A152ADF5090
:10A8B800126E16C0D9FF17C0DAFF164A172ADF50E2
:10A8C800136E1350125C186E196AD8A01906185026
:10A8D8001910D8B4DED718C00CF019C00DF012004A
:10A8E8001050111012101310D8B424D0010E146E89
:10A8F80006D0D8901036113612361336142A13AEF5
:10A90800F8D710500C5C11500D5812500E581350B7
:10A918000F58D8A008D010500C5E11500D5A125084
:10A928000E5A13500F5AD890133212321132103275
:10A93800142EE7D70CC00CF00DC00DF00EC00EF0B1
:10A948000FC00FF01200010E0E6E000E0F6E8886FB
:10A9580087828784050EE82EFED700F08794050EBF
:10A96800E82EFED700F0000E0D6E000E0C6E8DA6C0
:10A9780003D00F500E100F6E0E500E240E6E8790DF
:10A98800050EE82EFED700F08780050EE82EFED7CC
:10A9980000F087900C4A0D2A0DBEE9D70D5004E14E
:10A9A800030E0C5CD8A0E3D70F5012000001876F8C
:10A9B800F50E0001886FFA0E896F000E866F0CD0B5
:10A9C80088C0F6FF89C0F7FF884B892B0800F5502F
:10A9D8000009D8A4F5D7862B87518619D8B409D091
:10A9E80088C0F6FF89C0F7FF0800F5500009D8A411
:10A9F800E7D7AA0E606FFE0E616F87C062F0636BC7
:10AA080088C064F089C065F021EC5AF0120096EC19
:10AA180057F00009D8A402D0000E1200105040ECE4
:10AA28005AF0FD0E1018D8B420D0020E126E000E87
:10AA3800116E0EC0D9FF0FC0DAFFDF5040EC5AF09C
:10AA48000E4A0F2A1106D8A0120611501210D8A4C7
:10AA5800F0D758EC5AF058EC5AF058EC5AF0136EFC
:10AA680013501F0B050AD8A4D7D7010E12008380F4
:10AA780052500209526E2BEE34F095C1DFFF000EE2
:10AA8800E8CF35FB0D0EE8CF36FB000EE8CF37FBDD
:10AA98008FA403D0600EE8CF37FB8FA407D036CB46
:10AAA8008CF0200E00018C138CC036FB000E0001C8
:10AAB800876F040E866FB0EC38F05250FD0B526E63
:10AAC800000E0101956F8390120012C017F013C099
:10AAD80018F012D01506D8A01606142A1404D96E38
:10AAE800DA6A17C0E1FF18C0E2FF174A182ADFCF59
:10AAF800E7FFE750D8B40DD015501610D8B409D0D8
:10AB0800E9D717C0D9FF18C0DAFF000EDF6E174A61
:10AB1800182A1506D8A016061528F3E11628D8B461
:10AB28001200EFD70FC013F010C014F011C015F0C9
:10AB380012C016F032EC58F0CC0EFCEC59F0990E1D
:10AB4800FCEC59F00C0EFCEC59F0000E186E000EDF
:10AB5800176E1750130FD96EDA6ADF50FCEC59F0F4
:10AB6800174A182A18BEF5D7185004E1040E175CC6
:10AB7800D8A0EFD732EC58F01200000E146E000E79
:10AB8800156E000E166E000E176E0CA008D0105031
:10AB98001426115015221250162213501722D8903D
:10ABA8001036113612361336D8900F320E320D3257
:10ABB8000C320C500D100E100F10D8A4E6D714C08C
:10ABC8000CF015C00DF016C00EF017C00FF01200F3
:10ABD80015D00DC0F6FF0EC0F7FF000EF86E0E0E72
:10ABE800F76403D00800F55005D0F6CFE9FFF7CF9A
:10ABF800EAFFEF502CEC5AF00D4A0E2A0DC0F6FF72
:10AC08000EC0F7FF000EF86E0E0EF76403D00800B2
:10AC1800F55005D0F6CFE9FFF7CFEAFFEF5000096E
:10AC2800D8B41200D6D70D6E8792050EE82EFED73F
:10AC380000F00CB002D0879401D08784000E0F6E0C
:10AC4800010E0E6E0DAE02D0838A01D0839A0D508C
:10AC58000D240D6E8790878087900E4A0F2A0FBEAD
:10AC6800F1D70F5004E1090E0E5CD8A0EBD787820C
:10AC7800120046C074F047C075F0000E0101796FEC
:10AC8800000E786F0DD045C037F0740E386E48C08E
:10AC980039F0FFEC42F0375001017827385079231A
:10ACA80074C0F6FF75C0F7FF0800F5500009D8A476
:10ACB800EAD778C145F079C146F012009F0E146EAC
:10ACC800FF0E156E12C016F013C017F0145016269A
:10ACD80015501722175006E11A0E165CD8B002D08C
:10ACE800010E01D0000E186E196A18501910D8B448
:10ACF80005D05F0E1214126E136A120012C012F001
:10AD080013C013F0120002D00C4A0D2A0CC0F6FF33
:10AD18000DC0F7FF0800F5500009D8B40FD00CC0DB
:10AD2800F6FF0DC0F7FF0800F550106E116A0E50BF
:10AD38001018EAE10F501118D8A4E6D70CC0F6FF96
:10AD48000DC0F7FF0800F5500C6E0D6A1200800068
:10AD58004C4142454C3100000002800000000000D8
:10AD6800000E000068706469736B2E6366670001EB
:10AD7800091220010001001700002D119420D00FA6
:10AD8800000100000000000000000000099F028090
:10AD98000102E8050EC015F00FC016F00CC013F044
:10ADA8000DC014F010D015C0D9FF16C0DAFFDF505F
:10ADB800126E154A162A13C0D9FF14C0DAFF12C042
:10ADC800DFFF134A142A1006D8A011061028EBE159
:10ADD8001128D8B41200E7D77A0E7E6F76C07FF0BC
:10ADE80077C080F0000E826F000E816F000E846FB6
:10ADF800000E836F7F0E456E78C046F079C047F02D
:10AE08007E0E486E3DEC56F0000181517625D96ED4
:10AE180082517721DA6E000EDF6E120012C014F034
:10AE280013C015F002D0124A132A12C0F6FF13C03D
:10AE3800F7FF000EF86E0E0EF76403D00800F55009
:10AE480005D0F6CFE9FFF7CFEAFFEF500009D8A405
:10AE5800EAD71450125C126E15501358136E120074
:10AE680020EE1AF00C50D9260D50DA220EC0DFFF62
:10AE780020EE1BF00C50D9260D50DA220FC0DFFF50
:10AE880020EE14F00C50D9260D50DA2210C0DFFF46
:10AE980020EE15F00C50D9260D50DA221150DF6E35
:10AEA8001200196E19AE12D0199E000E0E6E000E09
:10AEB8000F6E000E106E000E116E370E00EC52F081
:10AEC8001A6E010E1A6402D01A50120015C00EF044
:10AED80016C00FF017C010F018C011F0195000EC90
:10AEE80052F012000CC012F00DC013F00EC014F096
:10AEF8000FC015F00ED014C0D9FF15C0DAFF12C06C
:10AF0800E1FF13C0E2FFDFCFE7FF144A152A124A18
:10AF1800132A1006D8A011061028EDE11128D8B47C
:10AF28001200E9D7130E0D6E880E0C6E0FD058EC78
:10AF38005AF0FF0AD8B40ED0E40E00D000D0E82EA4
:10AF4800FCD700D000D00C06D8A00D060C500D1070
:10AF5800D8A4EDD70C500D10D8B402D0010E1200B1
:10AF6800000E1200340E0C6E0B0E0D6E000E0F6EDE
:10AF7800000E0E6E010E116E000E106EB5EC45F04F
:10AF8800010EE8CF34FB52500209526E000E000148
:10AF9800876F010E866FB0EC38F05250FD0B526E81
:10AFA80012000C6E0C50D8B40ED06EEC5AF0200E75
:10AFB800E82EFED771EC5AF0CC0E00D0E82EFDD763
:10AFC80000D000D012006EEC5AF0C00E00D0E82E6F
:10AFD800FDD771EC5AF0350EE82EFED700F01200BE
:10AFE80073C047F074C048F0DBEC3AF0756F7551E8
:10AFF800D8A413D073C00DF074C00EF015EC50F047
:10B008000001756F7551D8A408D073C0D9FF74C0FA
:10B01800DAFF000EDE6E000EDD6E75511200010EB5
:10B02800126E200E0C180D10D8B414D0F70E0E6E38
:10B03800FF0E0F6E0CC010F00DC011F00E50102650
:10B048000F501122115004E1050E105CD8A002D057
:10B05800000E126E12C00CF00D6A12006EEC5AF05F
:10B068000A0E0D6EF80EE82EFED70D2EFCD700D076
:10B0780071EC5AF0E00E00D0E82EFDD737EC5AF00C
:10B088000E6E090E0D6E840EE82EFED70D2EFCD71F
:10B0980071EC5AF00E501200340E0C6E0B0E0D6E41
:10B0A800000E0F6E000E0E6E010E116E000E106E69
:10B0B800B5EC45F02BEE34F097C1DFFF000E000130
:10B0C800876F010E866FB0EC38F0000E0101976FA4
:10B0D8001200000EF2BE010E0F6E0D50030B7F6EB4
:10B0E8000CC07EFF0EC080FF3F0E81168184F29E49
:10B0F800550E826EAA0E826E818281B2FED781942D
:10B108000FB002D0F29E01D0F28E120060900F0EA6
:10B118000F01596F070E396F070E356F4F0E936E7B
:10B12800000E8A6E8A888A828A82000E8F6E130EBB
:10B138000E01B76F0F0EFA6F100EFC6F140EB86F7A
:10B1480012009F869E84090E0E01FD6F9F98890E3E
:10B158009B6E000E9C6E9E989D8E9D889D9AC599AB
:10B16800F28AF28E9E909D9C9E9A9E8A01019B91E6
:10B17800000E9C6F1200000E1A6E000E196E09D098
:10B1880018C00DF00E6A17C00FF0A8EC50F0194A5D
:10B198001A2A19501524D96E1A501620DA6EDF5063
:10B1A800186E1850D8B41200EBD79F0E0E6EFF0E13
:10B1B8000F6E200E0C10106E000E0D10116E0E503A
:10B1C80010260F501122115006E11A0E105CD8B04B
:10B1D80002D0010E01D0000E0C6E0D6A12009F0EF7
:10B1E8000E6EFF0E0F6E0CC010F00DC011F00E5059
:10B1F80010260F501122115006E11A0E105CD8B01B
:10B2080002D0010E01D0000E0C6E0D6A1200BF0EA6
:10B218000E6EFF0E0F6E0CC010F00DC011F00E5028
:10B2280010260F501122115006E11A0E105CD8B0EA
:10B2380002D0010E01D0000E0C6E0D6A1200D00E65
:10B248000E6EFF0E0F6E0CC010F00DC011F00E50F8
:10B2580010260F501122115006E10A0E105CD8B0CA
:10B2680002D0010E01D0000E0C6E0D6A12000C6E99
:10B278000C50D8B40AD0000E966E4F0E936E2A0E5C
:10B28800966E400E956E968A1200000E966E100EFF
:10B29800966E2A0E966EF00E936EF3D7000E116E10
:10B2A800110E106E09D0050EE82EFED700F0010E23
:10B2B8000C6E200E17EC56F01006D8A011061028B8
:10B2C800F2E11128D8B41200EED70CC012F00DC06C
:10B2D80013F008D012C0D9FF13C0DAFF0EC0DFFF89
:10B2E800124A132A1006D8A011061028F3E11128D3
:10B2F800D8B41200EFD79150070B0C6E888A8DAA2C
:10B3080003D00C50080F0C6E020E0101A119D8A42D
:10B3180004D00C50FF0A0F0B0C6E0C501200000EDC
:10B32800E8CF00F5000EE8CF01F5000EE8CF02F5F2
:10B33800000EE8CF03F5000EE8CF04F5000EE8CFC5
:10B3480005F512006EEC5AF0200EE82EFED771ECCF
:10B358005AF0300EE82EFED737EC5AF00D6EB00ECC
:10B3680000D0E82EFDD70D5012000C500E02F3CF7E
:10B3780010F0F4CF11F00C500F02F35011260D50BD
:10B388000E02F350112610C00CF011C00DF012007F
:10B39800000E0E6E000E0F6ED8900E32A6EC59F00D
:10B3A8000009D8A40E8E0F2A070E0F64F5D70E5089
:10B3B80012004D5946494C453132333400010000E2
:10B3C800000100002000131012000000010000001E
:10B3D800000076EC5AF058EC5AF096EC57F0000959
:10B3E800D8B402D0010E120069EC5AF0000E120017
:10B3F8000D6E000E0E6E0D50010BD5EC57F0D89067
:10B408000D320E2A070E0E64F6D712000D50030BEC
:10B418007F6E0CC07EFF3F0E8116818000F000F029
:10B42800805012000C6E03D07AEC5AF004000E0122
:10B43800CDA9FAD70CC09AFF1200620E486E60C000
:10B4480019F061C01AF0480E1B6EE2EC23F01200EE
:10B458000C6E03D07AEC5AF004000E01CDA9FAD78D
:10B468000CC09AFF120088888DA802D0010E01D066
:10B47800000E0C6E0C5012000C6E0CC092FF95B0B2
:10B48800FED795A0FED7925012000C6E0C50D8B47F
:10B4980002D0010E1200535012008380010E4F6E2D
:10B4A800000E4F6E83901200926895B0FED795A05B
:10B4B800FED7925012008390000E0101976F120080
:10B4C80004C50CF005C50DF0120074EC5AF058ECE8
:10B4D8005AF012008398889812008398888812007E
:0BB4E8008F8012008F901200340BE7E1
:03B4F40012000142
:10FAF400004F4B004449534B5F455252004E4F5404
:10FB04005F5245414459004E4F5F46494C45004EB3
:10FB14004F545F4F50454E4544004E4F545F454E41
:10FB240041424C4544004E4F5F46494C455F535952
:10FB34005354454D00000D0A2025325820253258D3
:10FB44002025327320253273202532732025327309
:10FB540020253273202532732025327320253273F9
:10FB640020253473202534732025347320253473E1
:10FB740020253473202534732025347320253473D1
:10FB840020000D0A48504469736B204D6B2049498D
:10FB9400202831384634364B34302920257320252B
:10FBA40073202573205374617274696E672E2E2E30
:10FBB4000D0A000D0A547269656420746F20746123
:10FBC4006C6B207768696C7374206E6F7420616449
:10FBD40064726573736564000D0A4D61782056651F
:10FBE40063746F72206469736B20256420256C64D0
:10FBF4002028256C582920000D0A2530325825303C
:10FC040032582053533830783A5374617475735BA7
:10FC140025645D20255820000D0A44736B73656CC0
:10FC24002069732025642C206E756D6265722069CD
:10FC3400732025642000466F756E6420616E205227
:10FC440054432066696C652061742025580D0A00B0
:10FC54004C6F6F6B696E6720666F7220616E205205
:10FC640054432066696C650D0A0046696E644669F2
:10FC74006C65206661696C65642073656172636894
:10FC84000D0A000D0A5365656B20746F20256C64A2
:10FC9400206661696C6564202564000D0A446973FB
:10FCA4006B2073656C656374206E756D626572207C
:10FCB4002564005365656B696E6720746F207365F6
:10FCC40063746F722025580D0A0046696E64466994
:10FCD4006C65206661696C656420726561640D0AF7
:10FCE400000D0A4F70656E696E67206578697374DC
:10FCF400696E6720257320000D0A476F7420256CF8
:10FD04007520202D20726573657474696E67000D0B
:10FD14000A57616974696E6720666F722063617245
:10FD24006420000D0A46696C6520257320697320E0
:10FD34006F70656E20000D0A57726F7465206469D8
:10FD4400736B6E6F3A202564000D0A4F70656E69FF
:10FD54006E67206E657720257320000D0A253032EA
:10FD64005825303258204578697420004E6F74202D
:10FD740061204C4946206469736B0D0A000D0A54D6
:10FD84005844415441206C656E20256420000D0ABE
:10FD940046696C6520255820697320257320000D61
:10FDA4000A4469736B202558206973202573200049
:10FDB4000D0A4873742062797465733220256400D7
:10FDC4000D0A5772697465206661696C20256400A8
:10FDD4000D0A52656164696E67205254430D0A002E
:10FDE4000D0A416D69676F2039313231440D0A00C3
:10FDF4000D0A53532F38302039313232440D0A0062
:10FE04000D0A44736B73656C2069732025642000AC
:10FE14000D0A52656164202564206279746573005B
:10FE2400566563746F722069732025580D0A002289
:10FE34002A2B2C3A3B3C3D3E3F5B5D7C7F000D0A08
:10FE44004F70656E696E672025732020000D0A448B
:10FE54006562756720697320256420000D0A50725D
:10FE64006F746F20697320256420000D0A52656148
:10FE74006420636F6E66696720000D0A46696C65CD
:10FE84006E616D6520257320002041544E206173FE
:10FE940073657274656420000D0A466F726D617437
:10FEA40074696E67200072633D25752046525F2594
:10FEB400730D0A000D0A4E6F20636172642025647D
:10FEC400002F6C6966646174612E62696E000D0AAC
:10FED40025732025582025580D0A000D0A736279D0
:10FEE400746573202564000D0A4D6F756E74696E18
:10FEF4006720004170722020382032303230004CAC
:10FF04006F6164696E672E2E2E0068706469736B6E
:10FF14002E63666700466D74206578697420005B03
:10FF2400535251206F66665D0031393A31303A31AF
:10FF340037005B2532582025645D005B5352512005
:10FF44006F6E5D0048504469736B20004E6F2063F0
:10FF54006172640072633D256420002D3E202558A3
:10FF640020005458446174610044534B53454C0081
:10FF74004E414D452558004449534B2558005B4D8F
:10FF84004C415D0044454255470050524F544F0088
:10FF94005265616479002025303258007B45525205
:10FFA4007D00302E3130004946432000454F492022
:10FFB4000052454E200041544E200053525120001F
:10FFC40044415620004E444143004E5246440052A0
:10FFD4005443002025580025325800207C2000443A
:10FFE400300044310044320044330044340044358A
:0BFFF400004436004437002563000085
:020000040020DA
:10000000FF0FFF0FFF0FFF0FFF0FFF0FFF0FFF0F80
:020000040030CA
:0C0000008CFFFFFF8EFFFFFFFFFFFFFFE4
:00000001FF
